:100000000C9448200C9465200C9465200C940DA54C
:100010000C9465200C9465200C9465200C9471A3BD
:100020000C9465200C9465200C9465200C9465203C
:100030000C9465200C9465200C9465200C94684DFC
:100040000C9465200C9465200C948B390C94BA396F
:100050000C94ED390C94C9300C944E520C946520DC
:100060000C9465200C943F9C0C9465200C946520A6
:100070000C94CD8B0C9465200C9465200C94652019
:100080000C9465200C9465200C946520FFFFFFFF05
:10010000642F363B3E40424345464748494A4B4BA5
:100110004C4D4D4E4E4F4F505051515252525353E1
:100120005354545455555556565656575757575875
:10013000585858595959595A5A5A5A5A5B5B5B5B25
:100140005B5C5C5C5C5C5D5D5D5D5D5D5E5E5E5EE2
:100150005E5E5F5F5F5F5F5F6060606060606161A7
:10016000616161616162626262626263636363636F
:10017000636364646464646464656565656565653A
:100180006666666666666666676767676767676806
:10019000686868686868696969696969696A6A6AD2
:1001A0006A6A6A6A6B6B6B6B6B6B6C6C6C6C6C6C9D
:1001B0006C6D6D6D6D6D6D6E6E6E6E6E6E6F6F6F64
:1001C0006F6F707070707070717171717172727226
:1001D00072737373737374747474757575757676DE
:1001E000767777777878787979797A7A7B7B7C7C7F
:1001F0007D7D7E7E7F80818283848587898B9064EC
:1002000064FFFFFFFFFFFFFFFFFFFFFFFFFFFFFF99
:10021000FFFFFFFFFFFAF6F2EEEBE7E4E1DEDBD8EB
:10022000D6D3D1CECCCAC8C6C3C1C0BEBCBAB8B67C
:10023000B5B3B2B0AEADABAAA9A7A6A4A3A2A19F25
:100240009E9D9C9A9998979695949392908F8E8D57
:100250008C8B8A89888787868584838281807F7E4C
:100260007E7D7C7B7A797978777675747473727118
:1002700071706F6E6E6D6C6B6B6A696868676665CE
:1002800065646363626160605F5E5E5D5C5B5B5A78
:100290005959585757565555545352525150504F1B
:1002A0004E4E4D4C4C4B4A4A4948474746454544BB
:1002B0004343424140403F3E3D3D3C3B3A3A393862
:1002C00037373635343433323130302F2E2D2C2B16
:1002D0002A2A292827262524232221201F1E1D1CE7
:1002E0001B1A18171615141211100E0D0B090806FB
:1002F0000402000000000000000000000000006494
:10030000D2FFFFFFFFFFFFFFFFFFFFFFFFFFFFFF2A
:10031000FFFFFFFFFFFBF7F3EFEBE8E5E1DEDCD9E2
:10032000D6D4D1CFCCCAC8C6C4C2C0BEBCBAB9B775
:10033000B5B3B2B0AFADACAAA9A8A6A5A3A2A1A01F
:100340009E9D9C9B9A9897969594939291908F8E50
:100350008D8C8B8A89888786858483828181807F42
:100360007E7D7C7B7B7A7978777676757473727212
:1003700071706F6F6E6D6C6C6B6A696968676666C9
:1003800065646463626161605F5F5E5D5D5C5B5A72
:100390005A59585857565655545453525251504F13
:1003A0004F4E4D4D4C4B4B4A4949484747464544B3
:1003B0004443424241403F3F3E3D3D3C3B3A3A3957
:1003C00038373736353433333231302F2F2E2D2C0A
:1003D0002B2A29292827262524232221201F1E1DD8
:1003E0001C1B19181716151312110F0E0C0B0908E8
:1003F000060402000000000000000000000000D21F
:1004000072316F316C3189315A31863157319531C2
:1004100092315A3157315D318F3157315D315A3117
:100420008C31693166316331983183317531A9324C
:10043000B232B232AD3296328B32873283327F3271
:100440007B326F3262325E3256324E324832303256
:100450002C3228320E320A32FE31F931F531F231C6
:10046000F231F231F231F231F231F231F231F23174
:10047000F231F231F231F231F231F231F231EB326A
:10048000F231F231F231F231F231F231B632C631BB
:1004900071379C37A0372C372C372C372C37C43783
:1004A0002C37CB372C3726372C37D037D5372C374E
:1004B000DA372C37FE3722382C372C372C372C37AD
:1004C0002C372C372C372C372C372C372C372C3714
:1004D0002C372C372C372C372C372C372C37273808
:1004E0002C375A382C3787382C37B438E138553800
:1004F0002C372C372C3739392C370C39663905AB6A
:1005000099AB9BA986A965A964AB58AB23AB1CAB7F
:10051000B8A9ACA9C0A949A926AADFAAD3AA6AAAE0
:100520004EAAB1ABA7AB3DA9BFAB3DAA8BAB86AB87
:10053000CCAB79AB48AB11AB9FABE5ACE1ACDDAC80
:1005400045B845B845B845B8D9AC45B845B8E9ACA3
:1005500045B845B845B845B887AC45B883AC7FAC1D
:1005600045B87BAC29AC25AC45B845B845B845B8CD
:1005700045B845B845B845B845B845B845B845B893
:1005800045B845B845B845B845B820AC45B845B8B4
:1005900045B845B845B81BAC16AC11AC45B845B824
:1005A00045B845B845B845B845B845B845B845B863
:1005B00045B845B845B845B845B845B845B845B853
:1005C00045B845B845B845B845B845B845B845B843
:1005D00045B845B845B845B845B845B845B845B833
:1005E00045B845B845B845B845B845B845B845B823
:1005F00045B845B845B845B845B845B845B845B813
:1006000045B845B845B845B845B845B845B845B802
:1006100045B845B845B845B845B845B845B845B8F2
:1006200045B845B845B845B845B845B845B845B8E2
:1006300045B845B845B845B845B845B845B845B8D2
:1006400045B845B845B845B845B845B845B845B8C2
:1006500045B845B845B845B845B845B809AC45B8FA
:1006600045B845B845B845B845B845B802ACF1AC51
:100670001DAD07ADEDAC92AD77ADEDACEDAC60ADC1
:1006800049AD40AE37AE20AEEDAC0FAE6EAE57AE5C
:10069000EDACF9ADEDACEDACA3AD2FB0EDACCFAFA3
:1006A000EDACEDACEDACEDACEDACEDACEDACEDAC82
:1006B000EDACAEAFEDACEDACEDACEDACEDACA4AFF4
:1006C000EDACEDACEDACEDACEDAC99AF8CAF79AF82
:1006D000EDACEDACEDACEDACEDACEDACEDACEDAC52
:1006E000EDACEDACEDACEDACEDACEDACEDACEDAC42
:1006F000EDACEDACEDACEDACEDACEDACEDACEDAC32
:10070000EDACEDACEDACEDACEDACEDACEDACEDAC21
:10071000EDACEDACEDACEDACEDACEDACEDACEDAC11
:10072000EDACEDACEDACEDACEDACEDACEDACEDAC01
:10073000EDACEDACEDACEDACEDACEDACEDACEDACF1
:10074000EDACEDACEDACEDACEDACEDACEDACEDACE1
:10075000EDACEDACEDACEDACEDACEDACEDACEDACD1
:10076000EDACEDACEDACEDACEDACEDACEDACEDACC1
:10077000EDACEDACEDACEDACEDACEDACEDACEDACB1
:10078000EDACEDACEDACEDACEDACEDAC6EAF5AAFAD
:1007900046AF32AF1EAF0AAFF6AEE2AECEAE94B009
:1007A00082B035ADD3C1C6C1C6C1C6C1F6C1BDC1D7
:1007B000C9C1BDC1C1C1BDC1C1C1BDC1C1C1BDC131
:1007C000EFC1BDC1EBC1E7C1E3C1DFC1DBC1D6C130
:1007D000BDC1C1C1BDC1F2C1C6C1FFFFFFFF0080E5
:1007E000555500403333AB2A92240020721C9A19CD
:1007F00046175515B1134912111100100F0F390E7C
:10080000790DCD0C310CA30B210BAB0A3D0AD90994
:100810007B092509D408890842080008C20788070F
:1008200050071C07EB06BD06900666063E06180636
:10083000F405D105B00591057205550539051F056B
:100840000505EC04D504BE04A80492047E046A04E1
:10085000570444043204210410040004F003E103AB
:10086000D203C403B603A8039B038E03820376035B
:100870006A035E03530348033E03330329031F0344
:1008800016030C030303FA02F102E902E002D802A4
:10089000D002C802C102B902B202AB02A4029D0298
:1008A00096028F02890283027C02760270026A023B
:1008B00064025F02590254024E02490244023F029E
:1008C0003A02350230022B02270222021E021902CE
:1008D000150211020C02080204020002FC01F801D8
:1008E000F401F001ED01E901E501E201DE01DB01C6
:1008F000D701D401D101CE01CA01C701C401C10190
:10090000BE01BB01B801B501B201AF01AC01AA0142
:10091000A701A401A1019F019C019A0197019501E2
:10092000920190018D018B01880186018401820171
:100930007F017D017B0179017601740172017001F3
:100940006E016C016A016801660164016201600167
:100950005E015D015B0159015701550154015201CE
:1009600050014E014D014B0149014801460144012E
:100970004301410140013E013D013B013A01380183
:10098000370135013401320131012F012E012D01D2
:100990002B012A012901270126012501230122011A
:1009A00021011F011E011D011C011A01190118015D
:1009B00017011601150113011201110110010F0198
:1009C0000E010D010B010A010901080107010601D1
:1009D00005010401030102010101FF1814009090B8
:1009E0009090A505A5059D05A5055904E904A40653
:1009F000E90456454D532047656E626F617264206D
:100A000076332C2000761862185E185A184B184658
:100A10001834182F181E18000000000000000000F5
:100A2000000000000000000000131800000000009B
:100A3000000000000000000000000000000218F9A3
:100A400017F117E717DF17D717D017C817BE17AC5E
:100A500017A5179D178C17871700007417691700C3
:100A60000000000000631700000000000054174B56
:100A70001744173B172D171F170F17FC16F216E414
:100A800016DB16D216C916C016B716AB16A5169DDC
:100A90001694168B16821676166916601652164430
:100AA0001631161E1611160416F115DE15CB15B3E8
:100AB00015A915A2159B159415891572155B154579
:100AC0001538152915121506150000000000000044
:100AD0000000000000000000000000F614E814DA36
:100AE00014C414AF149D1494148C14801475146AD7
:100AF000145F14541449143A142B14201415140BB5
:100B0000140014F113E013D213C313B313A51398F5
:100B1000138513731364134F133D132C131913060A
:100B200013F312DC12CB12BA12A91294127B1270B8
:100B3000125A1249123D122B121A120E12FC11EC0B
:100B400011DA11C911B411A2118F117C1168115B56
:100B5000114E113D112A1117110411F110DD10CEA3
:100B600010BF10B110AA10A010921089107D106B48
:100B70001059104810381026101A100C10F60FE9F2
:100B80000FD50FC10FAB0F950F800F730F670F5C61
:100B90000F4A0F420F390F280F180F070FF70EE2F9
:100BA0000ECD0EBF0EB00EA20E970E890E790E69F5
:100BB0000E590E490E390E290E180E080EF80DE8C2
:100BC0000DD80DC80DB80DA70D9B0D8B0D7F0D6FAA
:100BD0000D660D560D4B0D3A0D280D1B0D0E0D011A
:100BE0000DF00CE20CD20CC50CB80CA80C950C85C1
:100BF0000C740C640C540C470C3E0C300C1F0C1184
:100C00000C050C0000736F667472706D5F72706D0E
:100C10000073686966746375745F74696D650073E9
:100C2000686966746375745F6368616E6E656C0095
:100C300073686966746375745F636F6E6600746170
:100C400063685F64697600746163685F6368616E9E
:100C50006E656C006675656C6375745F6D61785F59
:100C60006B7061006675656C6375745F6D696E5F4E
:100C70006B706100746F6F746872656C5F6D69731F
:100C800073696E6700746F6F746872656C5F6E6F06
:100C9000726D616C0077617465725F70756D705F05
:100CA0006368616E6E656C0077617465725F707504
:100CB0006D705F68797374006879627269645F72DD
:100CC000706D5F6D006879627269645F72706D5FEC
:100CD000610077617465725F70756D705F74656DCA
:100CE0007000626F6F73745F6368616E6E656C0035
:100CF000626F6F73745F7069645F696C696D69744A
:100D000000626F6F73745F7069645F6B6400626F21
:100D10006F73745F7069645F6B6900626F6F737487
:100D20005F7069645F6B7000626F6F73745F6D6991
:100D30006E707265737375726500626F6F73745F46
:100D40007461726765746F66667300626F6F737447
:100D50005F636F6E6600616C735F746B735F636873
:100D6000616E6E656C00656774315F63616C006114
:100D700063745F72706D5F6368616E6E656C006155
:100D800063745F72706D5F72706D006163745F7722
:100D90006F745F6368616E6E656C006163745F772A
:100DA0006F745F72706D006D697363326F75745F1D
:100DB0006368616E6E656C006D697363326F757424
:100DC0005F6D61786D6170006D697363326F75740A
:100DD0005F6D696E6D6170006D697363326F7574FC
:100DE0005F6D6178747073006D697363326F7574D1
:100DF0005F6D696E747073006D697363326F7574C3
:100E00005F6D617872706D006D697363326F7574B8
:100E10005F6D696E72706D006D697363316F7574AB
:100E20005F6368616E6E656C006D697363316F75C9
:100E3000745F6D61786D6170006D697363316F759A
:100E4000745F6D696E6D6170006D697363316F758C
:100E5000745F6D6178747073006D697363316F7561
:100E6000745F6D696E747073006D697363316F7553
:100E7000745F6D617872706D006D697363316F7549
:100E8000745F6D696E72706D00616C735F72657610
:100E90005F6C696D697400616C735F726574617217
:100EA0006400616C735F64656163745F656774009F
:100EB000616C735F64656163745F74696D65006123
:100EC0006C735F64656163745F72706D00696E6AF4
:100ED0005F7374616765325F73746172745F6D61B3
:100EE0007000696E6A5F7374616765325F73746105
:100EF00072745F74707300696E6A5F7374616765A2
:100F0000325F72617465006675656C70756D705FD7
:100F10006368616E6E656C0070756D705F6F6E5F9B
:100F20006D696E74696D6500656E67696E655F6F8A
:100F300066665F64656C61790069676E63686D61A0
:100F4000780069676E5F6F75740069676E5F6372C2
:100F5000616E6B5F616476616E63650069676E5F89
:100F60006477656C6C360069676E5F6477656C6C7E
:100F700031340069676E5F74646364656C61790025
:100F800072657365745F656E6770686173655F61D4
:100F9000667465720063616D5F73796E635F665F2F
:100FA000656467655F70686173650063616D5F7339
:100FB000796E635F725F656467655F7068617365B2
:100FC00000746F6F74685F776865656C5F747769CC
:100FD0006474683200746F6F74685F776865656CFD
:100FE0005F74776964746831006372616E6B5F6D02
:100FF000696E70657200616E6F746865725F74729D
:1010000069676765725F746F6F746800747269678F
:101010006765725F746F6F746800746F6F74685F78
:10102000776865656C007365636F6E646172795F84
:1010300074726967676572007072696D6172795F59
:1010400074726967676572006C63645F646566618A
:10105000756C745F7669657700616C735F72657437
:101060006172645F6D617874707300616C735F723C
:1010700065746172645F6D696E7470730069676E28
:101080005F62616C616E6365006B70615F636F6E60
:1010900066006C63645F6261636B6C6967687400AF
:1010A0006C63645F64656C6179006C63645F63307A
:1010B0000076655F6C6561726E5F636F6E66007669
:1010C000655F6C6561726E5F6C696D6974007665F1
:1010D0005F6C6561726E5F73706565640076655FF5
:1010E0006C6561726E5F6D696E5F77656967687464
:1010F0000076655F6C6561726E5F65676F5F7363D5
:10110000616C650076655F6C6561726E5F6B7061C6
:101110005F7363616C650076655F6C6561726E5FBD
:1011200072706D5F7363616C650076655F6C65619D
:10113000726E5F6D61785F706F7765720076655F64
:101140006C6561726E5F636F6F6C616E74006B6E65
:101150006F636B5F6D617872706D006B6E6F636B48
:101160005F6D696E72706D006B6E6F636B5F616453
:1011700076616E63655F64656C6179006B6E6F6349
:101180006B5F616476616E63655F73746570006B3D
:101190006E6F636B5F7265746172645F64656C61CE
:1011A00079006B6E6F636B5F7265746172645F73FD
:1011B000746570006B6E6F636B5F64656661756C00
:1011C000745F726574617264006B6E6F636B5F6DE8
:1011D00061785F726574617264006B6E6F636B5FE0
:1011E0006E6F6973655F7363616C65006B6E6F63CF
:1011F0006B5F7468726573686F6C64006B6E6F63AD
:101200006B325F696E7465677261746F72006B6ECA
:101210006F636B325F6761696E006B6E6F636B3219
:101220005F6672657175656E6379006B6E6F636B77
:10123000315F696E7465677261746F72006B6E6F97
:10124000636B315F6761696E006B6E6F636B315FFB
:101250006672657175656E6379006B6E6F636B5F47
:1012600073616D706C696E675F77696E646F77002C
:101270006B6E6F636B5F636F6E660077626F325F7A
:1012800072695F636F6E666964656E63655F7363E1
:10129000616C650077626F325F70756D705F706949
:1012A000645F696C696D69740077626F325F707535
:1012B0006D705F7069645F6B640077626F325F703E
:1012C000756D705F7069645F6B690077626F325F24
:1012D00070756D705F7069645F6B700077626F32FC
:1012E0005F6865617465725F7069645F696C696D80
:1012F00069740077626F325F6865617465725F70F0
:1013000069645F6B640077626F325F686561746502
:10131000725F7069645F6B690077626F325F6865E6
:10132000617465725F7069645F6B700077626F32C1
:101330005F63616C6962726174696F6E0077626F7E
:10134000325F70756D705F70775F7A65726F00776E
:10135000626F325F6E65726E737464635F74617224
:101360006765740077626F325F72695F746172677C
:1013700065740077626F325F6564676574696D6577
:101380005F6D696E0077626F325F6564676574696F
:101390006D655F636F72720077626F325F72657442
:1013A00072795F740077626F325F66616C6C626144
:1013B000636B0077626F325F6C696D69745F6D613A
:1013C00078740077626F325F6162735F6C696D6918
:1013D0007400616C735F72656163745F7470730035
:1013E00077626F325F7761726D75705F72616D7079
:1013F0000065676F5F7069645F77696E646F77001F
:1014000065676F5F7461726765740065676F5F64BD
:10141000656C746100616C735F656E72696368000E
:1014200065676F5F7069645F6B700065676F5F729F
:101430006963685F6C696D69740065676F5F6C658F
:10144000616E5F6C696D69740065676F5F7761726B
:101450006D75700065676F5F6D617872706D0065A6
:10146000676F5F6D696E72706D0065676F5F6D614C
:10147000786D61700065676F5F6D6178747073007F
:1014800065676F5F636F6F6C616E740065676F5F38
:101490006C61670065676F5F636F6E6600696163AB
:1014A0005F69676E5F7468726573686F6C6400690A
:1014B00061635F69676E5F7265746172645F6C69B6
:1014C0006D6974006961635F69676E5F616476610D
:1014D0006E63655F6C696D697400736F66747270BA
:1014E0006D5F72616E6765006961635F69676E5FFA
:1014F000736C6F7065006961635F736F6C5F6368C5
:10150000616E6E656C006961635F7265665F706FC6
:1015100073006961635F6F766572636C6F73655F9B
:10152000696E74657276616C00616C735F6375746B
:101530005F6D6178747073006961635F6465616495
:1015400062616E64006961635F696E746567726190
:101550006C5F6465616462616E64006961635F69A8
:101560006E74656772616C5F6C696D69745F696EDA
:1015700063006961635F696E74656772616C5F6C5B
:10158000696D69745F646563006C61756E63685F43
:1015900072706D006961635F6B64006961635F6BAA
:1015A00069006961635F6B70006961635F73706597
:1015B0006564006961635F6166746572737461720A
:1015C000745F6475726174696F6E006961635F61F5
:1015D0006674657273746172745F72706D006961B4
:1015E000635F7761726D5F73746172745F706F7344
:1015F000006961635F636F6C645F73746172745FD1
:10160000706F73006961635F7761726D5F72706D97
:10161000006961635F636F6C645F72706D00696124
:10162000635F7761726D5F69646C655F74656D702F
:10163000006961635F636F6C645F69646C655F74AC
:10164000656D70006961635F7470735F7468726563
:1016500073006961635F6D61785F737465707300B7
:101660006961635F636F6E66006961635F73746570
:10167000705F7365710066616E5F6368616E6E6551
:101680006C0066616E5F687973740066616E5F748A
:10169000656D70007470735F68696768007470735B
:1016A0005F6C6F7700646261726F00616C735F6D75
:1016B00061785F637574006661737469646C65005A
:1016C000626174745F63616C00636F6E6669673139
:1016D0003300636F6E666967313200636F6E6669EF
:1016E0006731310061697264656E5F69676E6F7240
:1016F00065007265765F6C696D6974006F766572FE
:1017000072756E5F6675656C726573756D65006F79
:1017100076657272756E5F6675656C637574006C64
:1017200061756E63685F726574617264006C617587
:101730006E63685F656E726963680074707361637D
:101740006F6C640061636D756C74007470736173A9
:10175000796E6300616C735F6375745F6D696E743D
:10176000707300747073617100747073646F74725D
:1017700061746500747073646F745F6B7061646F23
:10178000745F636F6E660072706D6B00616C735F87
:101790006C61756E63685F696E70757400696E6AFE
:1017A00070776D7400696E6A70776D00696E6A7229
:1017B000616D7075705F6261747466616300696EFB
:1017C0006A6F636675656C006B70616F6666730047
:1017D0006B70616661630062617474666163006965
:1017E0006E6A6F70656E00616C7465726E617465AF
:1017F0000064697669646572007265715F6675651B
:101800006C007761726D75705F72706D5F7363618C
:101810006C65007761726D75705F636C74007761E1
:10182000726D75705F636C745F72616E6765006185
:1018300077656300617765765F74656D705F73636C
:10184000616C696E670061776576006372616E6BCB
:10185000696E675F746872657300637768006377A9
:101860006C007072696D65705F74656D705F736335
:10187000616C696E67007072696D657000004E661C
:1018800076838D969EA5ABB1B6BBBFC3C7CBCED179
:10189000D4D7DADCDEE1E3E5E6E8EAEBEDEEF0F101
:1018A000F2F3F4F5F6F7F8F9F9FAFBFBFCFCFDFDB1
:1018B000FDFEFEFEFFFFFFFFFFFFFFFFFF01100425
:1018C00008804020100804020130313233343536AC
:1018D000373839414243444546003F3F0045727224
:1018E000007988BF88AF89BC8932897889C68968C0
:1018F0008828883A884C885A88E589068B068B06A2
:101900008B351A2B1A1F1A0F1A011AFB19EF19E13E
:1019100019CF19CD19C119B319A7199B198F197F9F
:10192000197919711967196319471A471A471A471C
:101930001A471A471A471A471A471A471A471A479F
:101940001A4B1A471A471A471A5B195319471A476D
:101950001A0000D596EB92F092000093969896C7E5
:10196000960000709400004E94599462946B940019
:1019700000FD930F943F940000DA93DF9300008AF8
:10198000945F9138935F91BF935F918C9300009720
:10199000935F91A2935F91AD9300006B935F9176FB
:1019A000935F918193000058935D935F913A9127E3
:1019B0009300008A945F915893389327935F910026
:1019C00000BB92C0926391D794DC94000000003574
:1019D000913A915F91C295D2955F91FD91029200EB
:1019E000008A945F915893389327935F910000BBCE
:1019F00092C0926391D794DC940000619647960060
:101A00000035913A915F91C295CA95D29500008AAE
:101A1000945F91E696EB965F91D794DC940000BBBF
:101A200092C0926391EB92FE9200005F9264925F8B
:101A3000917C92000035913A915F917691A1915FEE
:101A400091FD91029200005F910000E696EB9600F6
:101A500000A23D683D403D183DFB3CC73C8A3C6DC3
:101A60003C3D3C00000000000000000000000000C1
:101A700000000000000E3C0000000000000000001C
:101A8000000000000000000000CE3BB53B993B5D2C
:101A90003B373B123BE93ABB3A8A3A5C3A223AEC92
:101AA00039C439893900005C393839000000000038
:101AB000000239000000000000F338D3389C385F82
:101AC0003840381738DE37A137863751370F37DEC1
:101AD00036AC368A365F3653362D361A360736E838
:101AE00035D035B235873540352735FE34D534AC61
:101AF000348E347034533436340634DC33A7339B9D
:101B0000338F33833378335B333E330133EB32DB54
:101B100032BA3298320000000000000000000000DD
:101B20000000000000000085325E3247322032FBA8
:101B300031C731A831673136310D31E930C2309AC1
:101B400030833040301D30F52FE62FC62FAB2F8667
:101B50002F602F4E2F222FF62ECA2EA92E812E5106
:101B60002E232E042ED32DB82DA42D902D7C2D5C4C
:101B70002D4A2D382D262D082DD32CA52C702C4E1A
:101B80002C412C1F2CFD2BF02BCE2BBD2BA32B7B04
:101B90002B4F2B262B022BD82AB32A9B2A832A4988
:101BA0002A042AD529A629772947291C29DF28A60E
:101BB000285F281F280128CE2787277527632749F4
:101BC000270227BB2691265C2632260C26E825BC58
:101BD00025802543252B250825EF24CF24A3245D2C
:101BE0002433240124CA23B223812353231C23003A
:101BF00023E722C522A2227E225F22402222220443
:101C000022E121BE219D217E215F2141212321004E
:101C100021DD20BC2096207C2056203C2021200A5B
:101C200020C31F8C1F6B1F571F431F2F1F0F1FEA3F
:101C30001ECC1EA41E761E5F1E441E151EDB1DA795
:101C40001D681D411D0F1DD51CB01C8A1C7A1C531C
:101C50001C00004E6F206D6F7265207661726961A5
:101C6000626C652C20676F206261636B2C20646F4F
:101C70006E277420746F7563680049676E20536F18
:101C8000667472706D2052504D0069676E63757492
:101C90002074696D6520616674657220696E707567
:101CA0007470756C7365205B34206D7365635D00C3
:101CB0007368696674637574206D6370333230388D
:101CC000206368616E6E656C2C2064697361626C60
:101CD000653A464600626974343A736869667463AB
:101CE0007574206675656C2C20626974313A73686E
:101CF00069667463757420737061726B20626974B5
:101D0000303A72657663757420737061726B00642B
:101D1000697669646520746865207461636820660B
:101D200072657120627920582F33323B20757365BC
:101D3000204646206966206E6F74207573696E6751
:101D40000074616368207369676E616C206F7574DD
:101D5000707574206368616E6E656C2046463D64E4
:101D6000697361626C6564006375742074686520D2
:101D70006675656C2069662074686520656E6769A4
:101D80006E65206B7061206578636565647320748F
:101D90006869732076616C756520307846463D64CD
:101DA000697361626C65006675656C637574206249
:101DB000656C6F772074686973204D41502028301E
:101DC000303A64697361626C653B20313020726522
:101DD000636F6D6D656E64656429004D6D3A2074A6
:101DE000675F70726576202A2028312E3235202BCD
:101DF000206D2F3829203C3D207467203C3D207405
:101E0000675F70726576202A2028322E35202B20BD
:101E10004D2F3829004E6E3A2074675F70726576D8
:101E2000202A206E2F3136203C3D207467203C3D17
:101E30002074675F70726576202A2028312B4E2F20
:101E40003136290077617465722070756D702C20B1
:101E50006F7574707574206368616E6E656C007761
:101E6000617465722070756D702C2068797374656B
:101E70007265736973005645206D6F64653A7370BF
:101E80006565642064656E7369747920284D4150DE
:101E9000292061626F7665205B2A3130305D2052E7
:101EA000504D20005645206D6F64653A616C706836
:101EB000612D6E2028545053292062656C6F772065
:101EC0005B2A3130305D2052504D200077617465BF
:101ED000722070756D702C2073746172742074653B
:101EE0006D706572617475726500626F6F73746393
:101EF0006F6E74726F6C20736F6C656E6F696420A7
:101F00006F7574707574206368616E6E656C0062C5
:101F10006F6F7374636F6E74726F6C20706964207E
:101F2000696E74656772616C206C696D69740062BA
:101F30006F6F7374636F6E74726F6C20706964205E
:101F40006B6400626F6F7374636F6E74726F6C207A
:101F5000706964206B6900626F6F7374636F6E7475
:101F6000726F6C20706964206B70006163747561BE
:101F7000746F72204F46462062656C6F77207468DC
:101F8000697320707265737375726500626F6F7329
:101F900074636F6E74726F6C207461726765742005
:101FA0006F6666736574206170706C69656420612A
:101FB0006674657220625B52504D5D2A745B5450AA
:101FC000535D00626F6F7374636F6E74726F6C2019
:101FD000626974373A342050574D20706572696FCA
:101FE00064205B386D7365635D3B20626974333ACE
:101FF0006269743220726566706F733B2062697427
:102000003020303A626F6F737400414C5320544B50
:1020100053206F7574707574206368616E6E656CA3
:10202000004547542063616C6962726174696F6E28
:10203000206D756C7469706C6965720052504D202A
:10204000737769746368206F757470757420636842
:10205000616E6E656C0052504D20737769746368D1
:102060002052504D207468726573686F6C6420282C
:1020700046463D64697361626C652900574F542080
:10208000737769746368206F757470757420636802
:10209000616E6E656C00574F542073776974636886
:1020A0002052504D207468726573686F6C642028EC
:1020B00046463D64697361626C6529006D697363AE
:1020C000326F75742C6F7574707574206368616EEF
:1020D0006E656C2073656C6563746F72006D6973F7
:1020E00063326F75742C6D6178696D756D206D61EB
:1020F0006E69666F6C6420707265737375726500CB
:102100006D697363326F75742C6D696E696D756D71
:10211000206D616E69666F6C642070726573737593
:102120007265006D697363326F75742C6D617869C7
:102130006D756D2074707320706F736974696F6E44
:10214000006D697363326F75742C6D696E696D759E
:102150006D2074707320706F736974696F6E006D99
:10216000697363326F75742C6D6178696D756D205C
:1021700072706D205B3130302072706D5D006D6962
:102180007363326F75742C6D696E696D756D207235
:10219000706D205B3130302072706D5D006D697341
:1021A00063316F75742C6F7574707574206368611A
:1021B0006E6E656C2073656C6563746F72006D691B
:1021C0007363316F75742C6D6178696D756D206DF9
:1021D000616E69666F6C6420707265737375726589
:1021E000006D697363316F75742C6D696E696D75FF
:1021F0006D206D616E69666F6C64207072657373BB
:10220000757265006D697363316F75742C6D6178DB
:10221000696D756D2074707320706F736974696F68
:102220006E006D697363316F75742C6D696E696DC5
:10223000756D2074707320706F736974696F6E00B0
:102240006D697363316F75742C6D6178696D756D2F
:102250002072706D205B3130302072706D5D006DCA
:10226000697363316F75742C6D696E696D756D205E
:1022700072706D205B3130302072706D5D00526580
:1022800076206C696D6974207768656E20414C53C7
:1022900020616374697665205B3130302072706D27
:1022A0005D00616C732C6D61782069676E2E207201
:1022B0006574617264205B312F34206372616E6BD0
:1022C0006465675D00616C732C7377697463686F14
:1022D000666620656774205B3520646567206365EA
:1022E0006C736975735D00616C732C7377697463CB
:1022F000686F66662074696D65205B7365635D0059
:10230000616C732C7377697463686F666620727092
:102310006D205B3130302072706D5D007365636FCE
:102320006E6461727920696E6A6563746F7273207E
:102330006F70656E2061626F766520676976656E85
:10234000206D616E69666F6C642070726573737561
:102350007265007365636F6E6461727920696E6A7D
:102360006563746F7273206F70656E2061626F7643
:102370006520676976656E207468726F74746C6529
:10238000007365636F6E6461727920696E6A65635C
:10239000746F7273207261746520746F2063616C56
:1023A00063756C61746564207077205B302E342512
:1023B0005D006675656C70756D70206F75747075F5
:1023C00074206368616E6E656C006D696E696D7511
:1023D0006D2074696D6520746F206C656176652071
:1023E0006675656C70756D70206F6E2061742073FA
:1023F000746172747570205B3236326D7365635D23
:10240000007475726E206F6666206675656C7075F7
:102410006D7020616674657220696E61637469769F
:102420006974792074696D65205B3236326D73652D
:10243000635D00685B325D206D6178696E6465780C
:1024400020666F722069676E6974696F6E206368B9
:10245000616E6E656C206C6F6F6B757000454449E2
:10246000533A3078303F2064756D6D793A2030787A
:10247000373F2064697361626C653A307866662024
:10248000626974313A2069676E5F6475616C5F6F71
:10249000757420626974303A20696E766572746F63
:1024A00075740069676E6974696F6E206164766126
:1024B0006E6365206174206372616E6B696E672064
:1024C0005B302E32356372616E6B6465675D0061EF
:1024D00064646564206477656C6C2074696D652044
:1024E000617420365620283237757365632900647D
:1024F00077656C6C2061626F7665203134562028D8
:1025000036347573656329005444432061667465ED
:102510007220746865207472696767657228302E4E
:10252000356372616E6B6465672900656E677068FC
:102530006173652C207768656E20746F20726573F7
:1025400065740063616D2073796E632C2066616C25
:102550006C696E6720656467652C20656E67696EBF
:1025600065207068617365206174206E65787420E1
:102570007072696D61727920747269676765720043
:1025800063616D2073796E632C20726973696E6765
:1025900020656467652C20656E67696E65207068CC
:1025A000617365206174206E657874207072696D46
:1025B000617279207472696767657200746F6F74F5
:1025C0006820776865656C2C20616E67756C617238
:1025D000207769647468206F66206D697373696E13
:1025E0006720746F6F746800746F6F746820776809
:1025F00065656C2C20616E67756C6172207769640B
:102600007468206F6620746F6F7468004372616E27
:102610006B74696767657220706572696F64206D9D
:10262000696E696D756D20282A3136207573656372
:102630002900746F6F746820776865656C2C20645E
:102640006566696E6520616E6F746865722074726C
:10265000696767657220746F6F746800746F6F7458
:102660006820776865656C2C2061637469766520E5
:102670007472696767657220746F6F7468202830A0
:10268000303A6D697373696E6720746F6F7468296F
:1026900000746F6F746820776865656C2C206E75A8
:1026A0006D626572206F66207465657468206F6E58
:1026B0002074686520776865656C00747269676767
:1026C0006572322C206269743020303A66616C6C1D
:1026D000696E672F313A726973696E672C2062697F
:1026E000743120303A656E61626C652F313A6469ED
:1026F0007361626C652C206269743220313A6669BC
:102700006C0074726967676572312C20626974307D
:1027100020303A66616C6C696E672F313A7269736A
:10272000696E672C206269743120303A746F6F745F
:1027300068776865656C2F313A636F696C2C20622D
:1027400069743220303A6E6F004C43442C2064652B
:102750006661756C742072756E74696D652076693A
:10276000657700414C5320726574617264206D611D
:102770007874707300414C532072657461726420E8
:102780006D696E7470730069676E6974696F6E202D
:1027900062616C616E6365205B302E3235637261FD
:1027A0006E6B6465675D2C20646564756374656435
:1027B0002066726F6D20616476616E636520746F50
:1027C000206D6F7665207A65726F20706F00626988
:1027D00074372D343A206B70616661635F756E6982
:1027E000742C20626974332D303A206B70615F6302
:1027F0006F6E6669675F7265736F6C7574696F6E13
:10280000004C4344206261636B6C696768743A20D2
:1028100046462069732066756C6C79206F6E004C9B
:1028200043442D6361626C656C656E6774682064F7
:10283000656C6179732048696768657268616C6668
:102840003A6265666F7265454E61626C65204C6FD9
:1028500077657248616C663A454E61626C65004C02
:10286000434420666C61677320353A207377206299
:1028700072696768746E65737320343A2070776D7F
:10288000206272696768746E65737320333A72658B
:10289000696E697420313A6C63645F65617379674E
:1028A0006F746F2030005645206C6561726E2C206D
:1028B000636F6E6669672C20626974303A656E6179
:1028C000626C6520626974313A73696D756C61740C
:1028D0006520626974323A20327832626F7800562D
:1028E00045206C6561726E2C206D61782064657680
:1028F000696174696F6E20282B2F2D205B302E3478
:10290000255D292066726F6D207265666572656E41
:102910006365205645207461626C65005645206CE5
:102920006561726E2C207370656564206F6620632C
:1029300068616E67657320746F2074686520564502
:10294000207461626C65005645206C6561726E2C66
:10295000206D696E696D756D207765696768742093
:10296000666F72206D6F64696679696E672056457F
:1029700020656E747279005645206C6561726E2C0C
:102980002065676F207363616C696E6720666163A1
:10299000746F722028735E32203C203235352F73DD
:1029A00063616C6529005645206C6561726E2C2050
:1029B0006B7061207363616C696E6720666163741C
:1029C0006F722028735E32203C203235352F7363BE
:1029D000616C6529005645206C6561726E2C207211
:1029E000706D207363616C696E6720666163746FDC
:1029F000722028735E32203C203235352F7363619C
:102A00006C6529005645206C6561726E2C206175DD
:102A1000746F206D6F64696669636174696F6E209D
:102A20006F6620564520656E747279206F6E6C79E2
:102A30002062656C6F7720706F7765723D6D617095
:102A40002A72706D2F323536005645206C656172E2
:102A50006E2C206D696E20636F6F6C616E742066E2
:102A60006F72206175746F206D6F64696669636150
:102A700074696F6E206F6620564520656E747269AA
:102A80006573006B6E6F636B2C206D6178207270C4
:102A90006D205B31303072706D5D006B6E6F636BFB
:102AA0002C206D696E2072706D205B313030727039
:102AB0006D5D006B6E6F636B2C2069676E69746966
:102AC0006F6E20616476616E63652064656C617908
:102AD000205B31356D735D006B6E6F636B2C20690D
:102AE000676E6974696F6E20616476616E636520DC
:102AF00073746570205B312F34206465677265657F
:102B00005D006B6E6F636B2C2069676E6974696F13
:102B10006E207265746172642064656C6179205BFB
:102B200031356D735D006B6E6F636B2C2069676E62
:102B30006974696F6E207265746172642073746564
:102B400070205B312F34206465677265655D006BB2
:102B50006E6F636B2C2064656661756C74206967A9
:102B60006E6974696F6E20726574617264205B3186
:102B70002F34206465677265655D006B6E6F636BF3
:102B80002C206D61782069676E6974696F6E2072A0
:102B90006574617264205B312F34206465677265EF
:102BA000655D006B6E6F636B2C206E6F69736520C3
:102BB0007363616C6520666163746F72006B6E6F26
:102BC000636B2C207468726573686F6C64006B6E45
:102BD0006F636B322C20696E746567726174696F04
:102BE0006E2074696D6520636F6E7374616E74001E
:102BF0006B6E6F636B322C206761696E006B6E6F5A
:102C0000636B322C2062616E647061737320636544
:102C10006E746572206672657175656E6379006B9E
:102C20006E6F636B312C20696E74656772617469B5
:102C30006F6E2074696D6520636F6E7374616E745E
:102C4000006B6E6F636B312C206761696E006B6E79
:102C50006F636B312C2062616E64706173732063EB
:102C6000656E746572206672657175656E63790054
:102C70006B6E6F636B2C2073616D706C696E672077
:102C800077696E646F77205B342064656772656571
:102C90005D206C656E6774683A7374617274284164
:102CA00054444329006B6E6F636B2C20636F6E6618
:102CB00069672E206269743020313A656E61626CFA
:102CC0006520626974313A20303A6368616E6E65DE
:102CD0006C300077626F322C20526920636F6E6611
:102CE0006964656E6365207363616C696E672066F5
:102CF0006163746F722028735E32203C2032353558
:102D00002F7363616C65290077626F322C207075B8
:102D10006D702070696420696E74656772616C20E3
:102D20006C696D69740077626F322C2070756D70FC
:102D300020706964206B640077626F322C2070759C
:102D40006D7020706964206B690077626F322C208F
:102D500070756D7020706964206B700077626F32DF
:102D60002C206865617465722070696420696E74D6
:102D7000656772616C206C696D69740077626F328F
:102D80002C2068656174657220706964206B640032
:102D900077626F322C206865617465722070696497
:102DA000206B690077626F322C20686561746572F0
:102DB00020706964206B700077626F322C20636131
:102DC0006C6962726174696F6E20636F6E73746197
:102DD0006E740077626F322C2070756D70207A658A
:102DE000726F20647574796379636C6520286465FB
:102DF0006661756C743A20363629205B35562F3261
:102E000035365D0077626F322C20746172676574AD
:102E1000206E65726E73744443205B35562F3235D5
:102E2000365D0077626F322C2074617267657420A2
:102E30005269202870756C736520616D706C6974BF
:102E40007564653A4333295B35562F343039365D26
:102E50000077626F322C20736D616C6C6572206537
:102E600064676574696D657320617265206E65675E
:102E70006C6563746564205B302E35757365635DC6
:102E80000077626F322C206564676574696D652018
:102E9000636F7272656374696F6E20636F6E7374B3
:102EA000616E7420432F52200077626F322C2072A3
:102EB0006574727920636F6E74726F6C20616674D2
:102EC0006572205B347365635D0077626F322C201E
:102ED00066616C6C6261636B20562061667465721A
:102EE000206D617874205B31633D31305620666619
:102EF0003D3330565D0077626F322C206D61782053
:102F000074696D65207370656E74206174206162F0
:102F1000735F6C696D6974205B3236326D73656303
:102F20005D0077626F322C20686561746572206184
:102F300062736F6C757465206C696D6974205B32A7
:102F4000613D3132562066663D3330565D00414C5E
:102F50005320747073207468726573686F6C6400BA
:102F600077626F322C207761726D75702072616D9F
:102F700070207370656564205B33663D302E325679
:102F80002F7365635D0065676F2C206D696E696DD9
:102F9000756D2077696E646F7720666F7220706937
:102FA0006420746F2072656163740065676F2C2004
:102FB00074617267657420766F6C74616765202830
:102FC0004E424F32290065676F2C20737465702064
:102FD00073697A65202870657263656E7429205B59
:102FE000302E34255D00414C5320656E7269636854
:102FF0006D656E740065676F2C20696E6372656421
:1030000069626C65207370656564206C696D6974B4
:1030100020286F7220706964206B70290065676FCB
:103020002C206D61782070657263656E7420746FFA
:103030002072696368206166725B302E34255D0002
:1030400065676F2C206D61782070657263656E74A2
:1030500020746F206C65616E206166725B302E3467
:10306000255D28696E2053494E474C455F544152B7
:10307000474554206D6F6465207269636820746FE2
:103080006F290065676F2C207761726D75702074F1
:10309000696D65205B7365635D0065676F2C206DEE
:1030A00061782072706D20666F72204F3220636FDE
:1030B0007272656374696F6E205B31303072706D4F
:1030C0005D0065676F2C206D696E2072706D2066E3
:1030D0006F722065676F20656E61626C696E672034
:1030E0005B31303072706D5D0065676F2C206D61F3
:1030F00078206D617020666F72204F3220636F728E
:1031000072656374696F6E5B6B50615D0065676FBC
:103110002C206D61782074707320706F73697469EE
:103120006F6E20666F722065676F20636F727265C5
:103130006374696F6E0065676F2C206D696E206324
:103140006F6F6C616E742074656D706572617475FB
:10315000726520666F722065676F20656E61626CB4
:10316000696E675B465D0065676F2C2074696D65ED
:10317000636F6E7374616E742028656E67696E6527
:10318000206379636C65732920666F7220636861C0
:103190006E67696E6720636F7272656374696F6EC4
:1031A00020666163746F720065676F2C20626974BA
:1031B000353A4E424F325F61646337206269743042
:1031C0003A5049442020006961632C20746872657C
:1031D00073686F6C6420666F7220616374697661D6
:1031E00074696E672061697220636F6E74726F6CB0
:1031F000205B302E32356465675D006961632C2089
:1032000069676E6974696F6E20726574617264209B
:103210006C696D6974205B302E32356465675D00C2
:103220006961632C2069676E6974696F6E206164DF
:1032300076616E6365206C696D6974205B302E3237
:10324000356465675D200049676E6974696F6E203B
:10325000536F667452504D2072616E6765006961EC
:10326000632C2069676E6974696F6E206164766192
:103270006E6365205B302E32356465672F323536DC
:1032800072706D5D00696163206F75747075742074
:103290006368616E6E656C006961632C207265669F
:1032A0006572656E636520706F736974696F6E20F7
:1032B00028666E2074656D7029006961632C207327
:1032C00065636F6E6473206265747765656E206FE9
:1032D000766572636C6F73696E67006961632C2039
:1032E000637574206D6178747073006961632C205C
:1032F0006465616462616E64205B312072706D5D33
:10330000006961632C20696E74656772616C20646A
:1033100065616462616E64205B312072706D5D2056
:10332000286265696E672074657374656420666FD2
:10333000722075736566756C6E65737329006961BB
:10334000632C20696E74656772616C20696E6372AC
:1033500065617365206C696D6974006961632C2017
:10336000696E74656772616C206465637265617310
:1033700065206C696D6974004C61756E63682052DC
:10338000504D006961632C20442D7465726D006995
:1033900061632C20492D7465726D006961632C2076
:1033A000502D7465726D006961632C2061637475C2
:1033B00061746F7220312F6672657175656E637905
:1033C000205B6D7365635D202870776D2F73746566
:1033D000707065723A2B342F2B3129006961632C90
:1033E000206475726174696F6E206F662061667407
:1033F000657273746172742072706D205B302E314F
:10340000207365635D006961632C20616674657279
:1034100073746172742072706D205B313020727031
:103420006D5D2C20616464656420746F2069646C38
:10343000652072706D006961632C206372616E6B30
:1034400020706F736974696F6E206174203137303A
:103450002046006961632C206372616E6B20706F7F
:10346000736974696F6E206174202D3430204600BA
:103470006961632C2069646C652072706D20287707
:1034800061726D29205B31302072706D5D00696161
:10349000632C2069646C652072706D2028636F6CEA
:1034A0006429205B31302072706D5D006961632C8E
:1034B000206D696E2074656D7065726174757265DA
:1034C00020666F72207761726D2069646C6520736D
:1034D00070656564006961632C206D617820746596
:1034E0006D706572617475726520666F7220636FAE
:1034F0006C642069646C6520737065656400696143
:10350000632C20656E67696E652E7470732076611A
:103510006C756520666F722069646C6520746872D2
:103520006573686F6C64006961632C206D6178203D
:10353000737465707320746F20657874656E6400B1
:103540006961632C20626974373A736F66746964C9
:103550006C6520626974363A6173796D20626974B2
:10356000353A6475616C736F6C20626974343D31F7
:103570003A69676E616476204F4E2C20626974331D
:103580003A7072656369006961632C2073746570B9
:1035900070696E672073657175656E636520286458
:1035A0006566696E652069616320776972696E6717
:1035B0002900636F6F6C616E742066616E2C206FE2
:1035C00075747075742073656C656374696F6E00D3
:1035D000636F6F6C616E742066616E2C2068797306
:1035E0007465726573697300636F6F6C616E7420CC
:1035F00066616E2C2073746172742074656D7065E1
:10360000726174757265007470732C206D6178201E
:103610006164632D636F756E74007470732C206D1C
:10362000696E206164632D636F756E74006D6178DF
:1036300020646966666572656E636520696E2062E6
:1036400061726F6D657472696320707265737375F2
:10365000726500414C53206D61782063757400469B
:1036600061737469646C652076616C7665206F6641
:10367000662061626F766520746869732054656D99
:10368000705B2E2E462D34305D00564261747420DE
:1036900063616C6962726174696F6E2061707072CF
:1036A0002E42433D64656661756C74006331332C52
:1036B00020626974333A6261726F20626974323ACF
:1036C000616C7068616E20626974313A57424F32A2
:1036D00020626974303A6F646466697265006331B0
:1036E000322C20626974372D343A696E6A6E756DBA
:1036F00020626974332D323A4D41547479706520DB
:10370000626974312D303A434C54747970650063AA
:1037100031312C20626974372D343A6E63796C2D07
:103720003120626974333A54424920626974323AF2
:10373000327374726F6B6520626974303A303D6D1C
:103740007078343131352F313D6D70783432353009
:103750000046616B652061697264656E7369747996
:10376000206C6F77206C696D697420286C6F7720EE
:1037700072706D206F6E6C79292C20303D3D64692C
:103780007361626C6500526576206C696D697420A6
:10379000286861726429205B3130302072706D5D61
:1037A000004F76657272756E206675656C72657312
:1037B000756D652C20696E6A6563746F7273207213
:1037C00065656E61626C65642062656C6F772074FC
:1037D000686973205B3130302072706D5D004F7608
:1037E000657272756E206675656C6375742C2069E0
:1037F0006E6A6563746F72732064697361626C656D
:10380000642061626F76652074686973205B313073
:10381000302072706D5D006C61756E63682C20667F
:10382000697865642069676E2E20726574617264C0
:10383000205B312F34206372616E6B6465675D00BD
:103840006C61756E63682C206675656C20656E72A0
:103850006963686D656E74205B302E34255D0043AE
:103860006F6C6420616363656C65726174696F6E0F
:1038700020616464656420616D6F756E74202861D9
:1038800074202D3430204620646567726565732985
:10389000205B31303020757365635D004163636583
:1038A0006C65726174696F6E20636F6C64206D75F6
:1038B0006C7469706C69636174696F6E20666163B2
:1038C000746F722C206269617365642061742031A9
:1038D000303000416363656C65726174696F6E209E
:1038E0006475726174696F6E205B302E3120736570
:1038F000635D00414C5320637574206D696E747074
:1039000073005450532F4D4150444F542061636312
:10391000656C65726174696F6E20616D6F756E7430
:103920002028666E20545053444F5429205B313078
:103930003020757365635D005450532F4D415044E2
:103940004F5420616363656C65726174696F6E20AA
:1039500062696E732C2064762F647400303A2054B0
:103960005053444F542C20313A204D4150444F5431
:1039700020616363656C65726174696F6E20656E4A
:10398000726963686D656E7400436F6E7374616E07
:103990007420666F722063616C63756C6174696E0C
:1039A000672C2072706D203D2031322C3030302F4A
:1039B0006E63796C2028303A2068696768206279E4
:1039C00074652900414C5320616E64206C61756EF2
:1039D00063682061637469766174696F6E20696ED3
:1039E000707574206368616E6E656C00496E6A65FF
:1039F00063746F722050574D2074696D6520617437
:103A000020776869636820746F20616374697661E8
:103A100074652070776D205B31303020757365637D
:103A20005D00496E6A6563746F722050574D206463
:103A3000757479206379636C6520287768656E20DA
:103A400063757272656E74206C696D6974696E67F6
:103A5000206973206163746976652900696E6A65FF
:103A600063746F722072616D70757020736C6F700B
:103A700065206261747465727920646570656E6436
:103A8000656E6365202846462900696E6A65637421
:103A90006F72206F70656E696E672065666665631C
:103AA000746976652072616D7075702074696D65DA
:103AB000205B323420757365635D004D4150207387
:103AC00069676E616C206F66667365742065672E2A
:103AD00030784138202D33322E2E2B33326B50610B
:103AE000205B32353050615D004D41502072616E77
:103AF0006765205B326B50615D20303A20757365DD
:103B000020412F42206C6F6F6B7570207461626C66
:103B10006500426174746572792067616D6D612022
:103B2000666163746F72205B313620757365632044
:103B300062617365645D00496E6A6563746F7220CB
:103B40006F70656E2074696D652061742031332E4D
:103B50003256205B313620757365635D00416C74AD
:103B600065726E61746520696E6A6563746F722038
:103B7000647269766572732C206269743420313AFC
:103B800062617463682066697265207768656E207B
:103B90006372616E6B696E67004952512064697689
:103BA00069646520666163746F7220666F7220704D
:103BB000756C7365004675656C20636F6E73746118
:103BC0006E7420287265715F6675656C2900576197
:103BD000726D757020656E726963686D656E7420B4
:103BE0007363616C657220617420686967686573CE
:103BF000742072706D2062696E3A2046463D727084
:103C00006D20696E646570656E64656E74005761E1
:103C1000726D757020656E726963686D656E742073
:103C200062696E7328666E2074656D70292C20623F
:103C300069617365642061742031303000576172AE
:103C40006D75702074656D70657261747572652034
:103C500072616E6765206F662062696E7320282B23
:103C600034302046206F666673657429004166749F
:103C7000657273746172742074696D6520283620D2
:103C80006372616E6B72657629004166746572734A
:103C900074617274207761726D7570207363616CEA
:103CA000696E672061742031373046202838303DF6
:103CB00068616C662C2066663D73616D652061737A
:103CC00020636F6C6429004166746572737461725D
:103CD00074207761726D757020656E726963686DAE
:103CE000656E74202870657263656E742C20616443
:103CF0006465642076616C756529004372616E6B42
:103D0000696E67207468726573686F6C64205B31DC
:103D100030302072706D5D004372616E6B696E674A
:103D20002070756C73657769647468205B3130301E
:103D300020757365635D2061742031373020460043
:103D40004372616E6B696E672070756C736577691D
:103D5000647468205B31303020757365635D206169
:103D600074202D34302046005072696D696E6720D2
:103D700070756C7365207363616C696E6720617424
:103D8000203137302046202838303D68616C662C61
:103D90002066663D73616D6520617320636F6C649E
:103DA00029005072696D696E672070756C736520AB
:103DB0006174202D34302046205B31303020757303
:103DC00065635D00562E452E4D2E532E00466972BA
:103DD0006D776172653A2000312E302E3533002028
:103DE0005570646174696E67204669726D7761729F
:103DF00065200052504D3A00202000202020202035
:103E000000540050004F32253D004F323A302E0012
:103E100065676F433A0065676F433A00636C743AB5
:103E200000207470733A0070773A006D617800700A
:103E30006F733A20006469723A20006961633A0046
:103E400020616374697665002020202020202000F6
:103E50005645206C6561726E3A0020616374697624
:103E600065002073696D0064633A006164763A000E
:103E70003F3F006477656C6C3A00446164763A2099
:103E80002000446477656C6C3A0047616D65206F73
:103E90007665722C20696E736572742031204575C9
:103EA000726F20746F20706C6179207468652022B5
:103EB00074756E652D7468652D656E67696E652015
:103EC00067616D652220616761696E2E2E2E00622A
:103ED0006F6F7374205467742000204D415000654B
:103EE00067743A00453A0074630020706F733D00B8
:103EF0002076616C3D0000F900F5F3F1F2FC00FA68
:103F0000F8F6F409A70000A20000A151210000006A
:103F10005A53415722000043584445A4230000202F
:103F2000564654522500004E42484759260000008C
:103F30004D4A552F2800003B4B494F3D2900003A80
:103F40005F4CD8503F000000C600C5600000000074
:103F50000D5E002A0000003E000000000800003155
:103F6000003437000000302C323536380100FB2B8E
:103F7000332D2A39000000F900F5F3F1F2FC00FAC4
:103F8000F8F6F4097C0000A20000A17131000000E5
:103F90007A736177320000637864653433000020FF
:103FA000766674723500006E6268677936000000CC
:103FB0006D6A75373800002C6B696F303900002E40
:103FC0002D6CF8702B000000E600E55C000000009E
:103FD0000DA800270000003C000000000800003190
:103FE000003437000000302C323536380100FB2B0E
:103FF000332D2A390000312E302E35330A00547506
:1040000065204170722032342031363A34373A30EC
:104010003820474D5420323030370A0048656C6CE8
:104020006F3E0D0A004F4B0D0A004F4B0D0A004D1D
:10403000454E555F63616E004279650D0A00596512
:10404000732C206D656E7520616E6420636F6D6DDD
:1040500020776F72780D0A004F4B0D0A004F4B0D01
:104060000A00444BB045E240B23C0539C335DB326F
:104070003F30E52DC22BD02909286626E524802370
:10408000362202210000003F0210F7022D15020225
:1040900011241FBECFEFD0E1DEBFCDBF11E0A0E005
:1040A000B1E0E6E3FBE801E00BBF02C007900D9230
:1040B000AA33B107D9F719E0AAE3B1E001C01D9214
:1040C000AC32B107E1F70C94352A0C9400008091D2
:1040D000A1062091A006883010F4223030F42091FF
:1040E00020032B77209320030895809120039927A4
:1040F00083709070039781F08091200399278370DB
:104100009070029799F1A058B14028F0B091200327
:10411000B360B093200308954F3F5105E0F730910D
:104120002003315030932003332721FF05C04091F5
:10413000200344604093200324FF05C050912003D6
:104140005068509320038091D5079091D607782F1F
:104150006627E091D307F091D407AF2FBB276A2BD6
:104160007B2B709311026093100208959091A20628
:10417000692F7727FB01EE0FFF1FEE0FFF1F8091C6
:10418000D5079091D607382F22278091D307909199
:10419000D407892F9927282B392B809110029091D1
:1041A0001102A901481B590B4E175F0708F4B3CF42
:1041B000660F771F660F771F660F771F64177507E7
:1041C00050F43093110220931002709120037877FD
:1041D0007093200398CF8E0F9F1F909311028093AE
:1041E0001002F3CF80915C0890915D08892B39F41F
:1041F00090910A02987F2BB32770922B9BBB089556
:104200008FE08BBBF8EFFABBE3E6E8BBBCEFB7BBD4
:10421000A0EEA5BB9FE194BB7FEE72BB60E161BBEA
:104220005FEA53B948E142B910926200109261000E
:1042300035E0309365002BE1209364008998919AD2
:104240008898909ABF9A80916C0680FF5DC0C79A4B
:1042500020910A022F7E20930A020E94D08262EAF5
:1042600078E080E00E94E89B10920A020E945F4D75
:104270000E94268D0E94793960E082EA98E00E94CF
:1042800016A980ED98E00E944BB88DEA98E00E9454
:104290004BB80E94514F80E00E94944E509194067A
:1042A000452F407F5F70252F33272230310509F4D9
:1042B00050C02330310554F12630310509F448C788
:1042C0002730310509F062C0842F992780779070DC
:1042D00095958795959587959595879595958795C6
:1042E00021E030E002C0220F331F8A95E2F7F2B1DD
:1042F000F22BF2B947FF02C00C94ED29522F5095D2
:1043000083B1852383B942C0C798A2CF2115310557
:1043100009F4E9C521303105C9F5842F9927807743
:104320009070959587959595879595958795959591
:10433000879502C0220F331F8A95E2F767B3622B7D
:1043400067BB47FDC4C7722F709588B3872388BBAE
:104350001DC0842F992780779070959587959595A6
:104360008795959587959595879521E030E002C0D2
:10437000220F331F8A95E2F794B3922B94BB47FD2B
:1043800098C7A22FA09585B38A2385BB809110067C
:10439000482F407F8F70282F33272230310509F4B2
:1043A0004FC02330310524F52115310509F47DC5B1
:1043B0002130310509F061C0842F992780779070F2
:1043C00095958795959587959595879595958795D5
:1043D00002C0220F331F8A95E2F767B3622B67BBD7
:1043E00047FD79C7722F709588B3872388BB45C076
:1043F0002630310509F4CAC62730310509F03DC021
:10440000842F9927807790709595879595958795B6
:10441000959587959595879521E030E002C0220F0C
:10442000331F8A95E2F7F2B1F22BF2B947FF02C0CF
:104430000C94FA29522F509583B1852383B91DC05E
:10444000842F992780779070959587959595879576
:10445000959587959595879521E030E002C0220FCC
:10446000331F8A95E2F794B3922B94BB47FD0CC798
:10447000A22FA09585B38A2385BB80918C06482FF7
:10448000407F8F70282F33272230310509F44CC02C
:104490002330310524F52115310509F47EC521307D
:1044A000310509F05EC0842F99278077907095952B
:1044B000879595958795959587959595879502C04C
:1044C000220F331F8A95E2F767B3622B67BB47FD64
:1044D00006C7722F709588B3872388BB42C02630E9
:1044E000310509F471C627303105D9F5842F992794
:1044F00080779070959587959595879595958795F3
:104500009595879521E030E002C0220F331F8A95F0
:10451000E2F7F2B1F22BF2B947FD7CC7522F50956A
:1045200083B1852383B91DC0842F9927807790702C
:104530009595879595958795959587959595879563
:1045400021E030E002C0220F331F8A95E2F794B3D6
:10455000922B94BB47FD95C6A22FA09585B38A23C5
:1045600085BB80918606482F407F8F70282F332788
:104570002230310509F44CC02330310524F52115D2
:10458000310509F4ECC42130310509F05EC0842FF7
:1045900099278077907095958795959587959595AE
:1045A00087959595879502C0220F331F8A95E2F76C
:1045B00067B3622B67BB47FD9AC6722F709588B3AD
:1045C000872388BB42C02630310509F42BC527302C
:1045D0003105D9F5842F9927807790709595879527
:1045E00095958795959587959595879521E030E0E8
:1045F00002C0220F331F8A95E2F7F2B1F22BF2B913
:1046000047FDE7C6522F509583B1852383B91DC05E
:10461000842F9927807790709595879595958795A4
:10462000959587959595879521E030E002C0220FFA
:10463000331F8A95E2F794B3922B94BB47FD3CC697
:10464000A22FA09585B38A2385BB80917F06482F32
:10465000407F8F70282F33272230310509F44CC05A
:104660002330310524F52115310509F45AC42130D0
:10467000310509F05EC0842F992780779070959559
:10468000879595958795959587959595879502C07A
:10469000220F331F8A95E2F767B3622B67BB47FD92
:1046A00022C6722F709588B3872388BB42C02630FC
:1046B000310509F4D5C427303105D9F5842F992760
:1046C0008077907095958795959587959595879521
:1046D0009595879521E030E002C0220F331F8A951F
:1046E000E2F7F2B1F22BF2B947FD8CC6522F50958A
:1046F00083B1852383B91DC0842F9927807790705B
:104700009595879595958795959587959595879591
:1047100021E030E002C0220F331F8A95E2F794B304
:10472000922B94BB47FDB6C5A22FA09585B38A23D3
:1047300085BB80918A06482F407F8F70282F3327B2
:104740002230310509F44CC02330310524F5211500
:10475000310509F48CC32130310509F05EC0842F86
:1047600099278077907095958795959587959595DC
:1047700087959595879502C0220F331F8A95E2F79A
:1047800067B3622B67BB47FD9EC5722F709588B3D8
:10479000872388BB42C02630310509F433C5273052
:1047A0003105D9F5842F9927807790709595879555
:1047B00095958795959587959595879521E030E016
:1047C00002C0220F331F8A95E2F7F2B1F22BF2B941
:1047D00047FDFBC5522F509583B1852383B91DC07A
:1047E000842F9927807790709595879595958795D3
:1047F000959587959595879521E030E002C0220F29
:10480000331F8A95E2F794B3922B94BB47FD48C5BA
:10481000A22FA09585B38A2385BB80918806482F57
:10482000407F8F70282F33272230310509F44CC088
:104830002330310524F52115310509F4DCC221307E
:10484000310509F05EC0842F992780779070959587
:10485000879595958795959587959595879502C0A8
:10486000220F331F8A95E2F767B3622B67BB47FDC0
:1048700026C5722F709588B3872388BB42C0263027
:10488000310509F429C427303105D9F5842F99273A
:10489000807790709595879595958795959587954F
:1048A0009595879521E030E002C0220F331F8A954D
:1048B000E2F7F2B1F22BF2B947FDA0C5522F5095A5
:1048C00083B1852383B91DC0842F99278077907089
:1048D00095958795959587959595879595958795C0
:1048E00021E030E002C0220F331F8A95E2F794B333
:1048F000922B94BB47FDCBC4A22FA09585B38A23EE
:1049000085BB80919906482F407F8F70282F3327D1
:104910002230310509F44CC02330310524F521152E
:10492000310509F44AC22130310509F05EC0842FF7
:10493000992780779070959587959595879595950A
:1049400087959595879502C0220F331F8A95E2F7C8
:1049500067B3622B67BB47FDDAC4722F709588B3CB
:10496000872388BB42C02630310509F497C327301E
:104970003105D9F5842F9927807790709595879583
:1049800095958795959587959595879521E030E044
:1049900002C0220F331F8A95E2F7F2B1F22BF2B96F
:1049A00047FD34C5522F509583B1852383B91DC06F
:1049B000842F992780779070959587959595879501
:1049C000959587959595879521E030E002C0220F57
:1049D000331F8A95E2F794B3922B94BB47FD66C4CC
:1049E000A22FA09585B38A2385BB80919E06482F70
:1049F000407F8F70282F33272230310509F44CC0B7
:104A00002330310524F52115310509F412C2213076
:104A1000310509F05EC0842F9927807790709595B5
:104A2000879595958795959587959595879502C0D6
:104A3000220F331F8A95E2F767B3622B67BB47FDEE
:104A400062C4722F709588B3872388BB42C026301A
:104A5000310509F4F5C327303105D9F5842F99279D
:104A6000807790709595879595958795959587957D
:104A70009595879521E030E002C0220F331F8A957B
:104A8000E2F7F2B1F22BF2B947FDB0C4522F5095C4
:104A900083B1852383B91DC0842F992780779070B7
:104AA00095958795959587959595879595958795EE
:104AB00021E030E002C0220F331F8A95E2F794B361
:104AC000922B94BB47FDDAC3A22FA09585B38A230E
:104AD00085BB80917006482F407F8F70282F332729
:104AE0002230310509F44CC02330310524F521155D
:104AF000310509F444C12130310509F05EC0842F2D
:104B00009927807790709595879595958795959538
:104B100087959595879502C0220F331F8A95E2F7F6
:104B200067B3622B67BB47FDEAC3722F709588B3EA
:104B3000872388BB42C02630310509F455C227308F
:104B40003105D9F5842F99278077907095958795B1
:104B500095958795959587959595879521E030E072
:104B600002C0220F331F8A95E2F7F2B1F22BF2B99D
:104B700047FD38C4522F509583B1852383B91DC09A
:104B8000842F99278077907095958795959587952F
:104B9000959587959595879521E030E002C0220F85
:104BA000331F8A95E2F794B3922B94BB47FD7BC3E6
:104BB000A22FA09585B38A2385BB8091EE05482F4F
:104BC000407F8F70282F33272230310509F44CC0E5
:104BD0002330310524F52115310509F4B2C0213007
:104BE000310509F05EC0842F9927807790709595E4
:104BF000879595958795959587959595879502C005
:104C0000220F331F8A95E2F767B3622B67BB47FD1C
:104C100072C3722F709588B3872388BB42C0263039
:104C2000310509F477C227303105D9F5842F99274A
:104C300080779070959587959595879595958795AB
:104C40009595879521E030E002C0220F331F8A95A9
:104C5000E2F7F2B1F22BF2B947FDE0C3522F5095C3
:104C600083B1852383B91DC0842F992780779070E5
:104C7000959587959595879595958795959587951C
:104C800021E030E002C0220F331F8A95E2F794B38F
:104C9000922B94BB47FD01C3A22FA09585B38A2315
:104CA00085BB80915C069927880F991F880F991FF3
:104CB000809366080E94A7300E9432420E9482417F
:104CC0001092F70234E13093F8021092F902109238
:104CD00007034FEF5FEF6FEF7FEF409303035093B6
:104CE0000403609305037093060310920A03109265
:104CF000090381E080931D0310921E0310920D039F
:104D00002091D00520FF13C02091FB023091FC02BE
:104D10008091580699278F709070029709F45BC1B3
:104D200083E02C3F380730F08FEF90E07BC3809119
:104D3000010378C33695279536952795822F9927B5
:104D400071C3842F99278077907095958795959555
:104D50008795959587959595879521E030E002C0D8
:104D6000220F331F8A95E2F73AB3322B3ABB47FD45
:104D7000F7C2422F40958BB384238BBB92CF842FF5
:104D800099278077907095958795959587959595B6
:104D900087959595879521E030E002C0220F331F5B
:104DA0008A95E2F73AB3322B3ABB47FDB4C2422FA1
:104DB00040958BB384238BBB00CF842F99278077BA
:104DC00090709595879595958795959587959595E7
:104DD000879521E030E002C0220F331F8A95E2F769
:104DE0003AB3322B3ABB47FD9EC2422F40958BB35C
:104DF00084238BBBFACD842F99278077907095956B
:104E0000879595958795959587959595879521E0B3
:104E100030E002C0220F331F8A95E2F73AB3322BFB
:104E20003ABB47FD88C2422F40958BB384238BBB8E
:104E300068CD842F99278077907095958795959563
:104E40008795959587959595879521E030E002C0E7
:104E5000220F331F8A95E2F73AB3322B3ABB47FD54
:104E600066C2422F40958BB384238BBB32CE842FF6
:104E700099278077907095958795959587959595C5
:104E800087959595879521E030E002C0220F331F6A
:104E90008A95E2F73AB3322B3ABB47FD5DC2422F07
:104EA00040958BB384238BBBB8CC842F9927807714
:104EB00090709595879595958795959587959595F6
:104EC000879521E030E002C0220F331F8A95E2F778
:104ED0003AB3322B3ABB47FD3BC2422F40958BB3CE
:104EE00084238BBBCACA842F9927807790709595AD
:104EF000879595958795959587959595879521E0C3
:104F000030E002C0220F331F8A95E2F73AB3322B0A
:104F10003ABB47FD14C2422F40958BB384238BBB11
:104F200035CA842F992780779070959587959595A8
:104F30008795959587959595879521E030E002C0F6
:104F4000220F331F8A95E2F73AB3322B3ABB47FD63
:104F5000FBC1422F40958BB384238BBBEACB842FBC
:104F600099278077907095958795959587959595D4
:104F700087959595879521E030E002C0220F331F79
:104F80008A95E2F73AB3322B3ABB47FDC8C1422FAC
:104F900040958BB384238BBB58CB842F9927807784
:104FA0009070959587959595879595958795959505
:104FB000879521E030E002C0220F331F8A95E2F787
:104FC0003AB3322B3ABB47FDCFC1422F40958BB34A
:104FD00084238BBBC6CA369527953695279536957B
:104FE0002795822F99271EC2842F9927807790704A
:104FF0009595879595958795959587959595879599
:1050000021E030E002C0220F331F8A95E2F7B1B3EE
:10501000B22BB1BB47FDD5C1E22FE09582B38E2301
:1050200082BBCBCD842F99278077907095958795FB
:1050300095958795959587959595879521E030E08D
:1050400002C0220F331F8A95E2F7B1B3B22BB1BB76
:1050500047FDB3C1E22FE09582B38E2382BBF5CA30
:10506000842F99278077907095958795959587954A
:10507000959587959595879521E030E002C0220FA0
:10508000331F8A95E2F7B1B3B22BB1BB47FD91C193
:10509000E22FE09582B38E2382BB4BCB842F9927DE
:1050A0008077907095958795959587959595879537
:1050B0009595879521E030E002C0220F331F8A9535
:1050C000E2F7B1B3B22BB1BB47FD6FC1E22FE09560
:1050D00082B38E2382BB89CC842F992780779070EE
:1050E00095958795959587959595879595958795A8
:1050F00021E030E002C0220F331F8A95E2F7B1B3FE
:10510000B22BB1BB47FD49C1E22FE09582B38E239C
:1051100082BBF7CB842F99278077907095958795E0
:1051200095958795959587959595879521E030E09C
:1051300002C0220F331F8A95E2F7B1B3B22BB1BB85
:1051400047FD27C1E22FE09582B38E2382BBA9CD14
:10515000842F992780779070959587959595879559
:10516000959587959595879521E030E002C0220FAF
:10517000331F8A95E2F7B1B3B22BB1BB47FD04C12F
:10518000E22FE09582B38E2382BB00C9842F99273A
:105190008077907095958795959587959595879546
:1051A0009595879521E030E002C0220F331F8A9544
:1051B000E2F7B1B3B22BB1BB47FDE2C0E22FE095FD
:1051C00082B38E2382BB59C9842F99278077907030
:1051D00095958795959587959595879595958795B7
:1051E00021E030E002C0220F331F8A95E2F7B1B30D
:1051F000B22BB1BB47FDC0C0E22FE09582B38E2336
:1052000082BBAFC9842F9927807790709595879539
:1052100095958795959587959595879521E030E0AB
:1052200002C0220F331F8A95E2F7B1B3B22BB1BB94
:1052300047FD9EC0E22FE09582B38E2382BBEDCA6C
:10524000842F992780779070959587959595879568
:10525000959587959595879521E030E002C0220FBE
:10526000331F8A95E2F7B1B3B22BB1BB47FD99C0AA
:10527000E22FE09582B38E2382BB2BCC85B3822BA9
:1052800027CC85B3822B6CC985B3822BF5C885B337
:10529000822B36CB85B3822B4BCA85B3822B00CDB4
:1052A00085B3822BB9CA85B3822B86CC85B3822B7A
:1052B0009BCB85B3822B69C885B3822BC5C988B3C4
:1052C000822B88BB1ECB88B3822B88BBA6CA88B32F
:1052D000822B88BB5BC888B3822B88BBCEC888B3BF
:1052E000822B88BB3EC988B3822B88BB22CA88B375
:1052F000822B88BBAAC988B3822B88BBD2CC88B347
:10530000822B88BB5ACC88B3822B88BBE2CB88B374
:10531000822B88BB6ACB8BB3822B8BBB4ECC8BB3DF
:10532000822B8BBB92C98BB3822B8BBB5ECB8BB397
:10533000822B8BBBCECB8BB3822B8BBBE2CA8BB3C6
:10534000822B8BBB0C94C6218BB3822B8BBBF1C9F8
:105350008BB3822B8BBB91C88BB3822B8BBB5DCA6B
:105360008BB3822B8BBB9DCC8BB3822B8BBBF9C8B1
:1053700082B3822B82BB51CA82B3822B82BBF1C81B
:1053800082B3822B82BB79C882B3822B82BB0C94FE
:10539000C62182B3822B82BB84CC82B3822B82BB98
:1053A000B0CA82B3822B82BB94CB82B3822B82BBE6
:1053B0001CCB82B3822B82BBBCC982B3822B82BB43
:1053C00044C982B3822B82BBF8CB83B1822B83B9D1
:1053D00024CA83B1822B83B938C983B1822B83B9A4
:1053E0000C94C62183B1822B83B9E7CB83B1822B86
:1053F00083B96FCB83B1822B83B93FC883B1822B32
:1054000083B97FCA83B1822B83B993C983B1822BBD
:1054100083B9EBCA83B1822B83B9A3C883B1822B32
:1054200083B93FCC80930203A0916B06A0930E0337
:105430009BE0909384010E94333A0E9434BA0E9408
:10544000BF6D0E94D8470E9478A463E087E998E086
:105450000E9416A90E94BEA47AE07093140261E033
:10546000609313020E9443BF0895CFEFD0E1DEBFE7
:10547000CDBF0E945A8E0E9400210E9443460E9486
:105480004ABF0E94188D78940E9482410E94605207
:105490000E94A0540E94E05680915C0890915D08A3
:1054A000892B39F490910A02987F2BB32770922BA5
:1054B0009BBB3091F80230FDABC20E948E3A0E9435
:1054C0009F5D50910703552321F16091F80264FF1D
:1054D00007C0A09107037091A9057A1708F0CBC205
:1054E000B091F702B1FDABC2E0918401E13009F463
:1054F000ADC20E94CC5A8091A1062091A0068830AE
:1055000018F4223008F045C2809120038B778093F5
:1055100020030E94AE3A0E94F3420E94E05D0E9486
:105520005B3F0E94DB40B0911802BB2309F06DC2C3
:105530008091170281FF23C08D7F80931702F09125
:10554000E505F1FF6FC20E940F909091F70290FF66
:1055500007C080918401823018F0815080938401CB
:10556000F8943091F80235FF09C020910D032F3FC8
:1055700029F060910D036F5F60930D037894F894A8
:10558000E091D307F091D4074091880050918900B1
:105590005093D4074093D3074E175F0748F4809188
:1055A000D5079091D60701969093D6078093D5079B
:1055B000CA0178942091850130918601821B930B5A
:1055C00061E6883A960708F491C08155934C08F437
:1055D000D9C150938601409385010E94C73BA09199
:1055E0000103409126064A1780F05091CD0552954F
:1055F0005F70583008F4F7C180B399279C0122707E
:10560000307081FFFDC1C1E0D0E0F89410920D032D
:1056100078946091D5077091D6079B014427552750
:105620008091D9079091DA07A091DB07B091DC0750
:10563000CD01AA27BB27281B390B4A0B5B0B809196
:105640006E069927AA27BB2782179307A407B507D9
:1056500038F480916F0699278617970708F403C2DC
:1056600080911402815009F08AC1BAE0B09314020B
:10567000E0911502F09116023196F0931602E09334
:10568000150270911702726070931702F091F00585
:10569000F3FF07C080915708882309F493C10E9443
:1056A000E86A9091F70290FF04C03091540630FDF3
:1056B000DFC180913A018F5F843009F4B6C18093D5
:1056C0003A01F89440910A02486040930A027894A3
:1056D00080911F098F3F31F0882309F4C1C18150A7
:1056E00080931F094091D3075091D40780918D0674
:1056F0008823F1F0992796958795782F7877E52F6D
:10570000FF272E2F60910D02261B271788F03327C5
:10571000A72FBB27AA0FBB1FA217B3070CF055C1B9
:10572000E0930D020E9476BD4091D3075091D407BB
:10573000452F5527842F20913D02821B8F30A8F0E2
:1057400099274F970CF4CBC040933D0250915A08D3
:1057500050FD07C020916C07222309F43AC10E9432
:1057600053830E9410580E946E590E94265260ED89
:1057700078E082EA98E00E94E3B862EA78E08DEA95
:1057800098E00E9416B90E942FA780916C07882389
:1057900009F438C17091F00572FD62C08091FB057B
:1057A00099278F7390700097B1F1FC013496F695AC
:1057B000FE2FEE27F795E795F8946091D307709147
:1057C000D40740918800509189005093D4074093AA
:1057D000D3074617570748F4A091D507B091D607CD
:1057E0001196B093D607A093D5079A01789460914B
:1057F000370270913802261B370B2E173F0788F0AF
:10580000CF01880F991F8217930708F0F0C05093BB
:105810003802409337020E94AC6E4091D3075091FA
:10582000D407452F5527842F20911202821B8730E1
:1058300068F099270F970CF456C0409312020E940B
:10584000AFBAE0910F03E43009F457C080911E080D
:1058500090911F08019690931F0880931E0814CE04
:105860008091FB0599278F7390700196F82FEE2792
:10587000F8942091D3073091D4074091880050913B
:1058800089005093D4074093D3074217530748F435
:10589000A091D507B091D6071196B093D607A093E3
:1058A000D5079A0178946091370270913802261BCF
:1058B000370B2E173F0708F4B4CFCF01880F991F7D
:1058C0008217930708F088C050933802409337023C
:1058D0000E94386E4091D3075091D407A2CF215F28
:1058E00020933D0233CF295F209312020E94AFBA6A
:1058F000E0910F03E43009F0A9CF409103035091E8
:1059000004036091050370910603BB27A72F962F10
:10591000852F8F3F41F1803408F098CF6091D307F5
:105920007091D407A0911B03B0911C036A1B7B0BE1
:105930009B01442755278091030390910403A09174
:105940000503B0910603880F991FAA1FBB1F82177A
:105950009307A407B50708F079CF472F552740389C
:10596000510508F073CFF8947894E0914608F091CF
:1059700047083196F0934708E093460867CF809335
:10598000140284CE28553E49309386012093850128
:1059900024CE80912003992783709070039709F497
:1059A0006DC080912003992783709070029709F44D
:1059B00090C061E00038160708F4ABCD8091200359
:1059C0008360A5CD0E940C6B6CCE670F60930D02B7
:1059D000A9CE0E940F97C5CE6E0F7F1F709338021D
:1059E0006093370275CFCC2309F413CE0ECE6E0F21
:1059F0007F1F70933802609337020E94AC6E0DCF08
:105A0000E90107CE0E94B47BC5CE0E94334E90CDF3
:105A1000F8944091F8024E7F4093F80278940E94E7
:105A200088454BCD0E944DBA8ECD10923A01F89424
:105A300060910A02677F60930A02789449CE0E94BF
:105A4000983AE0918401E13009F053CD109284013D
:105A5000F894F091F802FF7EF093F802789449CD23
:105A60000E9452BF3FCEF8940E94F6497894F8CD38
:105A70000E9471681ECE0E943A463BCD0F3F110531
:105A800008F047CD90912003915090932003332745
:105A900021FF05C03091200334603093200324FFA0
:105AA00005C0209120032068209320038091D50712
:105AB0009091D607782F6627E091D307F091D4070D
:105AC000AF2FBB276A2B7B2B7093110260931002C0
:105AD00020CD5091A206652F7727FB01EE0FFF1F07
:105AE000EE0FFF1FA091D507B091D6073A2F2227BE
:105AF0008091D3079091D407492F5527242B352B1C
:105B00008091100290911102A901481B590B4E1768
:105B10005F0708F4FECC660F771F660F771F660FCE
:105B2000771F6417750750F4309311022093100209
:105B3000709120037877709320033BCF8E0F9F1FC7
:105B40009093110280931002F3CF0F93CF93DF93C2
:105B5000801730F5061718F0822F99272CC0681B84
:105B6000081BE62FFF27EE0FFF1FE652F84F659147
:105B70007491FF27EE27609FE001709FD00DE11D1B
:105B800011248D2F9E2FAF2FBB27082F421758F0BF
:105B9000842F821B809FD00111248B2F9927481BB3
:105BA000842F992708C0241B289FE00111248D2FE2
:105BB0009927840F9927DF91CF910F9108950F9323
:105BC000CF93DF93742F522F302F681728F0801750
:105BD00040F0272F332768C0601760F1252F332747
:105BE00063C00617D8F7681B381BE62FFF27EE0F98
:105BF000FF1FE652F84FA591B491FF27EE27A39F10
:105C0000E001B39FD00DE11D1124CE01DF01892FEA
:105C10009A2FAB2FBB27082F421708F43CC0842FC4
:105C2000821B809F90011124832F9927781B272F97
:105C300033273AC0081708F0CCCF861B361BE82F55
:105C4000FF27EE0FFF1FE652F84FA591B491FF27F3
:105C5000EE27A39FE001B39FD00DE11D1124CE01DB
:105C6000DF01892F9A2FAB2FBB27082F241748F06D
:105C7000822F841B809F90011124832F9927581B0A
:105C8000ADCF721B789FE00111248D2F9927820FD1
:105C9000282F332709C0541B589FE00111248D2F52
:105CA0009927840F282F3327822F9927DF91CF91AF
:105CB0000F910895CF92DF92EF92FF920F931F936F
:105CC000CF93DF93EA01A901801710F09E014BC02A
:105CD000061708F048C0681B081BE62FFF27EE0FC9
:105CE000FF1FE652F84F85919491FF24EE24809F88
:105CF0006001909FD00CE11C1124D701C6019601D0
:105D0000C417D507D0F06E01C41AD50A44279D9D4B
:105D100080018C9D70019C9DF00C011D141F8D9DB8
:105D2000F00C011D141F1124A8019701CA01AA2714
:105D3000BB279E01281B390B16C04C1B5D0B882707
:105D4000359F7001249F6001349FD00CE11CF81E28
:105D5000259FD00CE11CF81E1124C701AA27BB27E0
:105D60009C012C0F3D1FC901DF91CF911F910F9115
:105D7000FF90EF90DF90CF900895CF93DF9384173B
:105D800018F080E090E01CC04617C0F4681BE62FB6
:105D9000FF27EE0FFF1FE652F84F65917491481BE5
:105DA000FF27EE27649FE001749FD00DE11D1124B1
:105DB0008D2F9E2FAF2FBB27992702C08FEF90E02A
:105DC000DF91CF910895CF93DF93DC01E90191E05A
:105DD00020E0822F261780F4282FFD01E80FF11D07
:105DE0008081481708F490E0822F8F5F861710F4A7
:105DF000992391F7222319F42983288304C0215081
:105E000028832F5F2983DF91CF9108959B0199E229
:105E1000899FD0011124EE27B39FB001A29FA0015A
:105E2000B29F500D611D7E1FA39F500D611D7E1FEF
:105E3000112452956295729540EF76277423762748
:105E40006527642365279B01C90108959B019DEC8B
:105E5000899FC0011124EE27939FB001829FA0016A
:105E6000929F500D611D7E1F839F500D611D7E1FEF
:105E70001124DB01CA013BE0B695A795979587955C
:105E80003A95D1F70895CF93DF93FB0169E2552747
:105E90004427869F9001969F300D411D1124232F8A
:105EA000342F452F5527BB27AA27E69FC001F69F11
:105EB000900DA11D1124892F9A2FAB2FBB27662788
:105EC000399FF001289FE001389FD00DE11DF61F9A
:105ED000299FD00DE11DF61F11248D2F9E2FAF2F6E
:105EE000BB27DF91CF910895CF93DF9320E8FF2761
:105EF000EE27829FE001929FD00DE11D1124CE017B
:105F0000DF01292F3A2F4B2F55275CEDFF27EE2776
:105F1000659FE001759FD00DE11D1124AE01BF0109
:105F2000BB27A72F962F852F6627399FF001289F23
:105F3000E001389FD00DE11DF61F299FD00DE11D16
:105F4000F61F1124CE01DF01892F9A2FAB2FBB271B
:105F5000DF91CF910895CF93DF9320E1FF27EE27C4
:105F6000829FE001929FD00DE11D11242D2F3E2F25
:105F70004F2F552749E2FF27EE27649FE001749FCA
:105F8000D00DE11D11248D2F9E2FAF2FBB2766272B
:105F9000399FF001289FE001389FD00DE11DF61FC9
:105FA000299FD00DE11DF61F11248D2F9E2FAF2F9D
:105FB000BB27DF91CF910895FC013181328320818D
:105FC00021836083261740F4862F321740F4622F16
:105FD000861740F499270895822F3217C0F3632F54
:105FE0008617C0F3862F992708956817790714F448
:105FF000AB0104C0841795070CF0AC01CA010895E9
:1060000068172CF4862F992787FD9095089584179B
:106010002CF4842F992787FD90950895992787FD63
:1060200090950895681718F4862F99270895841776
:1060300018F4842F9927089599270895861710F446
:1060400099270895862F99270895681710F499279E
:106050000895862F99270895CF93DF93EC01942F0D
:106060004F7092959F70E92FFF279F012F5F3F4F41
:10607000A62FBB272A173B072CF0AC0FBD1F11978B
:106080008C911DC0EC0FFD1F5081252F3327C0E1DF
:10609000D0E0C41BD1092C9FD0012D9FB00D3C9F97
:1060A000B00D1124CD012181249FB0011124860F50
:1060B000971F929582958F7089279F7089279927BE
:1060C000DF91CF910895CF93DF93EC01942F4F711F
:1060D000929596959770E92FFF279F012F5F3F4F6D
:1060E000A62FBB272A173B072CF0AC0FBD1F11971B
:1060F0008C911FC0EC0FFD1F5081252F3327C0E26C
:10610000D0E0C41BD1092C9FD0012D9FB00D3C9F26
:10611000B00D1124CD012181249FB0011124860FDF
:10612000971F96958795929582958F7089279F7076
:1061300089279927DF91CF9108958770806487B967
:10614000369A349BFECF349A84B195B1089587E88E
:1061500086B920E0322F3770306437B9369A349BD5
:10616000FECF349A44B155B1E22FFF27EE0FFF1F47
:10617000E15CFD4F440F551F518340832F5F263054
:1061800048F3089510923E0220E427B98FEC86B9B7
:1061900008951F920F920FB60F9211242F933F93E1
:1061A0004F938F939F93EF93FF9340913E02E42F81
:1061B000FF27EE0FFF1FE15CFD4F808191819695D7
:1061C000879524B135B1820F931F918380834F5FF0
:1061D000463020F010923E02339806C040933E02B3
:1061E0004770406447B9369AFF91EF919F918F9124
:1061F0004F913F912F910F900FBE0F901F901895C8
:10620000883008F080E0809352080895DC012091E6
:10621000E002422F55274F5F5F4F9A014150504097
:10622000F901E07FF1702E1B3F0B80914D02281782
:10623000B1F0FA01EE0FFF1FEE0FFF1FEE0FFF1F71
:10624000E40FF51FE25BFD4FB183A08362831382ED
:10625000158214822093E00280E090E008958FEF91
:1062600090E00895823138F4E82FFF27EE50F64F82
:106270008491992708958251863038F4E82FFF27BA
:10628000E050FF4F80819927089580E090E00895C5
:106290009927AA27BB278731910590F4FC01E0508C
:1062A000FE4FEE0FFF1F0590F491E02D099481E35E
:1062B00090E0089580E290E0089582E390E00895F0
:1062C00086E590E008958DE390E0089581E690E002
:1062D000089580E790E008958DE490E0089585E4C6
:1062E00090E0089586E590E0089520915806422FA9
:1062F00055274F7050704F305105C9F2822F0E94C0
:106300008172992708958CE290E0089586E790E0E5
:10631000089583E590E008958BE690E0089588E77E
:1063200090E0089580E390E008958EE290E0089573
:1063300020915806822F9927929582958F708927F0
:106340009F7089270F9709F4B8CF822F0E94787227
:1063500099270895809115029927089580E090E08B
:10636000089580E090E008959927AA27BB278133FC
:10637000910548F4FC01E95EFD4FEE0FFF1F05900B
:10638000F491E02D099480E090E0089530915B084D
:1063900037FF28C02091E002422F55274F5F5F4F03
:1063A0009A0141505040C901807F9170281B390BE0
:1063B000A0914D022A17B1F0FA01EE0FFF1FEE0F68
:1063C000FF1FEE0FFF1FE40FF51FE25BFD4F44EBD5
:1063D00051E35183408351E3528313821582148227
:1063E0002093E00280E090E0089580915207992781
:1063F000089580910E03869599270895809117033B
:1064000090911803929582958F7089279F708927A4
:10641000992708958091EA0299270895A091E702AB
:10642000B091E80291E177276627A99FA001B99F63
:10643000500D611D1124BB27A72F962F852F9C017E
:10644000E32FFF27EF2B09F0F9C0822F992708953A
:106450008091E602992708958091EC02992708958A
:10646000A0912703B091280339E277276627A39FDD
:10647000A001B39F500D611D1124DB01CA013AE058
:10648000B695A795979587953A95D1F79927089549
:106490008091090390910A03992708958091090337
:1064A00090910A03892F9927992708958091E502F1
:1064B0008B3908F0C3C08C59992708958091E40264
:1064C000992708959091E30284E6989FB0011124E2
:1064D000872F992787FD9A958E5C9927089580913B
:1064E000410290914202969587959695879596954B
:1064F0008795992708958091FA02992708958091A8
:106500000103992708958091FD02992708958091AC
:10651000FE029927089520919706222309F491C03D
:1065200080910803880F880F992708958091970616
:10653000882309F491C08091080399270024880FCB
:10654000991F001C880F991F001C892F902D9927D7
:106550000895809115029927089580914B0290919A
:106560004C02C1CF8091F7029927089520E0309125
:10657000A1064091A0069091CD05592F52955F70CC
:10658000583008F464C0819B65C07091F80275FDB5
:1065900021609F70983008F466C0809B67C03830D7
:1065A00018F4423008F020624091F202411120615B
:1065B000B091F702B7FD5CC0F091F802F3FD2460E2
:1065C00060913E0870913F086B30710508F02260C1
:1065D000822F992708958091EB02992788539F4F26
:1065E00028E477276627829FA001929F500D611DA6
:1065F0001124DB01CA01E7E0B695A7959795879529
:10660000EA95D1F7E82FFF27EE0FFF1FE652F84F6C
:106610008591949177276627829FA001929F500DC4
:10662000611D1124DB01CA0177E0B695A795979506
:1066300087957A95D1F78954992708958FEF90E03F
:1066400008958091FB029091FC0299270895189477
:1066500009F09BCF20E899CF8091FB029091FC023A
:10666000892F992721CF189409F099CF206497CFCB
:106670002860A2CFCF93482F50914D02252F33276A
:10668000F901EE0FFF1FEE0FFF1FEE0FFF1FE20FCE
:10669000F31FE25BFD4F25818481C82FCF70782FD7
:1066A00072957F704530B0F4842F99278230910520
:1066B00009F486C08330910534F4009709F07AC05C
:1066C000822F9927E4C08330910509F4CEC0049746
:1066D00009F49AC0403F08F052C063E0E1E033277C
:1066E00027FD30952B36310509F46FC02C36310566
:1066F0000CF454C02E36310509F48CC02F36310508
:106700000CF071C02C36310509F47BC0A9E7B5E067
:10671000FCE0F69F802D11248B5F481709F47DC0A3
:10672000242F3327992701972817390709F49AC08E
:10673000242F2450F79FC00111244E2F5527849FEA
:10674000F001859FF00D949FF00D1124EA0FFB1FBF
:1067500003C0261BE40FF51F2617D8F73327223076
:106760003105E9F1233031059CF52115310521F082
:106770002130310509F440C080E290E088C0652FE7
:106780007727FB01EE0FFF1FEE0FFF1FEE0FFF1F1E
:10679000E60FF71FE25BFD4F138292CF22363105E1
:1067A000B1F12A36310509F0B1CF65E0E2E0AAE3A4
:1067B000B3E0AECF019709F08DCF8BE590E067C0D5
:1067C000872F0E948172992762C0A5E8B5E0A0CF0B
:1067D0002330310581F02430310571F63197808105
:1067E0000E948172F0CF2437310509F08FCFADE9D7
:1067F000B5E0F8E08ECF319780810E9478729927BA
:1068000046C0A9EEB4E084CF8DE390E040C0A1E99A
:10681000B5E07ECFA4EAB6E07BCF7C1749F17F5F7D
:10682000A52FBB27FD01EE0FFF1FEE0FFF1FEE0F81
:10683000FF1FEA0FFB1FE25BFD4F522F4427872FFC
:10684000992782959295907F9827807F9827480F67
:10685000591F4C0F511D558344838FEE83838AE06B
:1068600090E015C08DE090E012C08DE590E00FC083
:10687000252F3327F901EE0FFF1FEE0FFF1FEE0F3D
:10688000FF1FE20FF31FE25BFD4F8EEFE7CFCF91CB
:106890000895CF93782FC0914D028C2F9927FC013A
:1068A000EE0FFF1FEE0FFF1FEE0FFF1FE80FF91F88
:1068B000E25BFD4FA481B5819D012A0F3B1F2B5F39
:1068C000354F60E003C0225030406F5FF9014591C1
:1068D000549141155105B9F3783F38F5470F511DD3
:1068E000FA018491882309F03CC0662361F42E5F8D
:1068F0003F4FF90185919491892B09F058C0AE3F23
:10690000B10508F054C04C2F5527FA01EE0FFF1FB8
:10691000EE0FFF1FEE0FFF1FE40FF51FE25BFD4FB1
:1069200027EF23838BE590E063C0872F99278B3F68
:10693000910591F08C3F9105B4F4893F910509F4DC
:1069400052C08A3F91050CF041C0883F910509F47F
:1069500046C08AE790E04CC0AB55BA4F8C910E947C
:106960007872992745C08D3F910509F43FC08D3F4E
:1069700091057CF18E3F910561F78C2F9927FC01E1
:10698000EE0FFF1FEE0FFF1FEE0FFF1FE80FF91FA7
:10699000E25BFD4FA481B5811196B583A483AF3F1F
:1069A000B10510F45FEF53838AE090E021C06C2FB3
:1069B0007727FB01EE0FFF1FEE0FFF1FEE0FFF1FEC
:1069C000E60FF71FE25BFD4F3AEF33838DE390E074
:1069D0000FC0AB55BA4F8C910E948172C2CF862FE7
:1069E0000E948172BECF8DE590E002C08DE090E004
:1069F000CF9108958F3F39F0E82FFF27EB55FA4FDD
:106A000080819927089580E090E008959091E002B8
:106A1000292F3327F901EE0FFF1FEE0FFF1FEE0F97
:106A2000FF1FE20FF31FE25BFD4F44815581282FCA
:106A300033272115310531F02130310539F4842F08
:106A400099270895852F9927992708958AE790E037
:106A5000089590914D02292F3327F901EE0FFF1F62
:106A6000EE0FFF1FEE0FFF1FE20FF31FE25BFD4F64
:106A70000480F581E02DE80FF11D808199270895AC
:106A800090914D02292F3327F901EE0FFF1FEE0FD2
:106A9000FF1FEE0FFF1FE20FF31FE25BFD4F0480AD
:106AA000F581E02DE80FF11D8491992708959091CB
:106AB0004D02492F5527FA01EE0FFF1FEE0FFF1F62
:106AC000EE0FFF1FE40FF51FE25BFD4F24813581C0
:106AD000280F311DC901AA27BB27A160ABBFFC014C
:106AE000879199270895CF93382FC0914D028C2F0D
:106AF0009927DC01AA0FBB1FAA0FBB1FAA0FBB1F40
:106B0000A80FB91FA25BBD4FFD012481822F9927D9
:106B1000FC01E652F64F4491341770F5243009F425
:106B20003EC0880F991F8E51964FFC01A591B491DC
:106B3000632F7727A60FB71F5C91273009F444C055
:106B40002230D9F124502430A0F0842F99270197C6
:106B50006817790774F06C2F7727FB01EE0FFF1F82
:106B6000EE0FFF1FEE0FFF1FE60FF71FE25BFD4F5B
:106B70001282852F992759C0832F841B8C3038F4BB
:106B8000E82FFF27E758FA4F808199274EC08C5095
:106B90008C3068F08B3068F3FD011282EACFE32F6E
:106BA000FF27EE0FFF1FE75CFC4F8181EECFE82F40
:106BB000FF27EB57FA4F5081EDCF383018F2FB0129
:106BC000E757FA4F5081BECFA52FBB27A853BF4F21
:106BD00028E477276627A29FA001B29F500D611D70
:106BE0001124DB01CA0137E0B695A79597958795E3
:106BF0003A95D1F7E82FFF27EE0FFF1FE652F84F27
:106C00008591949177276627829FA001929F500DCE
:106C1000611D1124DB01CA01C7E0B695A7959795C0
:106C20008795CA95D1F78954B0CFCF910895E82FB1
:106C3000FF27EB57FA4F60830895E82FFF27E758A7
:106C4000FA4F60830895CF93DF93382F90915208C5
:106C5000492F5527FA01E652F64F84913817A0F4D0
:106C6000943021F1923009F468C09730A1F1232FBC
:106C70003327440F551F4E51564FFA01C591D491F9
:106C8000C20FD31F688361C09450943008F05DC078
:106C9000381B832F3C30C8F08C508C3008F055C026
:106CA000E82FFF27EB57FA4F60834FC0A62FBB2773
:106CB0009A2F88278068232F3327E901C20FD31F1B
:106CC000C75CDC4F99838883D4CFE32FFF27E75835
:106CD000FA4F60833AC0862F9927875B9F4F28E43D
:106CE000FF27EE27829FE001929FD00DE11D112426
:106CF000CE01DF0177E0B695A795979587957A95B0
:106D0000D1F7E82FFF27EE0FFF1FE652F84F6591EE
:106D10007491FF27EE27629FE001729FD00DE11D65
:106D20001124CE01DF0167E0B695A7959795879569
:106D30006A95D1F7682F685C9ACF383008F497CFFE
:106D4000E32FFF27E757FA4F6083DF91CF91089534
:106D5000CF93DF93EC01722F2091E002A22FBB278B
:106D600011969D011197F901E07FF1702E1B3F0BE9
:106D700080914D022817B9F0FD01EE0FFF1FEE0FB5
:106D8000FF1FEE0FFF1FEA0FFB1FE25BFD4FD183DA
:106D9000C083628313825583448376832093E00209
:106DA00080E090E002C08FEF90E0DF91CF910895F6
:106DB000CF93DF93EC012091E002A22FBB27119625
:106DC0009D011197F901E07FF1702E1B3F0B80911F
:106DD0004D022817B9F0FD01EE0FFF1FEE0FFF1F48
:106DE000EE0FFF1FEA0FFB1FE25BFD4FD183C08355
:106DF000628313825583448316822093E00280E0ED
:106E000090E002C08FEF90E09927DF91CF91089535
:106E1000682F8091DF02282F332721303105E9F0D8
:106E20002230310501F1862F9927AA27BB27BC0103
:106E3000615470406733710578F4FB01E85BFD4FE6
:106E4000EE0FFF1F0590F491E02D099471E070930F
:106E5000DF022CE420933C01089560933B0122E083
:106E60002093DF02089540913C01242F33272E34D4
:106E7000310599F12F34310574F42A34310509F4C0
:106E80002AC22B34310514F528343105E1F481E0B0
:106E9000809352080CC02435310509F420C22535F1
:106EA000310554F42F34310571F410925208809159
:106EB0003B010E94233607C02037310509F413C275
:106EC00027373105A1F31092DF0208952C343105E4
:106ED000D1F787E080935208EACF86E0809352088A
:106EE000E6CF7091E002472F55274F5F5F4F9A0121
:106EF00041505040B901607F7170261B370B922FB3
:106F000030914D02931709F4A7CFFA01EE0FFF1F3E
:106F1000EE0FFF1FEE0FFF1FE40FF51FE25BFD4FAB
:106F2000A4EBB1E3B183A08381E382831382158252
:106F300014822093E002089580E00E94544F089547
:106F40002091E002422F55274F5F5F4F9A01415039
:106F50005040C901807F9170281B390BB0914D02C0
:106F60002B1709F479CFFA01EE0FFF1FEE0FFF1F69
:106F7000EE0FFF1FE40FF51FE25BFD4F4AEA51E3FE
:106F80005183408381E0D1CFB1E0B093DF0288E448
:106F900080933C01089531E03093DF028AE4F8CF1A
:106FA000E1E0E093DF028EE4F3CF31E03093DF02E3
:106FB0008FE4EECF9091E002492F55274F5F5F4F4E
:106FC0009A0141505040B901607F7170261B370B08
:106FD000E0914D022E1709F43FCFFA01EE0FFF1F8B
:106FE000EE0FFF1FEE0FFF1FE40FF51FE25BFD4FDB
:106FF000A8E4B1E3B183A08387E197CFF091E002E9
:107000004F2F55274F5F5F4F9A0141505040C901A4
:10701000807F9170281B390B70914D02271709F45E
:107020001BCFFA01EE0FFF1FEE0FFF1FEE0FFF1F2A
:10703000E40FF51FE25BFD4F42E351E351834083D0
:1070400088E173CF21E02093DF0284E5A1CF51E0F6
:10705000509352082091E002422F55274F5F5F4F17
:107060009A0141505040B901607F7170261B370B67
:1070700080914D02281709F4EFCEFA01EE0FFF1FA1
:10708000EE0FFF1FEE0FFF1FE40FF51FE25BFD4F3A
:1070900043E755E3518340837FEF7283138281E09E
:1070A00090E095838483168244CF52E05093DF02B0
:1070B00080E76ECF54E050935208F091E0024F2FDA
:1070C00055274F5F5F4F9A0141505040F901E07FD3
:1070D000F1702E1B3F0B70914D02271709F4BCCEA7
:1070E000FA01EE0FFF1FEE0FFF1FEE0FFF1FE40F61
:1070F000F51FE25BFD4FA3E7B5E3B183A0834FEF3C
:107100004283138284E090E095838483CCCF57E060
:10711000509352083091E002432F55274F5F5F4F45
:107120009A0141505040C901807F9170281B390B52
:10713000F0914D022F1709F48FCEFA01EE0FFF1FC9
:10714000EE0FFF1FEE0FFF1FE40FF51FE25BFD4F79
:1071500063E775E3718360839FEF9283138287E017
:1071600090E0958384839FCF76E0709352082091BE
:10717000E002422F55274F5F5F4F9A014150504028
:10718000B901607F7170261B370B80914D02281763
:1071900009F462CEFA01EE0FFF1FEE0FFF1FEE0F94
:1071A000FF1FE40FF51FE25BFD4F43E755E35183FB
:1071B0004083BFEFB283138286E090E0958384839F
:1071C00072CF10925208F091E0024F2F55274F5F77
:1071D0005F4F9A0141505040F901E07FF1702E1B42
:1071E0003F0B70914D02271709F436CEFA01EE0FCE
:1071F000FF1FEE0FFF1FEE0FFF1FE40FF51FE25BF7
:10720000FD4FA3E7B5E3B183A0834FEF4283138221
:107210001582148216828DCE50915208652F7727E1
:107220002091E002422F55274F5F5F4F9A01415056
:107230005040D901A07FB1702A1B3B0BE0914D0259
:107240002E1709F409CEFA01EE0FFF1FEE0FFF1FF4
:10725000EE0FFF1FE40FF51FE25BFD4F83E795E3A1
:10726000918380839FEF9283138275836483168258
:1072700060CE82E0809352083091E002432F552780
:107280004F5F5F4F9A0141505040D901A07FB170CC
:107290002A1B3B0BE0914D022E1709F4DDCDFA01BC
:1072A000EE0FFF1FEE0FFF1FEE0FFF1FE40FF51F86
:1072B000E25BFD4F63E775E3718360839FEF928329
:1072C000138282E090E095838483EDCE61E0609349
:1072D000DF0287E75DCE84E080935208E8CD82E04C
:1072E00080935208E4CD683008F060E06093520863
:1072F000EACD1092DE021092DF0238E93AB926E0B8
:10730000209395001092900087E689B910924D0263
:107310001092E00208951F920F920FB60F9211245F
:107320002F933F934F935F936F937F938F939F938D
:10733000AF93BF93EF93FF938BB1992788719070B0
:10734000892B11F08CB105C06CB180ED98E00E94E2
:1073500050B8FF91EF91BF91AF919F918F917F9125
:107360006F915F914F913F912F910F900FBE0F90B2
:107370001F9018951F920F920FB60F9211242F9302
:107380003F934F935F936F937F938F939F93AF93AD
:10739000BF93EF93FF938DEA98E00E94FFB89C01A2
:1073A000892F9927892B39F055982091DE022223C5
:1073B00019F0569A01C02CB9FF91EF91BF91AF918E
:1073C0009F918F917F916F915F914F913F912F91FD
:1073D0000F900FBE0F901F9018951F920F920FB62F
:1073E0000F9211242F938F939F9355990FC0209143
:1073F000DE02222361F09091E00280914D02981705
:1074000031F41092900029B91092DE0256989F91A3
:107410008F912F910F900FBE0F901F9018955D9B2D
:10742000FECF8CB90895AC01E7E2F3E02091CC05E2
:10743000293C30F489E1289F9001112482E008C0A2
:10744000285C6DE7269F9001112428573C4EF6CF0B
:107450008150F89434832383518340837894379602
:107460008823B1F7089530E83093E30224E62093AF
:10747000E4021092E5022093E60266EF75E0709355
:10748000E8026093E70240E054E65093EA0240933A
:10749000E90288E38093EB021092EC022093ED0264
:1074A0001092EE021092EF021092F0021092F1028E
:1074B0001092F2021092F3021092F402E7E2F3E06B
:1074C0009091CC05993C80F489E1989FC0011124EA
:1074D00022E02150F894948383831182108278945F
:1074E00037962223B1F708C0985C8DE7989FC001BA
:1074F000112488579C4EECCF2091D9073091DA07A0
:107500004091DB075091DC075F6F2093D9073093E0
:10751000DA074093DB075093DC07089525EF32E04C
:107520004091FD026AE08DEA95E00E94E32E089505
:10753000F8948091F70281FF08C08D7F8C60809362
:10754000F7028091AC058093E4077894209155066A
:1075500023FF089581E00E94688208950F93CF93DE
:10756000C0E08091F70282FF0CC00091E407002385
:1075700009F04EC0F8940091F7020B7F0093F702D8
:1075800078949091FD022091B605921778F0F894C6
:107590005091F702577F5093F70240910A024F7BB8
:1075A00040930A027894C093E50267C0F894F09182
:1075B0000A02F064F0930A02B091F702B860B09347
:1075C000F70278947091F602A72FBB27AB55BA4FFC
:1075D0008091F50299278B559A4F0091FD02FD018C
:1075E0002289FC014289FD016085FC0180850E94A1
:1075F000A52D853668F580E0282F2C0F312D311D03
:10760000A901832F9927892BF9F44093E50235C00E
:107610002091AA054C2F6091AC058C2F0E94A52DBE
:10762000382F8091AB05389FB0011124872F9927FF
:1076300087FD9A950091FD02282F432F6DEC8C2F2A
:107640000E94A52DC82F9DCF4FEF4093E50215C096
:10765000382F34568091C105389FC0011124892FDD
:10766000990F990B00910703282F432F60918405F0
:10767000809179050E94A52DBFCFCF910F910895DC
:107680002091FB023091FC028091580699278F705F
:107690009070029709F44AC083E02C3F3807A8F1A4
:1076A0002FEF30E080919C062817C0F133279927EF
:1076B0000296821793070CF040C04091EE024B7F78
:1076C0004093EE02909107033091E005391708F0DE
:1076D00040C0609107035091DF05651718F04160C5
:1076E0004093EE02A09101037091F2057A1798F58C
:1076F00080915A0899279C012270307081FD13C037
:107700004D7F4093EE02C901089536952795369531
:107710002795332780919C06281740F62091EE028A
:1077200024602093EE0281E090E00895369527953D
:107730003695279536952795ECCF4091EE02842F0C
:10774000992784709070882309F4BCCF81E090E081
:1077500008954E7FC5CFB091E407BB2331F04D7F34
:107760004093EE0280E090E00895242F3327C90172
:107770008170907020FD07C02D7F232B19F04D7F65
:107780004093EE02089542604093EE02CCCFEF9218
:10779000FF920F931F93CF93DF93CDB7DEB722975E
:1077A0000FB6F894DEBF0FBECDBF5091E1025F5F10
:1077B000F8946091D00560FF31C02091FB023091B8
:1077C000FC028091580699278F709070029709F4F7
:1077D00082C083E02C3F380708F46EC08FEF90E042
:1077E000082F4091020378940417F8F45093E102B3
:1077F00060FF42C02091FB023091FC02809158064C
:1078000099278F709070029709F46EC0F3E02C3FB7
:107810003F0708F459C08FEF90E0DEC000910103EC
:10782000409102037894041708F3F02EF41A809123
:10783000D105F81620F1E090F702E4FC5EC010914B
:10784000D5051093EC021092E102E090DA05E09287
:10785000E202F894F091F702F061F093F702B09130
:10786000F702BF7DB093F70270910A0270627093C5
:107870000A02789460FDBECF80910103ADC05093A1
:10788000E102A091F702A5FD05C0E091E2025E17BA
:1078900008F4AECFF8942091F7022F7C2093F702E2
:1078A00080910A028F7D80930A02789404E6009307
:1078B000ED021092EC029CCF3695279536952795D0
:1078C000822F9927082F8DCF3695279536952795A6
:1078D000822F992781C0369527953695279536951D
:1078E0002795822F9927EECF3695279536952795A0
:1078F00036952795822F99276FC05093E10200910A
:10790000FD0224E64091DB056DEC80E00E94A52D90
:10791000182F9E012F5F3F4F4F2D64E081ED95E0C2
:107920000E94E32E0A81A02FBB27AB55BA4F898155
:1079300099278B559A4F0F2DFD0120A9FC0140A9D5
:10794000FD0164A5FC0184A50E94A52D9927BC0119
:10795000812F0E94062F7C01E92FFF27EF2BC1F515
:107960000091FD0220E04091DC056DEC822F0E9429
:10797000A52D9701280F311D832F9927892B11F0F1
:107980002EEF30E08091EC0299278217930710F4D4
:107990002093EC02F090F702F5FC06C09091E10212
:1079A0002091E202921788F0F8945091F7025F7CE0
:1079B0005093F70240910A024F7D40930A02789457
:1079C00034E63093ED021092EC026091D00510CFB6
:1079D000A8ECEA2EF12CC4CF8093020322960FB6B6
:1079E000F894DEBF0FBECDBFDF91CF911F910F91F5
:1079F000FF90EF9008950F938091C5052091C605E3
:107A0000682F620F712D711DAB016F3F710511F071
:107A100008F04FEF281710F020E002C0821B282F3B
:107A20000091FA0264EA8DE30E94A52D99270F9137
:107A30000895FC01662319F480E090E00895809198
:107A4000FA022091CA058E3358F133279927CD9732
:107A5000289FA001299F500D389F500D1124CA0165
:107A6000892F990F990B8095282F3327629FD0017A
:107A700011248B2F992787FD9A95482F8AE2489FDA
:107A8000B0011124759567957595679575956795FE
:107A900075956795E617F70730F0842F99270895B5
:107AA0002FEF30E0E3CF242F332788E190E0E89FE9
:107AB000B001E99F700DF89F700D1124CB01B90141
:107AC0000E9447C5E62FFF27E358F74E8491489F51
:107AD000F00111248F2F992787FD9A9599270895F2
:107AE0000F93CF93DF93209107034091A006442387
:107AF00021F080912003882394F15091CD05052F2A
:107B000002950F70083070F1819B2EC08091E105C5
:107B1000992733278217930710F140FF04C002977B
:107B200082179307C8F180912003877F80932003F9
:107B30002091FB023091FC0240915806642F772778
:107B40006F7070706230710559F163E02C3F360739
:107B500070F02FEF30E030919D06321788F480E00E
:107B600090E0A5C1189491F680917806D1CF369512
:107B7000279536952795332730919D06321778F350
:107B800080915608882399F0992782959295907F45
:107B90009827807F98278BC1809120038860C6CF6B
:107BA000369527953695279536952795E4CF2091DC
:107BB000F80224FF23C090910703A091A905A917FB
:107BC000E8F0409101034B3950F64091A705493C3C
:107BD00008F060C1B9E14B9FA00111242091A805D4
:107BE000293C08F04FC1E9E12E9F9001112400913A
:107BF000FD026DEC80E00E945A2E59C152955F70D3
:107C0000583008F4BCC08199BDC08091E502992725
:107C10008C599F4FE091ED02DD27CC278E9FD0013C
:107C20009E9FB00DC11D11249D01AE019091E602F1
:107C30008091E402989FD00111246627B39FF00140
:107C4000A29FE001B29FD00DE11DF61FA39FD00DB2
:107C5000E11DF61F11249F01442755278091E3025F
:107C6000992780589F4F6627399FF001289FE00190
:107C7000389FD00DE11DF61F299FD00DE11DF61F85
:107C800011248D2F9E2FAF2FBB279C018091F002D6
:107C9000882311F48091EF02992780509F4F442749
:107CA000399FF001289FE001389FD00DE11DF41F9E
:107CB000299FD00DE11DF41F1124AE01BF01BB2788
:107CC000A72F962F852FDC019093E8028093E7027F
:107CD0008091E9029091EA0244279B9FF0018A9FDC
:107CE000E0019A9FD00DE11DF41F8B9FD00DE11D87
:107CF000F41F1124D295E295F295C0EFFE27FC23E4
:107D0000FE27ED27EC23ED27BF018091EB02992799
:107D100088539F4F4427799FF001689FE001789F27
:107D2000D00DE11DF41F699FD00DE11DF41F11243A
:107D3000AE01BF01BB27A72F962F852FBC01F09165
:107D4000E505F2FD3BC0009107035091970605172A
:107D500008F46AC08091FB029091FC020E94742F8B
:107D60007091C20555274427879F9001979F300D3A
:107D7000411D1124BB27A52F942F832F98C0189441
:107D800009F443CF2091FB023091FC02842F992704
:107D90008F709070029709F44FC073E02C3F370743
:107DA00008F43CC02FEF30E080919C062817A0F427
:107DB0000091EE0204600093EE02D1CE3CEAFF2770
:107DC000EE27839FE001939FD00DE11D11248D2F9D
:107DD0009E2FAF2FBB27C4CF332799270296821738
:107DE000930794F52091EE022B7F2093EE02709181
:107DF00007036091E005671788F12E7F2093EE025C
:107E0000909101034091F205491780F5B0915A080D
:107E1000B1FDA5CE2D7F2093EE02F7CE36952795A6
:107E2000369527953327C0CF809108039927880F6F
:107E3000991F880F991F92CF3695279536952795CC
:107E4000369527953327B0CF2091EE02822F9927C0
:107E500084709070882309F082CEC9CFA091070367
:107E60003091DF05A31760F22160C8CFC091E4070D
:107E7000CC2381F6822F992780FF14C022602093A3
:107E8000EE026DCE285CFDE72F9F9001112428574C
:107E90003C4EADCE485CCDE74C9FA0011124485725
:107EA0005C4E9CCE8D7F892B09F4AFCEB3CFDF9192
:107EB000CF910F910895EF92FF920F93CF93DF939D
:107EC0000E94703DEC01892BB9F14091C905442312
:107ED00009F0A5C020E030E0E22EFF24EE0CFF1CEC
:107EE000EE0CFF1CEC0EFD1E8091C5052091C60511
:107EF000682F620F712D711DAB016F3F710511F07D
:107F000008F04FEF281708F4BBC020E00091FA02F8
:107F100064EA8DE30E94A52DC82FDD27CC0FDD1F5D
:107F2000CC0FDD1F9091EC0289E1989FA0011124F4
:107F3000C40FD51FCE0DDF1DE7E2F3E09091CC0515
:107F4000993CE0F589E1989FC001112422E021507D
:107F5000F89494838383D183C083789437962223C3
:107F6000B1F7E0902703F0902803C0912A03D09145
:107F70002B03CE15DF0560F0E0912E03F0912F0367
:107F8000A0913103B0913203AE17BF0708F09CC037
:107F90003091CB05E091FA025E2F58535C36B0F079
:107FA000E32FFF278F2F9927892B09F435C08FEFF7
:107FB00090E0809330038093290386C0985C8DE71E
:107FC000989FC001112488579C4EC0CFFF27EE0F09
:107FD000FF1FE652F84FE590F49094EA7727662762
:107FE000E99EA001F99E500D611D1124BB27A72F0A
:107FF000962F852F77276627839FA001939F500D8B
:10800000611D1124BB27A72F962F852FFC018F2FD1
:108010009927892B09F0CBCF8E2F9927CACF809132
:10802000FA022091CA058E3370F133279927CD9734
:10803000289FB001299F700D389F700D1124872F44
:10804000992787FD9A958095282F3327429FD00145
:1080500011248B2F992787FD9A95482F8AE2489FF4
:1080600070011124F594E794F594E794F594E7945E
:10807000F594E794CE15DF0548F0242F33272CCF55
:10808000821B282F43CF2FEF30E0E0CF242F332760
:1080900088E190E0C89FB001C99F700DD89F700D16
:1080A0001124CB01B9010E9447C5E62FFF27E358F1
:1080B000F74E8491489FF00111248F2F992787FD57
:1080C0009A95282F332708CFDF91CF910F91FF90FA
:1080D000EF9008950F932091090330910A0336958C
:1080E0002795369527959091A30689E1989FC00121
:1080F00011248217930788F4281B390BC90180705B
:10810000892B71F4022F20E140E060911206842F48
:108110000E94A52D8093F30205C01092F30202C0C5
:108120000FEFF1CF0F9108950F9320910903309134
:108130000A0336952795369527959091FF0509E115
:10814000909FA00111248091CD058F70883070F030
:10815000809B0EC01092F4021092F002F8944091AD
:10816000F8024F7B4093F802789423C0189491F75B
:108170004217530778F7241B350BD901A070AB2B9E
:10818000B1F4022F20E140E060911206842F0E949A
:10819000A52D8093F402F8943091F8023064309366
:1081A000F80278942091DD052093F00202C00FEFD1
:1081B000E9CF0F9108950F93CF9320910903309148
:1081C0000A0336952795369527959091A30689E160
:1081D000989FC00111248217930708F052C0281BF2
:1081E000390BC9018070892B09F085C0022F20E16D
:1081F00040E060911206842F0E94A52D8093F30227
:10820000C091F3020091A006002309F043C0209121
:10821000090330910A033695279536952795909155
:10822000FF0579E1979FA00111246091CD056F7042
:10823000683008F43DC0809B3EC01092F40210925A
:10824000F002F8945091F8025F7B5093F802789412
:108250008091F402C81708F4C82F8091F102C81762
:1082600008F4C82F0E943C6A8091F202C81708F4F3
:10827000C82FC13108F0C0E1F894C0931E03789470
:108280003EC01092F302C091F3020091A0060023B9
:1082900009F4BDCF8091200399278C709070892BB1
:1082A00009F4B5CFF89420E120931E03789427C0F9
:1082B000189409F0C2CF4217530708F0BECF241B11
:1082C000350BD901A070AB2BC1F00FEF20E140E0DE
:1082D00060911206842F0E94A52D8093F402F894D9
:1082E0004091F80240644093F80278943091DD05A3
:1082F0003093F002ADCF0FEF7ACF022FE7CFCF91BF
:108300000F9108950F93CF93DF932091C7052223F8
:1083100009F432C08091490290914A02DD27CC27AE
:10832000829FD001929FB00DC11D11249D01AE010D
:10833000809158069927929582958F7089279F7012
:108340008927843009F451C0813009F451C088E094
:1083500090E004C056954795379527958A95D2F7B2
:108360000091C805200F311D2138310508F43AC0AD
:10837000C9018058904002C080E991E09093FC02CE
:108380008093FB02E0914502F0914602F695E79555
:10839000F695E795F695E795E050FD4F34913093CB
:1083A000FD02209147023091480236952795369577
:1083B000279536952795B90160507E4FFB01449172
:1083C0004093FE0220503F4FF90124914091E20575
:1083D000241788F4009107036EE088E00E94A52D21
:1083E000282F09C080E090E0C9CF87E090E0B1CFAE
:1083F00089E090E0AECF2093E40280914302909117
:108400004402969587959695879596958795082F1A
:108410002FEF40E06091EB058091EA050E94DF2D8F
:108420008093010380913F02909140029695879539
:108430009695879596958795982F8091E605989FB4
:10844000C0011124880F892F881F990B91959927B6
:108450008093FA02109200031092FF02DF91CF91F5
:108460000F910895CF93DF938091E50583FF55C069
:108470002091C705222309F052C080E991E0AC01A8
:1084800056954795569547956091E905262F3327D0
:1084900064E670E0DB01A21BB30B4A175B0708F42C
:1084A0006EC0260F371F2417350708F468C0CA01AD
:1084B0009070880F991F880F991F880F991F9093AC
:1084C0004C0280934B024436510508F06DC0641B8A
:1084D000750BAAE9B0E06A9FA0016B9F500D7A9FCF
:1084E000500D1124FA019F01442755272050304890
:1084F0004F4F5F4FCA01B90124E630E040E050E041
:108500000E941CC5DC01CB017FE0B695A79597952D
:1085100087957A95D1F7982F61C094E65FC0409116
:10852000490250914A02DD27CC27429FD001529F39
:10853000B00DC11D11249D01AE01809158069927EF
:10854000929582958F7089279F708927843031F1A9
:10855000813009F440C088E090E004C0569547950A
:10856000379527958A95D2F75091C805250F311D6B
:1085700021383105B0F0C9018058904080CFC0E269
:10858000D3E0D0934C02C0934B0294E6F894209130
:10859000F80222602093F802789420C087E090E0EF
:1085A000DCCF80E090E06BCF2AE930E0429FB00161
:1085B000439F700D529F700D1124CB0188529C4334
:1085C000AA27BB2720E030E840E050E0281B390B09
:1085D0004A0B5B0B8FCF89E090E0BFCF9093E60210
:1085E000DF91CF9108950F93F8944091F702509145
:1085F0000703009101036091FF02709100038091D5
:10860000CD0582958F70883038F080B399279C0112
:108610002270307081FD85C0822F2091F802207277
:1086200090910D03789441FD55C0882309F052C004
:1086300030917406351708F04DC040915B06401725
:1086400008F448C080917506882309F040C08091E5
:108650007606882351F09927880F991F880F991F54
:10866000880F991F86179707A8F1222321F5F89400
:108670008091F80280628093F802E0918C062E2FA0
:10868000207FF0E82F27EF704E2F552742305105FD
:1086900009F464C1433051050CF029C1411551055D
:1086A00009F476C14130510509F4BDC17894609157
:1086B00021066093EF0220E04091E80560910406F6
:1086C0008091D9050E94A52D8093F1021FC28917C0
:1086D00008F0BDCF222309F419C2F8942091F802C2
:1086E0002F7D2093F80200918C06202F207F0F70A1
:1086F000402F552742305105B1F143305105A4F0C8
:108700004630510509F463C04730510509F479C07A
:10871000BEEFB0930D0378941092EF021092F10225
:10872000F5C121E030E078CF41155105B1F141307C
:10873000510571F727FDFDC0822F99278077907032
:108740009595879595958795959587959595879511
:1087500002C0440F551F8A95E2F7542F509588B3F5
:10876000852388BBD5CF27FD66C03327207730709F
:1087700035952795359527953595279535952795E1
:1087800081E090E002C0880F991F2A95E2F7682FD8
:10879000609585B3862385BBBBCF27FD63C0332798
:1087A0002077307035952795359527953595279500
:1087B0003595279581E090E002C0880F991F2A9592
:1087C000E2F7982F90958BB389238BBBA1CF27FD20
:1087D00060C03327207730703595279535952795DC
:1087E000359527953595279581E090E002C0880F53
:1087F000991F2A95E2F7782F709582B3872382BB61
:1088000087CF27FD5DC033272077307035952795BA
:1088100035952795359527953595279581E090E0F5
:1088200002C0880F991F2A95E2F7A82FA09583B15F
:108830008A2383B96DCF822F992780779070959581
:10884000879595958795959587959595879521E039
:1088500030E002C0220F331F8A95E2F785B3822BE6
:1088600085BB56CF822F99278077907095958795F5
:1088700095958795959587959595879521E030E015
:1088800002C0220F331F8A95E2F78BB3822B8BBB7A
:108890003FCF822F992780779070959587959595F2
:1088A0008795959587959595879521E030E002C04D
:1088B000220F331F8A95E2F782B3822B82BB28CF27
:1088C000822F9927807790709595879595958795B4
:1088D000959587959595879521E030E002C0220F08
:1088E000331F8A95E2F783B1822B83B911CF4630CB
:1088F000510509F467C04730510509F0D7CE27FD6F
:10890000D9C0332720773070359527953595279531
:10891000359527953595279581E090E002C0880F21
:10892000991F2A95E2F7582F509583B1852383B973
:10893000BDCE822F992780779070959587959595D4
:108940008795959587959595879502C0440F551FF6
:108950008A95E2F788B3842B88BBDACE27FD4CC01A
:1089600033272077307035952795359527953595A0
:1089700027953595279581E090E002C0880F991FD3
:108980002A95E2F7482F409585B3842385BB8ECE88
:1089900027FD62C0332720773070359527953595B0
:1089A0002795359527953595279581E090E002C06C
:1089B000880F991F2A95E2F7382F30958BB38323C0
:1089C0008BBB74CE27FD5FC0332720773070359581
:1089D000279535952795359527953595279581E0E8
:1089E00090E002C0880F991F2A95E2F7982F909582
:1089F00082B3892382BB5ACE822F992780779070C9
:108A0000959587959595879595958795959587954E
:108A100021E030E002C0220F331F8A95E2F785B3D0
:108A2000822B85BB43CE27FD5CC0822F99278077A0
:108A3000907095958795959587959595879595953A
:108A4000879502C0440F551F8A95E2F7242F209581
:108A500088B3822388BB2ACE822F99278077907093
:108A600095958795959587959595879595958795EE
:108A700021E030E002C0220F331F8A95E2F78BB36A
:108A8000822B8BBB13CE822F992780779070959580
:108A9000879595958795959587959595879521E0E7
:108AA00030E002C0220F331F8A95E2F782B3822B97
:108AB00082BBFCCD822F9927807790709595879502
:108AC00095958795959587959595879521E030E0C3
:108AD00002C0220F331F8A95E2F783B1822B83B93C
:108AE000E5CD822F992780779070959587959595FC
:108AF0008795959587959595879502C0440F551F45
:108B00008A95E2F788B3842B88BBD0CD0F91089566
:108B1000CF93DF93F89420910303309104034091A5
:108B20000503509106037894809138089091390894
:108B3000A0913A08B0913B08281739074A075B070C
:108B400040F4209338083093390840933A08509302
:108B50003B08C0913408D0913508E0913608F09177
:108B60003708C217D307E407F50740F42093340809
:108B7000309335084093360850933708CA01AA2726
:108B8000BB27892B61F0F89424E630E030930A0388
:108B900020930903789481E08093070368C0B901AA
:108BA000809162069927880F991F880F991F2817AF
:108BB000390778F4232B09F44FC03FEF30930703B4
:108BC000F8944CE953E650930A03409309037894D0
:108BD0004EC08091CE059927382F22278091CF054E
:108BE0009927282B392BA4ECB9E044273B9FF001AF
:108BF0002A9FE0013A9FD00DE11DF41F2B9FD00D5D
:108C0000E11DF41F11249B0144275527BE01CF010C
:108C10000E945BC5DA01C901F89430930A032093DE
:108C20000903789459E2FF27EE27859FE001959F7D
:108C3000D00DE11D1124D295E295F295C0EFFE27EB
:108C4000FC23FE27ED27EC23ED279F01A32FBB2755
:108C5000AB2B59F08FEFA0CF10920703F89410922E
:108C60000A0310920903789402C020930703DF914E
:108C7000CF910895F8948091F7028260837F80936A
:108C8000F70278940895CF92DF92EF92FF920F93BC
:108C90001F93CF93DF934091A505442309F419C195
:108CA000809101038B3908F014C1493C08F4E3C0FA
:108CB000485C1DE7419FA001112448575C4ED090AD
:108CC000A605FF27EE274D9DE0015D9DD00DE11D1E
:108CD00011248D2F9E2FAF2FBB270091FD029C01E9
:108CE0006DEC80E00E945A2EAC0120912703309158
:108CF0002803C0902A03D0902B03C216D30660F03D
:108D000060912E0370912F03E0903103F0903203B5
:108D1000E616F70608F037C03091CB05E091FA026D
:108D20007E2F78537C3608F0AEC0FF27EE0FFF1F72
:108D3000E652F84FA591B49194EAFF27EE27A99F38
:108D4000E001B99FD00DE11D11248D2F9E2FAF2F73
:108D5000BB27FF27EE27839FE001939FD00DE11DE6
:108D600011248E019F01BB27A32F922F812FFC017D
:108D7000CF2FDD27CD2B09F483C08FEF90E08093B8
:108D80003003809329034115510509F4A2C0E7E29D
:108D9000F3E09091CC05993C08F078C089E1989F68
:108DA000C001112422E02150F894948383835183DD
:108DB0004083789437962223B1F74091D30750919E
:108DC000D40700918800109189001093D407009374
:108DD000D3070417150748F4E091D507F091D6079B
:108DE0003196F093D607E093D507C0912703D09131
:108DF00028032097F1F0C0902A03D0902B0378012C
:108E0000EC0EFD1EF0922D03E0922C03E1ECF8E154
:108E1000549130913607352730933607352309F0C2
:108E20004BC068E0C7010E94ED870091D307109105
:108E3000D407C0912E03D0912F032097C9F0C09082
:108E40003103D09032037801EC0EFD1EF092340312
:108E5000E0923303E2ECF8E12491B0913607B227B7
:108E6000B0933607B223D1F469E0C7010E94ED87C1
:108E70000E941E8B2EC009E1409FA00111241FCF2C
:108E80008E2F99277CCFE32FFF2772CF985C8DE739
:108E9000989FC001112488579C4E84CF0E94AA47F6
:108EA000D6015396AC17BD07F8F66BE0C8018C0DE0
:108EB0009D1D0E94ED87DCCF0E949E47C601439610
:108EC0008C179D0708F0ADCF6AE0C8018C0D9D1D81
:108ED000AACFDF91CF911F910F91FF90EF90DF907C
:108EE000CF9008953FB53F733FBDC59A209165006F
:108EF000277F20936500809124038E7F8093240335
:108F0000882329F440910A024F7740930A0208957A
:108F10003FB53F7C3FBDC69A209165002F7E2093D0
:108F20006500809124038D7F80932403882329F496
:108F300040910A024F7740930A02089520910A0255
:108F4000206820930A028091240381608093240387
:108F5000C598089520910A02206820930A02809102
:108F60002403826080932403C69808959091290376
:108F70008AE0989FA00111245BBD4ABD2FB5206CEB
:108F80002FBD809165008860809365000895909161
:108F900030038AE0989FA001112459BD48BD2FB528
:108FA00020632FBD809165008061809365000895E6
:108FB00080917006282F207F90E829278F70482FF6
:108FC00055274230510559F1433051054CF0463098
:108FD000510509F472C04730510509F454C0089591
:108FE00041155105B1F141305105C9F727FD96C032
:108FF000822F99278077907095958795959587957D
:10900000959587959595879502C0440F551F8A952C
:10901000E2F7342F309588B3832388BB089527FD6A
:1090200066C033272077307035952795359527957D
:10903000359527953595279581E090E002C0880FFA
:10904000991F2A95E2F7482F409585B3842385BB65
:10905000089527FD78C03327207730703595279500
:1090600035952795359527953595279581E090E09D
:1090700002C0880F991F2A95E2F7282F20958BB3FD
:1090800082238BBB089527FD8CC033272077307057
:1090900035952795359527953595279535952795B8
:1090A00081E090E002C0880F991F2A95E2F7A82F6F
:1090B000A09573B17A2373B9089527FD5BC0332758
:1090C00020773070359527953595279535952795D7
:1090D0003595279581E090E002C0880F991F2A9569
:1090E000E2F7582F509582B3852382BB0895822FD3
:1090F0009927807790709595879595958795959503
:1091000087959595879521E030E002C0220F331FA7
:109110008A95E2F785B3822B85BB0895822F992724
:109120008077907095958795959587959595879576
:109130009595879502C0440F551F8A95E2F788B32D
:10914000842B88BB0895822F9927807790709595FE
:10915000879595958795959587959595879521E020
:1091600030E002C0220F331F8A95E2F78BB3822BC7
:109170008BBB0895822F992780779070959587955E
:1091800095958795959587959595879521E030E0FC
:1091900002C0220F331F8A95E2F782B3822B82BB73
:1091A0000895822F9927807790709595879595954A
:1091B0008795959587959595879521E030E002C034
:1091C000220F331F8A95E2F763B1622B63B90895CA
:1091D00080917006282F207F8F70482F55274230AE
:1091E000510559F1433051054CF04630510509F411
:1091F00072C04730510509F454C008954115510516
:10920000B1F141305105C9F727FD96C0822F99274A
:109210008077907095958795959587959595879585
:109220009595879502C0440F551F8A95E2F7242F24
:10923000209588B3822388BB089527FD66C0332715
:109240002077307035952795359527953595279555
:109250003595279581E090E002C0880F991F2A95E7
:10926000E2F7382F309585B3832385BB089527FD1A
:1092700078C0332720773070359527953595279519
:10928000359527953595279581E090E002C0880FA8
:10929000991F2A95E2F7982F90958BB389238BBB62
:1092A000089527FD8CC0332720773070359527959A
:1092B00035952795359527953595279581E090E04B
:1092C00002C0880F991F2A95E2F7782F709563B135
:1092D000672363B9089527FD5BC03327207730707B
:1092E0003595279535952795359527953595279566
:1092F00081E090E002C0880F991F2A95E2F7482F7D
:10930000409582B3842382BB0895822F992780776A
:109310009070959587959595879595958795959551
:10932000879521E030E002C0220F331F8A95E2F7D3
:1093300085B3822B85BB0895822F99278077907003
:109340009595879595958795959587959595879505
:1093500002C0440F551F8A95E2F788B3842B88BB5F
:109360000895822F99278077907095958795959588
:109370008795959587959595879521E030E002C072
:10938000220F331F8A95E2F78BB3822B8BBB089594
:10939000822F9927807790709595879595958795D9
:1093A000959587959595879521E030E002C0220F2D
:1093B000331F8A95E2F782B3822B82BB0895822FF6
:1093C0009927807790709595879595958795959530
:1093D00087959595879521E030E002C0220F331FD5
:1093E0008A95E2F753B1522B53B908951092F702C0
:1093F0006091F80264616093F8021092F9025FEFE5
:109400005093E8071092F5074FEF5FEF60E070E0D0
:109410004093030350930403609305037093060382
:109420001092070310920A031092090330916B0601
:1094300030930E032BE020938401F8948091700602
:10944000282F207F8F70482F55274230510509F46F
:1094500045C04330510514F14630510509F413C19C
:109460004730510509F053C027FDD9C13327207774
:1094700030703595279535952795359527953595F0
:10948000279581E090E002C0880F991F2A95E2F7A6
:10949000E82FE09583B18E2383B939C0411551057A
:1094A00009F4BDC04130510591F527FD32C1822F2D
:1094B000992780779070959587959595879595953F
:1094C00087959595879502C0440F551F8A95E2F7B9
:1094D000742F709588B3872388BB19C027FD03C1FB
:1094E0003327207730703595279535952795359515
:1094F00027953595279581E090E002C0880F991F48
:109500002A95E2F7A82FA09585B38A2385BB789486
:109510000000F894F09110062F2F207FFF704F2F3E
:1095200055274230510509F446C0433051050CF52A
:109530004115510509F459C04130510509F09CC14C
:1095400027FDFCC0822F992780779070959587958D
:1095500095958795959587959595879502C0440F24
:10956000551F8A95E2F7342F309588B3832388BB43
:1095700083C14630510509F46CC04730510509F0EC
:109580007BC127FD63C13327207730703595279540
:1095900035952795359527953595279581E090E068
:1095A00002C0880F991F2A95E2F7682F609583B152
:1095B000862383B961C127FD80C0332720773070AF
:1095C0003595279535952795359527953595279583
:1095D00081E090E002C0880F991F2A95E2F7482F9A
:1095E000409585B3842385BB47C127FDD3C033276E
:1095F00020773070359527953595279535952795A2
:109600003595279581E090E002C0880F991F2A9533
:10961000E2F7282F20958BB382238BBB2DC127FD2A
:10962000A2C033272077307035952795359527953B
:10963000359527953595279581E090E002C0880FF4
:10964000991F2A95E2F7982F90958BB389238BBBAE
:109650005ECF27FDCDC03327207730703595279515
:1096600035952795359527953595279581E090E097
:1096700002C0880F991F2A95E2F7582F509582B3A0
:10968000852382BBF9C027FD9CC03327207730702B
:1096900035952795359527953595279535952795B2
:1096A00081E090E002C0880F991F2A95E2F7B82F59
:1096B000B09582B38B2382BB2ACF822F99278077E4
:1096C000907095958795959587959595879595959E
:1096D000879521E030E002C0220F331F8A95E2F720
:1096E00085B3822B80CF822F9927807790709595B4
:1096F000879595958795959587959595879521E07B
:1097000030E002C0220F331F8A95E2F785B3822B27
:10971000FDCE822F992780779070959587959595A6
:109720008795959587959595879502C0440F551F08
:109730008A95E2F788B3842B88BBE9CE822F9927DC
:109740008077907095958795959587959595879550
:109750009595879502C0440F551F8A95E2F788B307
:10976000842B88BB89C0822F99278077907095952C
:10977000879595958795959587959595879521E0FA
:1097800030E002C0220F331F8A95E2F78BB3822BA1
:109790008BBBBDCE822F992780779070959587954A
:1097A00095958795959587959595879521E030E0D6
:1097B00002C0220F331F8A95E2F78BB3822B8BBB3B
:1097C0005BC0822F992780779070959587959595A6
:1097D0008795959587959595879521E030E002C00E
:1097E000220F331F8A95E2F782B3822B82BB8FCE82
:1097F000822F992780779070959587959595879575
:10980000959587959595879521E030E002C0220FC8
:10981000331F8A95E2F782B3822B82BB2DC0822F41
:1098200099278077907095958795959587959595CB
:1098300087959595879521E030E002C0220F331F70
:109840008A95E2F783B1822B83B961CE822F992763
:10985000807790709595879595958795959587953F
:109860009595879521E030E002C0220F331F8A953D
:10987000E2F783B1822B83B978940000F894809149
:109880000A028F7380930A02789480E090E00E942D
:10989000133A089580917006282F207F90E8292799
:1098A0008F70482F55274230510509F445C0433089
:1098B000510514F14630510509F472C04730510585
:1098C00009F0F7C027FDDFC03327207730703595CA
:1098D000279535952795359527953595279581E0D9
:1098E00090E002C0880F991F2A95E2F7682F6095D3
:1098F00083B1862383B9DDC041155105B9F14130EB
:10990000510509F0D6C027FD7BC0822F99278077AB
:10991000907095958795959587959595879595954B
:10992000879502C0440F551F8A95E2F7342F309572
:1099300088B3832388BBBDC027FD4CC03327207765
:10994000307035952795359527953595279535951B
:10995000279581E090E002C0880F991F2A95E2F7D1
:10996000482F409585B3842385BBA3C027FD5DC0E8
:109970003327207730703595279535952795359580
:1099800027953595279581E090E002C0880F991FB3
:109990002A95E2F7282F20958BB382238BBB89C0B1
:1099A00027FD5AC033272077307035952795359598
:1099B0002795359527953595279581E090E002C04C
:1099C000880F991F2A95E2F7582F509582B3852367
:1099D00082BB6FC0822F992780779070959587956D
:1099E00095958795959587959595879521E030E094
:1099F00002C0220F331F8A95E2F785B3822BB4CFC2
:109A0000822F992780779070959587959595879562
:109A1000959587959595879502C0440F551F8A9512
:109A2000E2F788B3842B88BB44C0822F99278077C4
:109A3000907095958795959587959595879595952A
:109A4000879521E030E002C0220F331F8A95E2F7AC
:109A50008BB3822B8BBB2DC0822F99278077907080
:109A600095958795959587959595879595958795DE
:109A700021E030E002C0220F331F8A95E2F782B363
:109A8000822B82BB16C0822F992780779070959584
:109A9000879595958795959587959595879521E0D7
:109AA00030E002C0220F331F8A95E2F783B1822B88
:109AB00083B97091F70271607093F702089532E0F4
:109AC0003FBD29E12EBD88EE93E097BD86BD089588
:109AD0001F920F920FB60F9211240F931F932F9383
:109AE0003F934F935F936F937F938F939F93AF9326
:109AF000BF93CF93DF93EF93FF9350910A02506887
:109B000050930A0210912403126010932403C69804
:109B100030915608032F112702951295107F1027B8
:109B2000007F102769E0C8010E949D8C4091D307F7
:109B30005091D407040F151F10933403009333037F
:109B40000091D5071091D607EA01F8018091D90755
:109B50009091DA07A091DB07B091DC079E01AF017D
:109B6000281B390B4A0B5B0B209303033093040330
:109B7000409305035093060320910303309104039F
:109B8000409105035091060380913808909139085F
:109B9000A0913A08B0913B08281739074A075B079C
:109BA00080F4209103033091040340910503509108
:109BB0000603209338083093390840933A085093AD
:109BC0003B08209103033091040340910503509119
:109BD00006038091340890913508A0913608B09121
:109BE000370882179307A407B50780F44091030351
:109BF000509104036091050370910603409334086B
:109C0000509335086093360870933708C093D9078E
:109C1000D093DA07E093DB07F093DC076091F8025A
:109C200061606093F802A0911808B091190811962C
:109C3000B0931908A09318080E941E8BFF91EF9112
:109C4000DF91CF91BF91AF919F918F917F916F9154
:109C50005F914F913F912F911F910F910F900FBEE8
:109C60000F901F9018951F93CF93DF9310921802B7
:109C7000C0913503D0913603E0913703F09138035A
:109C8000CF01AA27BB270097A105B10561F0A091DC
:109C90004008B09141081196B0934108A093400844
:109CA00010920B033DC02091250330912603A09113
:109CB0003503B0913603CC273B9FB0012A9FA0010A
:109CC0003A9F500D611D7C1F2B9F500D611D7C1F05
:109CD0001124252F362F472F552710916806612F05
:109CE000772745E253E01127539FF001429FE0019F
:109CF000529FD00DE11DF11F439FD00DE11DF11FBB
:109D00001124CF01AA27BB27681B790BE72FFF2758
:109D1000EF2B21F03FEF30930B0302C060930B0356
:109D2000DF91CF911F910895982FE5EAF5E0A0E02B
:109D3000B0E08FEF182E0E9485C59130E9F0E9E37D
:109D4000F3E0AFEFB0E088E592E0019724F00E94E5
:109D50007DC50192FACFE4EAF6E0A7E5B3E030E989
:109D6000132E0E9485C5E1E9F5E0A7EEB3E084E19A
:109D7000182E0E9485C50895E9E3F3E04BEF53E008
:109D800088E592E0DA01019724F00E947DC50192F6
:109D9000FACFE4EAF6E0485A5D4F20E9DA01122EE4
:109DA0000E9485C5E1E9F5E040575F4F84E1DA01A3
:109DB000182E0E9485C50895CF93DF93982F809128
:109DC000390282FD6BC0892F99278B369105F9F0F6
:109DD0008C36910564F48336910509F446C08436C7
:109DE000910524F58236910509F058C04DC08E3694
:109DF000910509F43FC08F36910564F58C369105C5
:109E000009F04CC0E9EEF4E08FEA92E004C0E5E826
:109E1000F5E08BE493E0A62FBB27EA0FFB1FA80F0A
:109E2000B91F0E947DC5302D308338C0843691051E
:109E300031F18A36910591F5C62FDD27CC0FDD1F54
:109E4000DE01A150BF4F0E948AC5C75CDC4FF98379
:109E5000E88324C082379105E1F084379105F1F45D
:109E6000EDE9F5E083EF93E0D6CFE5EAF5E080E0B9
:109E700090E0D1CFE4EAF6E087E593E0CCCFE9E5E6
:109E8000F4E08FE192E0C7CFE1E9F5E087EE93E0FF
:109E9000C2CFE9E7F5E08FE393E0BDCFDF91CF914B
:109EA0000895109239020895982F80911F068138E5
:109EB00018F020E820931F0630911E06313818F064
:109EC00040E840931E065091390252FF03C080E0E3
:109ED00090E00895923008F090E0709139027F7020
:109EE00070933902892F992782959295907F9827B0
:109EF000807F982760913902682B666060933902F1
:109F000081E090E00895CF93DF9340911902509142
:109F10001A0220911B0230911C02DA01A20FB31F1A
:109F20000E947DC5802DC0913B02D0913C02F90179
:109F3000EC0FFD1FE0818E1731F18E1781F0420F7B
:109F4000531FDA010E2E0E948FC580913902816065
:109F500080933902E39A20911B0230911C02C09138
:109F60000B02D0910C0221972C173D0718F081E0CD
:109F700090E025C02F5F3F4F30931C0220931B02BF
:109F800080E090E01CC060910B0270910C02615067
:109F900070402617370788F62F5F3F4F30931C021B
:109FA00020931B02DA01A20FB31F0E947DC5802DF2
:109FB000F901EC0FFD1FE0818E1759F3BECFDF9141
:109FC000CF910895FF920F931F93CF93DF93FF24B8
:109FD00080910E02282F33272230310509F479C0F1
:109FE000233031055CF02330310509F452C12530AE
:109FF000310509F40FC131E0F32E20C221153105DE
:10A0000009F4CBC021303105B1F76091190270918C
:10A010001A0220911B0230911C02E901DB01A20F00
:10A02000B31F0E947DC5802D00913B0210913C0220
:10A03000F901E00FF11FE0818E1709F4B6C18E1708
:10A0400081F0620F731FDB010E2E0E948FC51091ED
:10A050003902116010933902E39A20911B0230916A
:10A060001C02C0910B02D0910C0221972C173D07C6
:10A0700008F408C120913902207F09F4DCC1309135
:10A08000390232953F70032F11278CEF92E0089F21
:10A09000F001099FF00D189FF00D1124CF0185509C
:10A0A0009C4F90931A028093190269E373E07093B6
:10A0B0003C0260933B0248E552E050930C0240930F
:10A0C0000B0210921C0210921B0282E080930E027F
:10A0D000B5C16091190270911A0220911B02309152
:10A0E0001C02E901DB01A20FB31F0E947DC5802D78
:10A0F00000913B0210913C02F901E00FF11FE08159
:10A100008E1709F464C08E1781F0620F731FDB0194
:10A110000E2E0E948FC55091390251605093390222
:10A12000E39A20911B0230911C02C0910B02D09146
:10A130000C0221972C173D0708F4A4C07091390236
:10A14000707F09F4F9C09091390292959F70292F80
:10A1500033278CEF92E0289FF001299FF00D389F64
:10A16000F00D1124CF018D5A994F90931A028093CC
:10A17000190244EA56E050933C0240933B0200E946
:10A1800010E010930C0200930B0210921C0210922C
:10A190001B0283E080930E0251C160E070E0709377
:10A1A0001A026093190245EA55E050933C0240932D
:10A1B0003B020FEF10E010930C0200930B02309360
:10A1C0001C0220931B0281E080930E0237C1409154
:10A1D0000B0250910C02415050402417350708F0F3
:10A1E00092CF9E012F5F3F4F30931C0220931B02A2
:10A1F000DB01A20FB31F0E947DC5802DF901E00F86
:10A20000F11FE0818E1709F07ECFE9012417350791
:10A2100040F379CF6091190270911A0220911B02CC
:10A2200030911C02E901DB01A20FB31F0E947DC522
:10A23000802D00913B0210913C02F901E00FF11FCB
:10A24000E0818E1709F47BC08E1781F0620F731FB7
:10A25000DB010E2E0E948FC53091390231603093A0
:10A260003902E39A20911B0230911C02C0910B022B
:10A27000D0910C0221972C173D0720F086E08093A7
:10A280000E02DCC02F5F3F4F30931C0220931B0255
:10A29000D5C06091190270911A0220911B02309171
:10A2A0001C02E901DB01A20FB31F0E947DC5802DB6
:10A2B00000913B0210913C02F901E00FF11FE08197
:10A2C0008E1709F495C08E1781F0620F731FDB01A2
:10A2D0000E2E0E948FC5B0913902B160B093390241
:10A2E000E39A20911B0230911C02C0910B02D09185
:10A2F0000C0221972C173D0728F2F0913902F07FCC
:10A3000009F040C087EE93E090931A0280931902FF
:10A3100001E915E010933C0200933B0284E190E0D8
:10A3200090930C0280930B0210921C0210921B025D
:10A3300085E080930E0282C087E593E016CF4091BE
:10A340000B0250910C02415050402417350708F081
:10A350007BCF9E012F5F3F4F30931C0220931B0247
:10A36000DB01A20FB31F0E947DC5802DF901E00F14
:10A37000F11FE0818E1709F067CFE9012417350737
:10A3800040F362CF1091390212951F70212F3327AD
:10A39000ECEFF2E02E9FB0012F9F700D3E9F700DED
:10A3A0001124CB018D51994FAFCF40910B025091A9
:10A3B0000C02415050402417350708F040CE9E0152
:10A3C0002F5F3F4F30931C0220931B02DB01A20F33
:10A3D000B31F0E947DC5802DF901E00FF11FE081C0
:10A3E0008E1709F02CCEE9012417350740F327CE4C
:10A3F00040910B0250910C024150504024173507F8
:10A4000008F061CF9E012F5F3F4F30931C022093D5
:10A410001B02DB01A20FB31F0E947DC5802DF90135
:10A42000E00FF11FE0818E1709F04DCFE9012417ED
:10A43000350740F348CF8FEF90E033CE8F2D99272B
:10A44000DF91CF911F910F91FF9008958091390274
:10A4500082FF23C02091390221FF0DC040913902B3
:10A460004D7F4093390210920E0230910A02306102
:10A4700030930A0208955091390250FD0EC00E9497
:10A48000E24F882351F0709139027B7F709339023B
:10A4900060910A026F7E60930A0208951F920F92E4
:10A4A0000FB60F9211248F93809139028E7F809383
:10A4B0003902E3988F910F900FBE0F901F9018955F
:10A4C0008091FD029091EC059817E0F4F89430919A
:10A4D000EE05232F207F90E829273F70432F552733
:10A4E0004230510509F46DC0433051050CF448C0A9
:10A4F0004630510509F4D8C04730510509F420C150
:10A5000078940895B091FD02EB2FFF27A92FBB2768
:10A510008091ED05A81BB109AE17BF0784F1F8942F
:10A52000F091EE052F2F207FFF704F2F55274230DF
:10A53000510509F461C0433051050CF092C041153A
:10A54000510509F4CBC041305105C1F427FDE3C1E9
:10A55000822F992780779070959587959595879507
:10A56000959587959595879502C0440F551F8A95B7
:10A57000E2F7942F909588B3892388BB7894089547
:10A580004115510509F453C04130510509F0B8CFC8
:10A5900027FD95C1822F9927807790709595879593
:10A5A00095958795959587959595879502C0440FC4
:10A5B000551F8A95E2F7542F509588B3852388BBA1
:10A5C0009FCF27FDD7C0332720773070359527954B
:10A5D00035952795359527953595279581E090E018
:10A5E00002C0880F991F2A95E2F7482F409585B33E
:10A5F000842385BB7894089527FD05C133272077F0
:10A60000307035952795359527953595279535954E
:10A61000279581E090E002C0880F991F2A95E2F704
:10A62000282F209585B3822385BB7894A8CF27FD5A
:10A63000D3C03327207730703595279535952795EA
:10A64000359527953595279581E090E002C0880FD4
:10A65000991F2A95E2F7282F20958BB382238BBB75
:10A660004FCF4630510509F49CC04730510509F0E1
:10A6700085CF27FD39C13327207730703595279551
:10A6800035952795359527953595279581E090E067
:10A6900002C0880F991F2A95E2F7482F409583B191
:10A6A000842383B978946BCF27FD33C03327207779
:10A6B000307035952795359527953595279535959E
:10A6C000279581E090E002C0880F991F2A95E2F754
:10A6D000682F609582B3862382BB12CF27FDAAC064
:10A6E0003327207730703595279535952795359503
:10A6F00027953595279581E090E002C0880F991F36
:10A700002A95E2F7382F30958BB383238BBB78944F
:10A7100036CF822F9927807790709595879595955C
:10A720008795959587959595879521E030E002C0AE
:10A73000220F331F8A95E2F782B3822B82BBE0CED1
:10A7400027FD8FC0332720773070359527953595B5
:10A750002795359527953595279581E090E002C09E
:10A76000880F991F2A95E2F7782F709583B1872378
:10A7700083B9C6CE822F992780779070959587955B
:10A7800095958795959587959595879521E030E0E6
:10A7900002C0220F331F8A95E2F785B3822B85BB57
:10A7A00029CF27FD75C03327207730703595279541
:10A7B00035952795359527953595279581E090E036
:10A7C00002C0880F991F2A95E2F7582F509582B33F
:10A7D000852382BB7894D3CE822F9927807790707F
:10A7E0009595879595958795959587959595879551
:10A7F00021E030E002C0220F331F8A95E2F78BB3CD
:10A80000822B8BBB7DCE822F992780779070959578
:10A81000879595958795959587959595879521E049
:10A8200030E002C0220F331F8A95E2F785B3822BF6
:10A8300085BBFBCE822F9927807790709595879561
:10A8400095958795959587959595879521E030E025
:10A8500002C0220F331F8A95E2F78BB3822B8BBB8A
:10A8600056CF822F992780779070959587959595EB
:10A870008795959587959595879521E030E002C05D
:10A88000220F331F8A95E2F783B1822B83B938CE2A
:10A89000822F9927807790709595879595958795C4
:10A8A000959587959595879521E030E002C0220F18
:10A8B000331F8A95E2F782B3822B82BB8BCF822F24
:10A8C000992780779070959587959595879595951B
:10A8D00087959595879502C0440F551F8A95E2F795
:10A8E00088B3842B88BB0CCE822F992780779070F9
:10A8F0009595879595958795959587959595879540
:10A9000021E030E002C0220F331F8A95E2F783B1C5
:10A91000822B83B9C7CE822F992780779070959527
:10A92000879595958795959587959595879502C077
:10A93000440F551F8A95E2F788B3842B88BB1ECE3F
:10A940008091FD02909195069817E0F4F89430916B
:10A950009906232F207F90E829273F70432F552702
:10A960004230510509F46DC0433051050CF448C024
:10A970004630510509F4D8C04730510509F420C1CB
:10A9800078940895B091FD02EB2FFF27A92FBB27E4
:10A9900080919806A81BB109AE17BF0784F1F894FF
:10A9A000F09199062F2F207FFF704F2F55274230AF
:10A9B000510509F461C0433051050CF092C04115B6
:10A9C000510509F4CBC041305105C1F427FDE3C165
:10A9D000822F992780779070959587959595879583
:10A9E000959587959595879502C0440F551F8A9533
:10A9F000E2F7942F909588B3892388BB78940895C3
:10AA00004115510509F453C04130510509F0B8CF43
:10AA100027FD95C1822F992780779070959587950E
:10AA200095958795959587959595879502C0440F3F
:10AA3000551F8A95E2F7542F509588B3852388BB1C
:10AA40009FCF27FDD7C033272077307035952795C6
:10AA500035952795359527953595279581E090E093
:10AA600002C0880F991F2A95E2F7482F409585B3B9
:10AA7000842385BB7894089527FD05C1332720776B
:10AA800030703595279535952795359527953595CA
:10AA9000279581E090E002C0880F991F2A95E2F780
:10AAA000282F209585B3822385BB7894A8CF27FDD6
:10AAB000D3C0332720773070359527953595279566
:10AAC000359527953595279581E090E002C0880F50
:10AAD000991F2A95E2F7282F20958BB382238BBBF1
:10AAE0004FCF4630510509F49CC04730510509F05D
:10AAF00085CF27FD39C133272077307035952795CD
:10AB000035952795359527953595279581E090E0E2
:10AB100002C0880F991F2A95E2F7482F409583B10C
:10AB2000842383B978946BCF27FD33C033272077F4
:10AB30003070359527953595279535952795359519
:10AB4000279581E090E002C0880F991F2A95E2F7CF
:10AB5000682F609582B3862382BB12CF27FDAAC0DF
:10AB6000332720773070359527953595279535957E
:10AB700027953595279581E090E002C0880F991FB1
:10AB80002A95E2F7382F30958BB383238BBB7894CB
:10AB900036CF822F992780779070959587959595D8
:10ABA0008795959587959595879521E030E002C02A
:10ABB000220F331F8A95E2F782B3822B82BBE0CE4D
:10ABC00027FD8FC033272077307035952795359531
:10ABD0002795359527953595279581E090E002C01A
:10ABE000880F991F2A95E2F7782F709583B18723F4
:10ABF00083B9C6CE822F99278077907095958795D7
:10AC000095958795959587959595879521E030E061
:10AC100002C0220F331F8A95E2F785B3822B85BBD2
:10AC200029CF27FD75C033272077307035952795BC
:10AC300035952795359527953595279581E090E0B1
:10AC400002C0880F991F2A95E2F7582F509582B3BA
:10AC5000852382BB7894D3CE822F992780779070FA
:10AC600095958795959587959595879595958795CC
:10AC700021E030E002C0220F331F8A95E2F78BB348
:10AC8000822B8BBB7DCE822F9927807790709595F4
:10AC9000879595958795959587959595879521E0C5
:10ACA00030E002C0220F331F8A95E2F785B3822B72
:10ACB00085BBFBCE822F99278077907095958795DD
:10ACC00095958795959587959595879521E030E0A1
:10ACD00002C0220F331F8A95E2F78BB3822B8BBB06
:10ACE00056CF822F99278077907095958795959567
:10ACF0008795959587959595879521E030E002C0D9
:10AD0000220F331F8A95E2F783B1822B83B938CEA5
:10AD1000822F99278077907095958795959587953F
:10AD2000959587959595879521E030E002C0220F93
:10AD3000331F8A95E2F782B3822B82BB8BCF822F9F
:10AD40009927807790709595879595958795959596
:10AD500087959595879502C0440F551F8A95E2F710
:10AD600088B3842B88BB0CCE822F99278077907074
:10AD700095958795959587959595879595958795BB
:10AD800021E030E002C0220F331F8A95E2F783B141
:10AD9000822B83B9C7CE822F9927807790709595A3
:10ADA000879595958795959587959595879502C0F3
:10ADB000440F551F8A95E2F788B3842B88BB1ECEBB
:10ADC0002091070380918906821780F590E8F89416
:10ADD00080918A06282F207F29278F70482F55279A
:10ADE00042305105B1F1433051050CF04DC04115D1
:10ADF000510509F06BC027FDD0C033272077307094
:10AE0000359527953595279535952795359527952A
:10AE100081E090E002C0880F991F2A95E2F7982FF1
:10AE200090958BB389238BBB78940895332799270A
:10AE3000029782179307CCF390E0F89480918A06EA
:10AE4000282F207F29278F70482F55274230510502
:10AE500051F627FD74C0332720773070359527953C
:10AE600035952795359527953595279581E090E07F
:10AE700002C0880F991F2A95E2F7382F309585B3C5
:10AE8000832385BB7894D1CF4630510509F43CC06B
:10AE90004730510549F627FD69C0332720773070C8
:10AEA000359527953595279535952795359527958A
:10AEB00081E090E002C0880F991F2A95E2F7582F91
:10AEC000509583B1852383B97894AFCF4130510534
:10AED00009F0AACF27FD8FC0822F99278077907025
:10AEE000959587959595879595958795959587954A
:10AEF00002C0440F551F8A95E2F7242F209588B38E
:10AF0000822388BB789491CF27FD5EC033272077BA
:10AF10003070359527953595279535952795359535
:10AF2000279581E090E002C0880F991F2A95E2F7EB
:10AF3000482F409582B3842382BB789476CF822FAA
:10AF40009927807790709595879595958795959594
:10AF500087959595879521E030E002C0220F331F39
:10AF60008A95E2F785B3822B85BB8CCF822F9927F8
:10AF70008077907095958795959587959595879508
:10AF80009595879521E030E002C0220F331F8A9506
:10AF9000E2F783B1822B83B997CF822F99278077ED
:10AFA00090709595879595958795959587959595A5
:10AFB000879521E030E002C0220F331F8A95E2F727
:10AFC0008BB3822B8BBB30CF822F992780779070E9
:10AFD0009595879595958795959587959595879559
:10AFE00021E030E002C0220F331F8A95E2F782B3DE
:10AFF000822B82BBA2CF822F992780779070959564
:10B00000879595958795959587959595879502C090
:10B01000440F551F8A95E2F788B3842B88BB72CF03
:10B0200040910703509101032091FB023091FC02F3
:10B030008091580699278F709070029709F4A2C0EA
:10B0400083E02C3F3807D8F18FEF90E0982F809164
:10B050007906481708F03FC090E0F89470917F0699
:10B06000272F207F29277F70472F552742305105F2
:10B0700009F46EC0433051050CF048C0411551052C
:10B0800009F487C04130510509F026C127FDCBC026
:10B09000822F9927807790709595879595958795BC
:10B0A000959587959595879502C0440F551F8A956C
:10B0B000E2F7A42FA09588B38A2388BB0DC13695EB
:10B0C000279536952795822F9927982F8091790675
:10B0D000481708F4C1CF20917A06241708F4BCCF92
:10B0E00030917B06531708F4B7CF40917C06451783
:10B0F00008F4B2CF50917D06951708F4ADCF60915A
:10B100007E06691708F4A8CF90E8A7CF463051050E
:10B1100009F459C04730510509F0DEC027FDC6C00B
:10B1200033272077307035952795359527953595B8
:10B1300027953595279581E090E002C0880F991FEB
:10B140002A95E2F7F82FF09583B18F2383B9C4C015
:10B1500027FD53C0332720773070359527953595D7
:10B160002795359527953595279581E090E002C084
:10B17000880F991F2A95E2F7B82FB09585B38B23D6
:10B1800085BBAAC036952795369527953695279580
:10B190009ACF27FD5DC033272077307035952795EE
:10B1A00035952795359527953595279581E090E03C
:10B1B00002C0880F991F2A95E2F7982F90958BB3BC
:10B1C00089238BBB89C027FD5AC033272077307075
:10B1D0003595279535952795359527953595279557
:10B1E00081E090E002C0880F991F2A95E2F7E82FCE
:10B1F000E09582B38E2382BB6FC0822F9927807720
:10B200009070959587959595879595958795959542
:10B21000879521E030E002C0220F331F8A95E2F7C4
:10B2200085B3822BADCF822F99278077907095952B
:10B23000879595958795959587959595879502C05E
:10B24000440F551F8A95E2F788B3842B88BB44C00E
:10B25000822F9927807790709595879595958795FA
:10B26000959587959595879521E030E002C0220F4E
:10B27000331F8A95E2F78BB3822B8BBB2DC0822FB5
:10B280009927807790709595879595958795959551
:10B2900087959595879521E030E002C0220F331FF6
:10B2A0008A95E2F782B3822B82BB16C0822F992740
:10B2B00080779070959587959595879595958795C5
:10B2C0009595879521E030E002C0220F331F8A95C3
:10B2D000E2F783B1822B83B97894089540910703F4
:10B2E000509101032091FB023091FC02809158069D
:10B2F00099278F709070029709F4A2C083E02C3FC9
:10B300003807D8F18FEF90E0982F8091800648178A
:10B3100008F03FC090E0F89470918606272F207FB8
:10B3200029277F70472F55274230510509F46EC0F9
:10B33000433051050CF048C04115510509F487C050
:10B340004130510509F026C127FDCBC0822F992736
:10B350008077907095958795959587959595879524
:10B360009595879502C0440F551F8A95E2F7A42F43
:10B37000A09588B38A2388BB0DC13695279536954D
:10B380002795822F9927982F80918006481708F4D7
:10B39000C1CF20918106241708F4BCCF30918206DA
:10B3A000531708F4B7CF40918306451708F4B2CF7E
:10B3B00050918406951708F4ADCF60918506691702
:10B3C00008F4A8CF90E8A7CF4630510509F459C03A
:10B3D0004730510509F0DEC027FDC6C0332720776E
:10B3E0003070359527953595279535952795359561
:10B3F000279581E090E002C0880F991F2A95E2F717
:10B40000F82FF09583B18F2383B9C4C027FD53C0B3
:10B4100033272077307035952795359527953595C5
:10B4200027953595279581E090E002C0880F991FF8
:10B430002A95E2F7B82FB09585B38B2385BBAAC0B8
:10B440003695279536952795369527959ACF27FDDA
:10B450005DC0332720773070359527953595279532
:10B46000359527953595279581E090E002C0880FA6
:10B47000991F2A95E2F7982F90958BB389238BBB60
:10B4800089C027FD5AC0332720773070359527951E
:10B4900035952795359527953595279581E090E049
:10B4A00002C0880F991F2A95E2F7E82FE09582B332
:10B4B0008E2382BB6FC0822F9927807790709595DD
:10B4C000879595958795959587959595879521E08D
:10B4D00030E002C0220F331F8A95E2F785B3822B3A
:10B4E000ADCF822F99278077907095958795959508
:10B4F0008795959587959595879502C0440F551F1B
:10B500008A95E2F788B3842B88BB44C0822F9927A1
:10B510008077907095958795959587959595879562
:10B520009595879521E030E002C0220F331F8A9560
:10B53000E2F78BB3822B8BBB2DC0822F99278077AC
:10B5400090709595879595958795959587959595FF
:10B55000879521E030E002C0220F331F8A95E2F781
:10B5600082B3822B82BB16C0822F9927807790707E
:10B5700095958795959587959595879595958795B3
:10B5800021E030E002C0220F331F8A95E2F783B139
:10B59000822B83B978940895EF92FF920F931F93B3
:10B5A000CF93C0919E06CF3F09F49FC2F89480913B
:10B5B000030390910403A0910503B09106039C013D
:10B5C000789480919F0611270027289F7001389F4B
:10B5D000F00C011D1124A8019701BB27A52F942F62
:10B5E000832F885F9F4008F46DC0ECEBFFE7F89471
:10B5F000E090D307F090D4076091880070918900A3
:10B600007093D4076093D3076E157F0548F4A0911B
:10B61000D507B091D6071196B093D607A093D5075A
:10B620009B0178944091340750913507241B350BCA
:10B630002E173F0708F459C28F01000F111F021780
:10B64000130708F44EC04E0F5F1F50933507409309
:10B650003407F0903D01F094F0923D01FF2009F491
:10B660004CC0F8942C2F207F10E82127CF704C2F4E
:10B6700055274230510509F4B4C0433051050CF050
:10B680006BC04115510509F4E2C041305105C1F4C8
:10B6900027FD16C2822F9927807790709595879500
:10B6A00095958795959587959595879502C0440FB3
:10B6B000551F8A95E2F7342F309588B3832388BBD2
:10B6C000789413C2B5E05695479537952795BA9566
:10B6D000D1F7F9012335310508F089CFE3E5F0E032
:10B6E00086CF7093350760933407F0903D01F09456
:10B6F000F0923D01FF2009F0B4CFF8942C2F207F69
:10B70000CF704C2F55274230510509F485C0433086
:10B7100051050CF044C04115510509F4B3C0413046
:10B720005105C1F427FDB7C1822F9927807790700A
:10B7300095958795959587959595879595958795F1
:10B7400002C0440F551F8A95E2F7B42FB09588B315
:10B750008B2388BB7894C9C14630510509F4ADC02C
:10B760004730510509F0ACCF27FD67C1332720775B
:10B7700030703595279535952795359527953595CD
:10B78000279581E090E002C0880F991F2A95E2F783
:10B79000682F609583B1862383B97894A6C146301B
:10B7A000510509F4A5C047305105A1F627FD5CC13C
:10B7B0003327207730703595279535952795359522
:10B7C00027953595279581E090E002C0880F991F55
:10B7D0002A95E2F7F82FF09583B18F2383B97894F7
:10B7E00084C127FDA0C03327207730703595279579
:10B7F00035952795359527953595279581E090E0E6
:10B8000002C0880F991F2A95E2F7482F409585B30B
:10B81000842385BB789469C127FD9CC0332720779A
:10B82000307035952795359527953595279535951C
:10B83000279581E090E002C0880F991F2A95E2F7D2
:10B84000C82FC09585B38C2385BB78944EC127FD46
:10B85000AFC03327207730703595279535952795DC
:10B86000359527953595279581E090E002C0880FA2
:10B87000991F2A95E2F7982F90958BB389238BBB5C
:10B88000789433C127FD7DC03327207730703595FC
:10B89000279535952795359527953595279581E0F9
:10B8A00090E002C0880F991F2A95E2F7782F7095D3
:10B8B0008BB387238BBB789418C127FDA7C0332790
:10B8C00020773070359527953595279535952795AF
:10B8D0003595279581E090E002C0880F991F2A9541
:10B8E000E2F7582F509582B3852382BB7894FDC030
:10B8F00027FD75C03327207730703595279535950E
:10B900002795359527953595279581E090E002C0DC
:10B91000880F991F2A95E2F7E82FE09582B38E23CE
:10B9200082BB7894E2C0822F99278077907095959A
:10B93000879595958795959587959595879521E018
:10B9400030E002C0220F331F8A95E2F785B3822BC5
:10B9500085BB60CF822F99278077907095958795CA
:10B9600095958795959587959595879521E030E0F4
:10B9700002C0220F331F8A95E2F785B3822B85BB65
:10B9800064CF822F992780779070959587959595AC
:10B990008795959587959595879521E030E002C02C
:10B9A000220F331F8A95E2F78BB3822B8BBB83CF99
:10B9B000822F992780779070959587959595879593
:10B9C000959587959595879521E030E002C0220FE7
:10B9D000331F8A95E2F78BB3822B8BBB51CF822F1B
:10B9E00099278077907095958795959587959595EA
:10B9F00087959595879521E030E002C0220F331F8F
:10BA00008A95E2F782B3822B82BB8BCF822F992754
:10BA1000807790709595879595958795959587955D
:10BA20009595879521E030E002C0220F331F8A955B
:10BA3000E2F782B3822B82BB59CF822F992780777E
:10BA400090709595879595958795959587959595FA
:10BA5000879521E030E002C0220F331F8A95E2F77C
:10BA600083B1822B83B999CE822F992780779070EA
:10BA700095958795959587959595879595958795AE
:10BA800021E030E002C0220F331F8A95E2F783B134
:10BA9000822B83B9A4CE822F9927807790709595B9
:10BAA000879595958795959587959595879502C0E6
:10BAB000440F551F8A95E2F788B3842B88BB4ACE82
:10BAC000822F992780779070959587959595879582
:10BAD000959587959595879502C0440F551F8A9532
:10BAE000E2F788B3842B88BBEBCDCF911F910F91E8
:10BAF000FF90EF9008952091E3053327207F307069
:10BB00003595279535952795359527952E5F772778
:10BB10006627829FA001929F500D611D1124DB01B9
:10BB2000CA0126EB77276627829FA001929F500DBE
:10BB3000611D1124BB27A72F962F852F08950F93E2
:10BB40000091070350919606609197062091FB02A1
:10BB50003091FC028091580699278F70907002975F
:10BB600069F083E02C3F380718F02FEF30E00DC06C
:10BB70003695279536952795332707C0369527950F
:10BB80003695279536952795F7CF40910103852F58
:10BB90000E94A52D99278093080327E337E0482FBB
:10BBA0006CE085E895E00E94E32E29E337E04091C0
:10BBB00007036CE089E795E00E94E32E0F9108955A
:10BBC0002F923F924F925F926F927F928F929F92AD
:10BBD000AF92BF92CF92DF92EF92FF920F931F939B
:10BBE000CF93DF93CDB7DEB760970FB6F894DEBF83
:10BBF0000FBECDBFC0903807EC2DFF27EB57FA4F93
:10BC0000508080903707E82DFF27EB57FA4F608070
:10BC10005618E52DFF27EE0FFF1FE652F84FA590AF
:10BC2000B49000913A07E02FFF27E758FA4F908130
:10BC3000E0903907EE2DFF27E758FA4F3080492E64
:10BC40004318E42DFF27EE0FFF1FE652F84F4591F2
:10BC5000549189E1989F900111248091090390915A
:10BC60000A0396958795969587958217930708F00E
:10BC70002FC2281B390B13EA77246624419F200129
:10BC8000519F500C611C1124B301A2015295629581
:10BC9000729540EF762774237627652764236527FE
:10BCA0003B01EE27739EB001629EA001729E500D73
:10BCB000611D7E1F639E500D611D7E1F1124BA0100
:10BCC0003B0160947094EE2DFF27EF56FA4F908061
:10BCD000E02FFF27EF56FA4F4081292D3327872D7C
:10BCE0009927289FF001299FF00D389FF00D11240E
:10BCF000CF015527472E5524449D1001459D300CFA
:10BD0000549D300C11249101929582958F70892752
:10BD10009F708927329522952F7023273F70232704
:10BD2000820F931F929582958F7089279F70892724
:10BD300080932303EC2DFF27EB57FA4FE08180918E
:10BD400008038E1708F052C2E81BBB27AA27AE9E35
:10BD5000C001BE9E900DA11D11245C0125014094DF
:10BD600050944427B79ED001A69EC001B69E900D68
:10BD7000A11DB41FA79E900DA11DB41F1124CD01BC
:10BD8000AA27BB279A8389834427B79CD001A69C06
:10BD9000C001B69C900DA11DB41FA79C900DA11DC4
:10BDA000B41F1124CD01AA27BB279C838B83442772
:10BDB000579ED001469EC001569E900DA11DB41FF6
:10BDC000479E900DA11DB41F1124CD01AA27BB27AA
:10BDD0001C01EE27579CB001469CA001569C500DBB
:10BDE000611D7E1F479C500D611D7E1F1124CB01DC
:10BDF000AA27BB272C015CE0859EC0011124DE2C04
:10BE0000D80EF02EF80EC59EC0011124E80E080FC2
:10BE10008D2C9924F401E80DF91DE75CFC4FA081FD
:10BE2000B181CF2CDD24F601EC0DFD1DE75CFC4F4C
:10BE3000808191819E838D83FF24F701EE0DFF1D8C
:10BE4000E75CFC4F608071801127F801E00FF11F63
:10BE5000E75CFC4FA080B180E981FA818F2F9927A0
:10BE60002B813C81432F552758874F83E32DFF2794
:10BE7000FE87ED87652D7727788B6F8755274427B9
:10BE8000A89F9001B89F300D411D1124DA01C9010E
:10BE9000ED81FE812F8177276627E29FA001F29F27
:10BEA000500D611D1124840F951FA61FB71F6D85AE
:10BEB00055274427669E9001769E300D411D112422
:10BEC000820F931FA41FB51F7F8555274427A79E68
:10BED0009001B79E300D411D1124820F931FA41FA6
:10BEE000B51F892F9A2FAB2FBB279093EA0280931F
:10BEF000E902F401E751FB4FB081F601E751FB4F36
:10BF00007081F701E751FB4FA080F801E751FB4F2B
:10BF10007080E981FA8155274427EB9F9001FB9FB0
:10BF2000300D411D1124DA01C901EB81FC81552737
:10BF30004427E79F9001F79F300D411D1124820F88
:10BF4000931FA41FB51F552744272A9C90013A9C94
:10BF5000300D411D1124820F931FA41FB51F5527BB
:10BF60004427479C9001579C300D411D1124820F9E
:10BF7000931FA41FB51FCD01AA27BB278093EB02F7
:10BF8000A4EA4A2FA6E05A2F840E951ED401BC9035
:10BF9000C40ED51EF6013081E40EF51ED7016C915A
:10BFA000040F151FF801708149815A81112700275C
:10BFB0004B9D70015B9DF00C011D11245701680120
:10BFC000EB81FC8111270027E39F7001F39FF00CA8
:10BFD000011D1124AE0CBF1CC01ED11E9924882443
:10BFE000269E3001369E700C811C1124A60CB71CB5
:10BFF000C81CD91C11270027479E7001579EF00CC2
:10C00000011D1124AE0CBF1CC01ED11EC601AA27E3
:10C01000BB27882E9924409159060FEF10E0041B8E
:10C020001109801691060CF0DFC0182F140FF09143
:10C03000F802F6FF50C08091DE05811708F45DC05C
:10C0400010E0812F0E94746A782F80916208882303
:10C0500009F45DC0782F60915906472F552710913C
:10C060006806212F3327220F331F260F311D421759
:10C07000530708F471C0E0E0F0E040916C0646FF21
:10C0800093C090906906492D552742955295507F4F
:10C090005427407F54272091FA022637B8F4A6E7A8
:10C0A000B0E0A21BB10920916A063327A29F40018C
:10C0B000A39F900CB29F900C11246401D594C79457
:10C0C000D594C794D594C7944C0D5D1DCA019AC0F0
:10C0D00060E070E0F5CD9091F80295FFB2CF00914D
:10C0E000010320E04091770660915B0680915A063B
:10C0F0000E94A52D811708F0A3CF181B812F0E9445
:10C10000746A782F80916208882309F0A3CF509039
:10C1100007033090A905351408F49DCF40916B06B4
:10C12000E42EFF24609159060FEF10E0061B110961
:10C13000E016F1060CF064C0742F760F472F5527D8
:10C1400010916806212F3327220F331F260F311D30
:10C150004217530708F08FCF241B350B8091E3055E
:10C160009927807F9070959587959595879595955A
:10C1700087958E5F77246624289F2001389F500C76
:10C18000611C112436EB11270027439E7001539E3A
:10C19000F00C011D1124BB27A12F902F8F2DFC0126
:10C1A00040916C0646FD6DCF8AE991E0B0900E0398
:10C1B000772466248B9D20019B9D500C611C1124CB
:10C1C000BB27A72D962D852D01E08836900798F086
:10C1D00029E130E0B0910703BB3058F443FF09C0B8
:10C1E000C90180509E4F0EC01FEF21CFAA24BB244F
:10C1F000B5CDC90107C020E831E0281B390BEACFD3
:10C200007FEF2BCFF89470930E03F0931A03E09313
:10C2100019039093180380931703789460960FB6D0
:10C22000F894DEBF0FBECDBFDF91CF911F910F916C
:10C23000FF90EF90DF90CF90BF90AF909F908F9046
:10C240007F906F905F904F903F902F900895CF9286
:10C25000DF92EF92FF920F931F93CF93DF93982F6C
:10C26000F42E722F203809F4A4C08091510684174F
:10C2700008F09FC0062F1127C92FDD272CE030E0E2
:10C28000029FF001039FF00D129FF00D1124EC0F9F
:10C29000FD1FEE0FFF1FE75CFC4F0190F081E02DCA
:10C2A00077FD81C080E8871B55274427E89F9001D0
:10C2B000F89F300D411D1124DA01C901292F3A2FB1
:10C2C0004B2F552780915206F89EA0011124662716
:10C2D000359F7001249F6001349FD00CE11CF61E35
:10C2E000259FD00CE11CF61E1124C701AA27BB27ED
:10C2F000AC0177FD4EC0E81BF90BAF016CE070E0BC
:10C30000069FF001079FF00D169FF00D1124EC0F12
:10C31000FD1FE75AFB4F208180915306289F700133
:10C3200011248F2D992787FD9A9533279927F90195
:10C33000E80FF91FEF3FF105E9F0E0F0EFEFFFEF55
:10C34000281B390B322F2227E417F507E8F4AF0139
:10C35000ACE0B0E00A9FF0010B9FF00D1A9FF00DCA
:10C360001124EC0FFD1FEE0FFF1FE75CFC4F518304
:10C3700040831FC0FE2FEE27EF6F281B390B322F93
:10C380002227E417F50718F34217530708F7A90106
:10C39000DFCFCC24DD24CE1ADF0A8C159D0530F0CA
:10C3A0004FEF5FEFABCF872F80587ECF4E0F5F1FD1
:10C3B000A5CFDF91CF911F910F91FF90EF90DF906C
:10C3C000CF9008952F923F924F925F926F927F92FB
:10C3D0008F929F92AF92BF92CF92DF92EF92FF9295
:10C3E0000F931F93CF93DF93CDB7DEB729970FB687
:10C3F000F894DEBF0FBECDBF6C0150913807E52F1A
:10C40000FF27EB57FA4FF08040913707E42FFF27C3
:10C41000EB57FA4F1081F11AEF2DFF27EE0FFF1F98
:10C42000E652F84FE590F490B0903A07EB2DFF27D5
:10C43000E758FA4F6080A0903907EA2DFF27E758A8
:10C44000FA4F70806718E62DFF27EE0FFF1FE652A8
:10C45000F84F059114919E012F5F3F4FFC014081E1
:10C460006CE089E795E00E94E32E9E012D5F3F4F2F
:10C47000F60141816CE085E895E00E94E32E3E01E3
:10C480000894611C711CF3013181A32EBB24F501BA
:10C49000E758FA4F9080F601508095184C80642D33
:10C4A0007727FB01EB57FA4F8080F6013180831824
:10C4B00055244424099D1001199D300C411C112460
:10C4C000BB27A52D942D832D182F55244424E89C9B
:10C4D0001001F89C300C411C1124BB27A52D942D74
:10C4E000832D982E812E8094582E509490913D0744
:10C4F00080913E07989F9001112499279695982F37
:10C50000882797958795281B390B232F3327022FD0
:10C5100000588091540682FFD4C1199DD001112486
:10C520008B2F9927848349803B803D82682F003878
:10C5300009F48EC070915106781708F089C0A32CB9
:10C54000BB24E42CFF248CE090E0A89EF001A99E7F
:10C55000F00DB89EF00D1124EE0DFF1DEE0FFF1F24
:10C56000E75CFC4F0190F081E02D002314F020E8FF
:10C57000201BBB27AA27E29FC001F29F900DA11D9F
:10C580001124892F9A2FAB2FBB278E839F83A887D7
:10C59000B98780915206689FD00111242E803F8078
:10C5A00022273B9EB0012A9EA0013A9E500D611D9C
:10C5B000721F2B9E500D611D721F1124DB01CA01D9
:10C5C000CD01AA27BB279C0107FDF2C3DF01A21BF7
:10C5D000B30B4CE050E0A49EF001A59EF00DB49E7C
:10C5E000F00D1124EE0DFF1DE75AFB4F20818091C5
:10C5F0005306289F10011124832D992787FD9A95B2
:10C60000422F55279927BA01680F791F6F3F71058F
:10C6100011F008F018C3762F66276F6F481B590B6F
:10C62000942F88276A177B0708F007C3DB018CE08B
:10C6300090E0A89EF001A99EF00DB89EF00D112487
:10C64000EE0DFF1DEE0FFF1FE75CFC4FB183A083D3
:10C65000159D700111248F2D9927F60185832C815A
:10C66000182F003829F0B0915106B81708F4C5C149
:10C67000899C500111248B2D9927F6018683F301A3
:10C680002181182F003809F48BC0F0915106F8175A
:10C6900008F086C09D81A92EBB24E22EFF246CE009
:10C6A00070E0A69EF001A79EF00DB69EF00D11243D
:10C6B000EE0DFF1DEE0FFF1FE75CFC4F60817181E7
:10C6C00007FD9AC380E8801B55274427689F900187
:10C6D000789F300D411D1124DA01C901892F9A2F4D
:10C6E000AB2FBB278E839F83A887B9878091520683
:10C6F000189FD00111242E803F80FF273B9EA00170
:10C700002A9E90013A9E300D411D5F1F2B9E300DD9
:10C71000411D5F1F1124CA01AA27BB2707FD5EC365
:10C72000681B790B4CE050E0A49EF001A59EF00D33
:10C73000B49EF00D1124EE0DFF1DE75AFB4F208132
:10C7400080915306289F10011124832D992787FD7E
:10C750009A9533279927A901480F591F4F3F510533
:10C7600011F008F079C2542F44274F6F281B390B62
:10C77000322F22274617570708F068C2BA01ACE0EB
:10C78000B0E0AA9EF001AB9EF00DBA9EF00D112410
:10C79000EE0DFF1DEE0FFF1FE75CFC4F7183608302
:10C7A000859C700111248F2D9927F6018783F30151
:10C7B00021813C81182F003809F40AC4C090510629
:10C7C000C81608F005C4A32EBB24C22EDD246CE0DD
:10C7D00070E0A69EF001A79EF00DB69EF00D11240C
:10C7E000EC0DFD1DEE0FFF1FE75CFC4F60817181BA
:10C7F00007FDFFC280E8801B55244424689F100178
:10C80000789F300C411C11245527452D342D232DA4
:10C8100080915206189F100111248824339D300105
:10C82000229D2001329D500C611C781C239D500CD0
:10C83000611C781C1124C301AA27BB2707FDC3C2B2
:10C84000681B790B0CE010E0A09EF001A19EF00D9A
:10C85000B09EF00D1124EC0DFD1DE75AFB4F208119
:10C8600080915306289F20011124852D992787FD4B
:10C870009A9533279927A901480F591F4F3F510512
:10C8800011F008F0D7C1542F44274F6F281B390BE4
:10C89000322F22274617570708F0C6C1BA012CE0ED
:10C8A00030E0A29EF001A39EF00DB29EF00D112487
:10C8B000EC0DFD1DEE0FFF1FE75CFC4F71836083E5
:10C8C00087C387FC20C1F6011682178257FCD0C1AE
:10C8D000F6011582199D700111248F2D99278483EB
:10C8E0004981EB81682F003809F472C3B09051067A
:10C8F000B81608F06DC3CE2EDD24E42EFF24ACE084
:10C90000B0E0CA9EF001CB9EF00DDA9EF00D11242E
:10C91000EE0DFF1DEE0FFF1FE75CFC4F0190F08155
:10C92000E02D07FD02C020E8201B55244424E29F8F
:10C930001001F29F300C411C11245527452D342D38
:10C94000232D80915206689F5001112466243B9D3F
:10C9500020012A9D10013A9D300C411C561C2B9D34
:10C96000300C411C561C1124C201AA27BB279C0174
:10C9700007FD45C2DF01A21BB30B8CE090E0C89E0F
:10C98000F001C99EF00DD89EF00D1124EE0DFF1D93
:10C99000E75AFB4F708180915306789FA0011124C4
:10C9A000852F992787FD9A95472F55279927BA01F3
:10C9B000680F791F6F3F710511F008F0E8C1762FFD
:10C9C00066276F6F481B590B942F88276A177B07C0
:10C9D00008F0D7C1DB010CE010E0C09EF001C19E61
:10C9E000F00DD09EF00D1124EE0DFF1DEE0FFF1F78
:10C9F000E75CFC4FB183A083EBC2E22EFF24A42CA2
:10CA0000BB24ACE0B0E0EA9EF001EB9EF00DFA9E94
:10CA1000F00D1124EA0DFB1DEE0FFF1FE75CFC4F2C
:10CA20006081718107FDC1C180E8801B55274427C3
:10CA3000689F9001789F300D411D1124DA01C901D2
:10CA4000892F9A2FAB2FBB278E839F83A887B98707
:10CA500080915206189FD00111242E803F80FF271D
:10CA60003B9EA0012A9E90013A9E300D411D5F1F02
:10CA70002B9E300D411D5F1F1124CA01AA27BB2721
:10CA800007FD88C1681B790B4CE050E0E49EF00183
:10CA9000E59EF00DF49EF00D1124EA0DFB1DE75A02
:10CAA000FB4F208180915306289F10011124832D74
:10CAB000992787FD9A9533279927A901480F591F70
:10CAC0004F3F510511F008F0D0C0542F44274F6F4D
:10CAD000281B390B322F22274617570708F0BFC0F3
:10CAE000BA01ACE0B0E0EA9EF001EB9EF00DFA9ED8
:10CAF000F00D1124EA0DFB1DEE0FFF1FE75CFC4F4C
:10CB000071836083B5CDF6011482158257FC82C112
:10CB1000F6011782899C20011124852D992786838F
:10CB2000EB81682F003809F453C230905106381653
:10CB300008F04EC2EE2EFF244CE050E0E49EF001DF
:10CB4000E59EF00DF49EF00D1124EA0DFB1DEE0F95
:10CB5000FF1FE75CFC4F0190F081E02D07FD02C054
:10CB600020E8201B55244424E29F1001F29F300C42
:10CB7000411C11245527452D342D232D809152061B
:10CB8000689F400111246624399D2001289D1001D1
:10CB9000389D300C411C561C299D300C411C561CE4
:10CBA0001124C201AA27BB279C0107FDDEC1DF01BA
:10CBB000A21BB30B0CE010E0E09EF001E19EF00D33
:10CBC000F09EF00D1124EA0DFB1DE75AFB4F50803B
:10CBD00080915306589E600111248D2D992787FD61
:10CBE0009A95452D55279927BA01680F791F6F3FF0
:10CBF000710511F008F0A3C1762F66276F6F481BEF
:10CC0000590B942F88276A177B0708F09BC1DB011B
:10CC10002CE030E0E29EF001E39EF00DF29EF00D7C
:10CC20001124EA0DFB1DE2CE6217730708F037CE20
:10CC3000B90135CE4FEF5FEF29CEA817B90708F03D
:10CC4000F6CCDC01F4CC6FEF7FEFE8CC6217730712
:10CC500008F095CDB90193CD4FEF5FEF87CD621707
:10CC6000730708F03ECFB9013CCF4FEF5FEF30CFF5
:10CC70001482159D500111248B2D9927858349819C
:10CC8000182F003809F4A4C130915106381708F064
:10CC90009FC1E42EFF24ACE0B0E06A9FF0016B9FDF
:10CCA000F00D7A9FF00D1124EE0DFF1DEE0FFF1F0A
:10CCB000E75CFC4F0190F081E02D07FD02C020E809
:10CCC000201B77246624E29F2001F29F500C611CF8
:10CCD00011245527472D362D252D80915206189F5A
:10CCE000A00111246624359F2001249F1001349F48
:10CCF000300C411C561C259F300C411C561C112425
:10CD0000C201AA27BB279C0107FD39C1DF01A21B75
:10CD1000B30B0CE010E0609FF001619FF00D709F7D
:10CD2000F00D1124EE0DFF1DE75AFB4F708080912E
:10CD30005306789E40011124892D992787FD9A95E5
:10CD4000472D55279927FA01E80FF91FEF3FF10505
:10CD500011F008F003C1FE2FEE27EF6F481B590BAF
:10CD6000942F8827EA17FB0708F0F2C0DF012CE0B8
:10CD700030E0629FF001639FF00D729FF00D11246F
:10CD800033CEA817B90708F026CEDC0124CE6FEF0A
:10CD90007FEF18CE22273327261B370B82179307E6
:10CDA00008F4CAC06FEF7FEF6FCE802F80583ECE61
:10CDB000662777276E1B7F0B8617970708F4B5C089
:10CDC000AFEFBFEF06CC88249924861A970A8815FE
:10CDD000990508F4A7C06FEF7FEF34CD22273327E2
:10CDE000261B370B8217930708F4A3C06FEF7FEF62
:10CDF00099CC802F805800CD802F805865CC662735
:10CE000077276E1B7F0B8617970708F4AAC0AFEF32
:10CE1000BFEFB3CD1682859CA0011124852F9927E1
:10CE20008783182F003809F4D3C0D0905106D81644
:10CE300008F0CEC0ACE0B0E06A9FF0016B9FF00D4F
:10CE40007A9FF00D1124EA0DFB1DEE0FFF1FE75C2A
:10CE5000FC4F0190F081E02D07FD02C020E8201B6F
:10CE6000BB27AA27E29FC001F29F900DA11D1124AC
:10CE7000292F3A2F4B2F552780915206189F70016A
:10CE8000112466243F9D20012E9D10013E9D300CF3
:10CE9000411C561C2F9D300C411C561C1124C201F4
:10CEA000AA27BB279C0107FD85C0DF01A21BB30B8E
:10CEB0000CE010E0609FF001619FF00D709FF00D9D
:10CEC0001124EA0DFB1DE75AFB4F90808091530619
:10CED000989E30011124872D992787FD9A95492D19
:10CEE00055279927FA01E80FF91FEF3FF10511F0D7
:10CEF00008F04FC0FE2FEE27EF6F481B590B942F01
:10CF00008827EA17FB0708F047C0DF012CE030E074
:10CF1000629FF001639FF00D729FF00D1124EA0DE6
:10CF2000FB1D64CD680F791F8DCCDF01A20FB31FED
:10CF300050CB680F791FF6CB680F791FA5CD6FEF27
:10CF40007FEF5DCEA817B90708F062CEDC0160CE96
:10CF5000A817B90708F00BCFDC0109CFEFEFFFEFFF
:10CF6000FDCEDF01A20FB31F08CD662777276E1B0A
:10CF70007F0B86179707B0F0AFEFBFEF1BCE882768
:10CF800099278E1B9F0B2817390780F0AFEFBFEF53
:10CF9000C0CEEFEFFFEFB1CFA817B90708F0B6CFBB
:10CFA000DC01B4CFDF01A20FB31F04CEDF01A20F5B
:10CFB000B31FAFCE222433242E1A3F0A82159305C5
:10CFC00018F0AFEFBFEF74CFDF01A20FB31F70CF28
:10CFD00029960FB6F894DEBF0FBECDBFDF91CF917B
:10CFE0001F910F91FF90EF90DF90CF90BF90AF9087
:10CFF0009F908F907F906F905F904F903F902F9079
:10D000000895869F90011124832F992787FD9A9573
:10D01000982F80914D06981718F481E090E00895BC
:10D0200080E090E00895CF92DF92EF92FF920F930D
:10D030001F93CF93DF93DC018B0140E050E0FC01B4
:10D040002FE08191480F511D215027FFFACFEA01AF
:10D05000D295C295CF70CD27DF70CD27F801C08360
:10D0600020E030E060E0FD01A901819199278C1B4F
:10D070009D0B2227999F7001889F6001989FD00C7B
:10D08000E11CF21E899FD00CE11CF21E11249A01B2
:10D090002C0D3D1D2417350720F06F5F603120F304
:10D0A00002C04FEF5FEF529542954F7045275F707A
:10D0B0004527E8015A834983DF91CF911F910F9152
:10D0C000FF90EF90DF90CF900895689FC0011124EA
:10D0D0008F3F910518F080E090E0089580959927A2
:10D0E0000895EF92FF920F931F93CF9340913E01CB
:10D0F000E42FFF27E05CFE4F80910703808370964A
:10D100002091FB023091FC028091580699278F7084
:10D110009070029709F463C103E02C3F3007B8F028
:10D120008FEF90E08083E42FFF27E05CFE4FE090DC
:10D13000E302E0A2E42FEF5FE031D8F4E0933E0198
:10D14000F090F802F3FC1BC010923F016CC13695C1
:10D15000279536952795822F99278083E42FFF27DF
:10D16000E05CFE4FE090E302E0A2E42FEF5FE031ED
:10D1700028F310923E01F090F802F3FEE5CF909173
:10D18000FD0200914C069017F8F2C0913F01CF5F6D
:10D19000CA3108F42BC120E030E0E0E4F1E09FE088
:10D1A0001191210F311D915097FFFACFB90172955E
:10D1B00062956F7067277F7067276093460780E0EE
:10D1C00090E030E0E0E4F1E0AC0181919927861B2A
:10D1D000970B2227999F8001889F7001989FF00CE0
:10D1E000011D121F899FF00C011D121F1124D8016F
:10D1F000C701840F951F8417950708F400C13F5F8E
:10D20000303110F3529542954F7045275F70452796
:10D21000E6E4F7E05283418320E030E0E0E5F1E02E
:10D220009FE04191240F311D915097FFFACFB90132
:10D23000729562956F7067277F70672760934907C3
:10D2400080E090E030E0E0E5F1E0AC0181919927E9
:10D25000861B970B2227999F8001889F7001989FBA
:10D26000F00C011D121F899FF00C011D121F1124CB
:10D27000D801C701840F951F8417950708F4BCC017
:10D280003F5F303110F3529542954F7045275F70E4
:10D290004527E9E4F7E05283418320E030E0E0E60F
:10D2A000F1E09FE05191250F311D915097FFFACF8A
:10D2B000B901729562956F7067277F7067276093D9
:10D2C0004C0780E090E030E0E0E6F1E0AC018191D5
:10D2D0009927861B970B2227999F8001889F7001B1
:10D2E000989FF00C011D121F899FF00C011D121F49
:10D2F0001124D801C701840F951F8417950708F4DE
:10D3000078C03F5F303110F3529542954F704527FA
:10D310005F704527ECE4F7E0528341832091460794
:10D3200030914907239FD00111248B2F992787FD26
:10D330009A9570914D06871708F04DC020933B07D2
:10D3400030933C0720914C0720933D07909147076D
:10D3500080914E06899FC00111248F3F910508F4EA
:10D3600058C080E090E0582F90914A0780914F0676
:10D37000899FC00111248F3F910508F447C080E0C8
:10D3800090E0482F90914D0780915006899FC001F1
:10D3900011248F3F910508F435C020E030E0509310
:10D3A00043074093440720934507549F700111247D
:10D3B00077276627E29EA001F29E500D611D112481
:10D3C000CB01AA27BB2780933E07882321F0309109
:10D3D000540631FF21C0BAE0B0933F0124C0369516
:10D3E00027953695279536952795B5CEC0933F015D
:10D3F0001AC04FEF5FEF88CF4FEF5FEF44CF4FEF93
:10D400005FEF00CF8095282F3327C9CF80959927CC
:10D41000B8CF80959927A7CFC0933F018BE397E0C2
:10D420000E94E261D8CFCF911F910F91FF90EF90B2
:10D43000089520E0E9E5F4E0DF01A052B1408D91CC
:10D440009D9180589F4F892F992781932F5F203975
:10D45000B0F3089520E0E9E5F4E0DF01A052B14027
:10D4600081919927982F88278F678D939D932F5FA0
:10D470002039B0F3089508950F936091010320912E
:10D48000090330910A033695279536952795009123
:10D49000F60599E1099FA00111248091F00587FD0F
:10D4A00003C01092F2021EC07091F80275FDF9CF10
:10D4B000A091F205A617A8F34217530790F7241B73
:10D4C000350BF901E070EF2B59F00FEF20E140E050
:10D4D0006091F505842F0E94A52D8093F20202C071
:10D4E000022FF4CF0F910895CF93DF93382F8091BF
:10D4F000F00584FF04C02091F70227FD04C0832FAC
:10D50000432F552758C04091090350910A03909129
:10D510004F078AE0989FC00111244817590720F54A
:10D52000841B950BA0911106772766278A9FA0017F
:10D530009A9F500D611D1124FB01EA018D2F9E2F32
:10D54000AF2FBB27BC018091130699278617970739
:10D5500078F1432F55279A01260F371FE32FFF2716
:10D56000EF2B41F18FEF27C0481B590B609111063B
:10D57000FF27EE27469FE001569FD00DE11D1124A5
:10D580008D2F9E2FAF2FBB27BC01809114069927AA
:10D590008617970758F0432F55279A01261B370BFC
:10D5A000832F9927892B31F080E005C0BC01F3CF90
:10D5B000BC01CFCF822F282F3327C901841B950BA5
:10D5C0009093630780936207C901DF91CF9108951B
:10D5D000282F8091F005992783FF12C082FF10C089
:10D5E0008091500782FD12C090915207291778F45C
:10D5F000921B909351078D7F81608093500708950F
:10D600002093660720935207109251070895291B13
:10D61000209351078360F1CFCF92DF92EF92FF9278
:10D620000F931F93CF93DF938091F70280FF04C085
:10D63000C090F702C1FE71C0F8940091F7020F7715
:10D640000093F70278941092560710925507809134
:10D65000010699279695982F8827979587959093F7
:10D66000540780935307109258071092570710924F
:10D670005A071092590710925C0710925B0710929C
:10D680005E0710925D071092600710925F079091FD
:10D6900005068AE0989FC0011124809361071092CB
:10D6A000630710926207E090FA05E0927201909190
:10D6B000F90590937301D090F505D90ED0924F07DC
:10D6C000D09274010091FD022091F8054091F70578
:10D6D0006DEC80E00E94A52D9091F105981708F05F
:10D6E00050C190936407209164078091F0059927B9
:10D6F00083FF40C182FF3EC18091500782FD36C248
:10D7000090915207291708F0EEC1921B9093510790
:10D710008D7F81608093500729C210910103F090A2
:10D72000F205F11608F430C12091F70227FD07C079
:10D73000F8943091F70230683093F7027894C090F3
:10D740000903D0900A030091FD022091F605409153
:10D75000F5056091F4058091F3050E94A52D282F11
:10D7600090917201992309F44AC1915090937201EA
:10D7700080917301820F80934F075AE0859F90013B
:10D7800011242C193D094091F00546FF05C01216E1
:10D79000130614F4220F331F3093560720935507B6
:10D7A00040915507509156079A0157FDAAC18091A3
:10D7B00003069927281739070CF42AC160917001D4
:10D7C000709171016C197D09709358076093570728
:10D7D0009A0157FDA7C1809102069927281739079A
:10D7E0000CF02EC17091FC054050504811270027C5
:10D7F000479F7001579FF00C011D1124BB27A12FDB
:10D80000902F8F2DFC01472F55275695542F4427D5
:10D8100057954795E41BF50BF0935C07E0935B0786
:10D82000C0915307D09154071091FD05C050D048C6
:10D8300077276627C19FA001D19F500D611D11243C
:10D84000BB27A72F962F852FBC01E12EFF24F6942E
:10D85000FE2CEE24F794E7946E197F0970935E070F
:10D8600060935D07A0915707B0915807F090FE05AF
:10D87000A050B04833272227AF9D8001BF9D100DD7
:10D88000211D1124BB27A32F922F812F8C018F2DB7
:10D8900099279695982F882797958795081B190B98
:10D8A0001093600700935F077F01E60EF71EE00EFE
:10D8B000F11EF594E794F594E794F594E794F594C4
:10D8C000E794F0925A07E0925907F091F6026F2F11
:10D8D00077276B557A4F9B012F593F4F9091F50257
:10D8E000E92FFF27EB55FA4FAF014F595F4F0091DA
:10D8F000FD02E9012881EA014881EB016885808504
:10D900000E94A52D9701280F311DE0915207EE23AB
:10D9100041F480916107882309F4F8C08150809315
:10D9200061078091F105992740E050E0BC01C901F1
:10D930000E94F52F80936407982FB091F0052B2F4C
:10D94000332723FFD7C022FFD5C08091500782FD27
:10D950000CC020915207921708F0FCC0291B20939D
:10D9600051078D7F816080935007D0927101C092E2
:10D970007001FCC020936607209352071092510754
:10D98000F5C080936407AFCEC090F702C7FEEEC02B
:10D99000F8943091F7023F773093F7027894109221
:10D9A0005607109255071092540710925307109281
:10D9B00058071092570710925A0710925907109261
:10D9C0005C0710925B0710925E0710925D07109241
:10D9D000600710925F07909105068AE0989FC0014A
:10D9E0001124809361078091F005992783FFBEC0C1
:10D9F00082FDBCC01092660710925207BFCF809183
:10DA00007301882309F4B6CE815080937301B2CE9E
:10DA1000209162073091630737FD89C08091150618
:10DA20009927281739070CF4A0CF8091520799271E
:10DA3000141615060CF08AC09C012F5F3F4F71CF62
:10DA400090916407992319F455230CF4CBCE70916F
:10DA5000F105791709F475C0A0915307B0915407E7
:10DA6000ED01EE27D7FDE095FE2FCA01AA2797FD0D
:10DA7000A095BA2FC80FD91FEA1FFB1F8D2F9E2F0D
:10DA8000AF2FBB27A7FDBA95803891050CF453C082
:10DA90008FEF9FE79093540780935307B09101064F
:10DAA000CB2FDD27D695DC2FCC27D795C795809136
:10DAB000000699279695982F882797958795909592
:10DAC00081959F4FAC01BE018091530790915407FF
:10DAD0000E94F52F90935407809353074091550768
:10DAE000509156077FCE291B209351078360809366
:10DAF00050073CC0909366079093520710925107CD
:10DB000034CF22273327241B350B51CE90910506A5
:10DB10008AE0989FC00111248093610751E05093DF
:10DB20005207FFCE22273327241B350B54CE3095C6
:10DB300021953F4F73CF80589F4F9CF480E090E831
:10DB4000A9CF141615060CF44DCE86CF9C0121509A
:10DB50003040E7CE921B909351078360809350072B
:10DB600004CFD0935407C093530798CFDF91CF9140
:10DB70001F910F91FF90EF90DF90CF9008958091CB
:10DB8000F005992783FF3DC082FD3BC0E5E6F7E045
:10DB900040E04093650740936607F8948091D3076F
:10DBA0009091D40720918800309189003093D40758
:10DBB0002093D3072817390748F4A091D507B091CF
:10DBC000D6071196B093D607A093D5077894BB27B4
:10DBD000AA27249FC001349F900DA11D1124892FD5
:10DBE0009A2FAB2FBB279483838336832583209181
:10DBF00050072A7F20935007109252071092510726
:10DC0000089545E0409350073091F105365F309319
:10DC1000520730935107089599278130910551F0AB
:10DC200082309105D4F08230910551F0039771F064
:10DC3000E0E018C0E091EF05E695E695E37012C0CC
:10DC4000E091EF05E295EF70E3700CC0E091EF0515
:10DC5000E295E695E695E37005C0892B49F7E091DA
:10DC6000EF05E370FF27E354F74E84919927089559
:10DC7000909151079923C9F18091F00581FF05C06A
:10DC80002091FA02253408F43FC0492F41504093B7
:10DC9000510720915007277F21FD37C03091750132
:10DCA000315080915207815080935207832F8370A7
:10DCB000992781309105B9F1823091050CF43FC06C
:10DCC00082309105B1F1039709F43FC0E0E0FF27EE
:10DCD000E354F74E5491526055BB30937501442381
:10DCE00089F42A7F209350070895409150074A7F76
:10DCF000409350073091F00530FF06C065B3607E59
:10DD000065BB0895209350070895309175013F5FDA
:10DD1000809152078F5F80935207832F83709927DA
:10DD20008130910549F6E091EF05E695E695E370BF
:10DD3000CECFE091EF05E295EF70E370C8CF892B6D
:10DD400029F6E091EF05E370C2CFE091EF05E2958F
:10DD5000E695E695E370BBCFAF92BF92CF92DF928C
:10DD6000FF920F931F93CF93DF93F090F005F3FE94
:10DD7000B2C005E617E0F8948091D3079091D407DC
:10DD800040918800509189005093D4074093D30765
:10DD90004817590708F4D5C07894E0916A07F091C4
:10DDA0006B077091660760916507C5E6D7E0209123
:10DDB0006807309169074E175F0730F4862F99275F
:10DDC000D82ECC242C193D097617A9F0671708F036
:10DDD000F1C0972F961BDD24CC24499F5001599FF9
:10DDE000B00CC11C1124BB27AD2D9C2D8B2D280FF1
:10DDF000391F709365073C832B835E834D83B090FE
:10DE00006707BB2041F0EA01CE1BDF0B2C0F3D1F43
:10DE1000F80134832383BB27AA27479FC001579F5C
:10DE2000900DA11D1124492F5A2F6B2F7727241BEA
:10DE3000350B832F9927853508F00BC120E030E0A2
:10DE4000E8012A83722FF89460911006362F3F70F4
:10DE5000262F207F2727432F55274230510509F0D1
:10DE60004FC027FD55C13327207730703595279552
:10DE700035952795359527953595279581E090E03F
:10DE800002C0880F991F2A95E2F7B82FB09585B385
:10DE90008B2385BBF5FE1DC078940000F894962F67
:10DEA000905F60E86727292F207F26279F70492FE2
:10DEB00055274230510509F4DDC0433051050CF0BF
:10DEC000A6C04115510509F409C14130510509F4B5
:10DED00035C1789431C20091FD029091E705091790
:10DEE000D0F170E0F89460911006362F3F70262F25
:10DEF000207F2727432F55274230510509F4B1CF02
:10DF000043305105ACF54115510509F063C027FDBB
:10DF100048C133272077307035952795359527955B
:10DF2000359527953595279581E090E002C0880FBB
:10DF3000991F2A95E2F7482F40958BB384238BBB1A
:10DF4000A9CFA091D507B091D6071196B093D60767
:10DF5000A093D50721CF1091FD02212F3327892FC0
:10DF600099270397281739070CF0E6C170E8BACF54
:10DF70004630510509F498C04730510509F08ACF61
:10DF800027FD6BC133272077307035952795359560
:10DF90002795359527953595279581E090E002C026
:10DFA000880F991F2A95E2F7C82EC09483B18C215F
:10DFB00083B970CF671BDD24CC24469F5001569F48
:10DFC000B00CC11C1124BB27AD2D9C2D8B2D281B03
:10DFD000390B0FCF4130510509F05CCF27FD6BC1E4
:10DFE000822F99278077907095958795959587953D
:10DFF000959587959595879502C0440F551F8A95ED
:10E00000E2F7542F509588B3852388BB43CF463021
:10E01000510509F4ACC04730510509F05ACF27FD2E
:10E020005FC1332720773070359527953595279533
:10E03000359527953595279581E090E002C0880FAA
:10E04000991F2A95E2F7E82FE09583B18E2383B9D3
:10E0500040CF8C3A60F4A0913C08B0913D081196F5
:10E06000B0933D08A0933C08F8015483438320E813
:10E0700030E0E6CE27FDACC03327207730703595F1
:10E08000279535952795359527953595279581E0E1
:10E0900090E002C0880F991F2A95E2F7A82EA0945D
:10E0A00085B38A2185BB15CF27FDA9C033272077EB
:10E0B0003070359527953595279535952795359564
:10E0C000279581E090E002C0880F991F2A95E2F71A
:10E0D000F82FF09582B38F2382BBDCCE27FDA6C03C
:10E0E00033272077307035952795359527953595C9
:10E0F00027953595279581E090E002C0880F991FFC
:10E100002A95E2F7F82EF0948BB38F218BBBE1CEEA
:10E11000822F99278077907095958795959587950B
:10E12000959587959595879521E030E002C0220F5F
:10E13000331F8A95E2F785B3822BABCE27FDE7C06C
:10E14000822F9927807790709595879595958795DB
:10E15000959587959595879502C0440F551F8A958B
:10E16000E2F7742F709588B3872388BBB2CE27FD62
:10E170008BC03327207730703595279535952795B7
:10E18000359527953595279581E090E002C0880F59
:10E19000991F2A95E2F7B82EB09482B38B2182BBE7
:10E1A00098CE822F99278077907095958795959531
:10E1B0008795959587959595879521E030E002C0E4
:10E1C000220F331F8A95E2F78BB3822B8BBB62CE73
:10E1D000822F99278077907095958795959587954B
:10E1E000959587959595879521E030E002C0220F9F
:10E1F000331F8A95E2F785B3822B85BB6ACE822FC7
:10E2000099278077907095958795959587959595A1
:10E2100087959595879521E030E002C0220F331F46
:10E220008A95E2F782B3822B82BB34CE822F992764
:10E230008077907095958795959587959595879515
:10E240009595879521E030E002C0220F331F8A9513
:10E25000E2F78BB3822B8BBB3CCE822F9927807742
:10E2600090709595879595958795959587959595B2
:10E27000879521E030E002C0220F331F8A95E2F734
:10E2800083B1822B83B906CE822F99278077907035
:10E290009595879595958795959587959595879566
:10E2A00021E030E002C0220F331F8A95E2F782B3EB
:10E2B000822B82BB0ECE822F992780779070959506
:10E2C000879595958795959587959595879502C09E
:10E2D000440F551F8A95E2F788B3842B88BBDACDAB
:10E2E000822F99278077907095958795959587953A
:10E2F000959587959595879521E030E002C0220F8E
:10E30000331F8A95E2F783B1822B83B9E2CD822F46
:10E310009927807790709595879595958795959590
:10E3200087959595879502C0440F551F8A95E2F70A
:10E3300088B3842B88BBCDCDDF91CF911F910F91F6
:10E34000FF90DF90CF90BF90AF9008958B9A9398F5
:10E35000E3B34E2F55274F7050708B98B0916400E7
:10E36000B160B0936400A0916500AE7FA09365009A
:10E3700042955295507F5427407F542783B3992765
:10E380008F709070482B592B909164009E7F9093D2
:10E390006400709164007260709364003091650055
:10E3A0003D7F3093650042955295507F5427407FC2
:10E3B000542763B3262F33272F7030708091640069
:10E3C0008D7F80936400CA01822B932B08958B9AD2
:10E3D0009398E3B32E2F33272F7030708B98B09122
:10E3E0006400B160B0936400A0916500AE7FA0931B
:10E3F000650022953295307F3227207F322783B304
:10E4000099278F709070282B392B909164009E7FF4
:10E4100090936400709164007260709364005091F6
:10E4200065005D7F5093650022953295307F3227DD
:10E43000207F322783B399278F709070282B392B38
:10E44000409164004D7F409364004091760150916B
:10E4500077016091780170917901462357234095A7
:10E460005095422B532B7093770160937601309334
:10E47000790120937801CA019F708F5F9F4091F0CE
:10E4800020E061E070E0CA0186279727FC01E17077
:10E49000F07080FD0AC0569547952F5F2C3098F399
:10E4A000CF01089580E090E00895E22FFF27E85F14
:10E4B000FE4F80819927089554B3507F54BB45B3D4
:10E4C0004F6045BB8B98309164003E7F3093640071
:10E4D000209164002D7F209364008FEF9FEF909335
:10E4E0007901809378019093770180937601089564
:10E4F00082958F70E82FFF27E753F74E8491992775
:10E500000895E82FFF27EF70F070E753F74E8491DE
:10E510009927089590E002C09C5E86518631E0F70D
:10E52000882361F0823068F0E82FFF27E459F84F24
:10E53000E90FF11D31978081992708958DE090E0D2
:10E5400008958AE090E00895282F8695869586950F
:10E55000A82FBB27A354B84FE22FFF27E770F07016
:10E56000EF53F74E94918C918923992787FD9095CD
:10E57000089580915606982F92959F709A95F1F77D
:10E58000949A8F708A95F1F794980895CF92DF92BC
:10E59000EF92FF920F931F93CF93DF939498F89489
:10E5A000109165001E7F12601093650078944BB344
:10E5B0004F70082F007F042B0BBBD09056063D2DCB
:10E5C00032953F70E32EEA94F1F7949A2D2D2F7037
:10E5D000C22ECA94F1F79498992782959295907FCC
:10E5E0009827807F9827482B4BBB3A95F1F7949A50
:10E5F0002A95F1F794980CEC17E0F8948091D307E2
:10E600009091D40740918800509189005093D4078D
:10E610004093D3074817590748F4A091D507B09104
:10E62000D6071196B093D607A093D5077894E091BA
:10E63000D107F091D2077091CD076091CC07CCEC57
:10E64000D7E02091CF073091D0074E175F0730F405
:10E65000E62EFF24DE2CCC242C193D097617A9F0D8
:10E66000671708F042C0972F961BFF24EE24499F9E
:10E670006001599FD00CE11C1124BB27AF2D9E2DAA
:10E680008D2D280F391F7093CC073C832B835E831D
:10E690004D83F090CE07FF2041F0EA01CE1BDF0B47
:10E6A0002C0F3D1FF80134832383BB27AA27479FE4
:10E6B000C001579F900DA11D1124492F5A2F6B2F78
:10E6C0007727241B350B832F99278535F0F480E0BD
:10E6D00090E0E8018A83892B49F5F8945091650010
:10E6E0005D7F50936500789421C0671BFF24EE2462
:10E6F000469F6001569FD00CE11C1124BB27AF2D13
:10E700009E2D8D2D281B390BBECF8C3A60F4A09125
:10E710003C08B0913D081196B0933D08A0933C0889
:10E72000F8015483438380E890E0D3CF0E94F22025
:10E73000DF91CF911F910F91FF90EF90DF90CF90DD
:10E740000895AF92BF92CF92DF92EF92FF921F9304
:10E75000CF93DF93F89448E04ABB949810916500FA
:10E760001D7F116010936500789430915606932FA9
:10E7700092959F70A92EAA94F1F7949A3F70232F37
:10E780002A95F1F719B394989A95F1F7949A3A95D6
:10E79000F1F79498BCECEB2EB7E0FB2EF894809147
:10E7A000D3079091D40740918800509189005093ED
:10E7B000D4074093D3074817590748F4A091D507C9
:10E7C000B091D6071196B093D607A093D507789449
:10E7D000E091D107F091D2077091CD076091CC07FD
:10E7E000CCECD7E02091CF073091D0074E175F07D0
:10E7F00030F4A62EBB249A2D8827281B390B7617B8
:10E80000A9F0671708F040C0B72FB61BDD24CC2451
:10E810004B9F50015B9FB00CC11C1124BB27AD2D39
:10E820009C2D8B2D280F391F7093CC073C832B8395
:10E830005E834D83B090CE07BB2041F0EA01CE1B32
:10E84000DF0B2C0F3D1FF70134832383BB27AA273F
:10E85000479FC001579F900DA11D1124492F5A2F8A
:10E860006B2F7727241B350B832F9927853508F5C8
:10E8700080E090E0E7018A83892BB1F0F8948091E1
:10E8800065008E7F826026C0671BDD24CC24469FF6
:10E890005001569FB00CC11C1124BB27AD2D9C2DDF
:10E8A0008B2D281B390BC0CFF894809165008C7F8D
:10E8B00011C08C3A60F4A0913C08B0913D081196CB
:10E8C000B0933D08A0933C08F7015483438380E84C
:10E8D00090E0D0CF8093650058EF5ABB78941078C1
:10E8E000812F9927DF91CF911F91FF90EF90DF90BB
:10E8F000CF90BF90AF900895982F862F8F5F80356F
:10E90000E8F01092C907262F3327D901A459B84F30
:10E91000FD018181891789F09183669566956695D9
:10E92000A62FBB27A354B84F277030702F53374EF4
:10E93000F90194912C91292B2C9308958093C90768
:10E94000E2CFCF93DF93EC01862F60E0982F8035E4
:10E95000B8F528812223A1F1A0E0B0E026C01092F2
:10E96000C907292F3327F901E459F84F7181751729
:10E9700089F05183969596959695A92FBB27A35418
:10E98000B84F277030702F53374EF90194913C9156
:10E99000392B3C93942F403598F4A62FBB27FE01CA
:10E9A000EA0FFB1F4081442359F0AC0FBD1F6F5F7E
:10E9B0005C91492F4F5F403590F64093C907D1CF06
:10E9C000DF91CF910895AC0197FD26C0862F8F5F10
:10E9D0008035F8F48093C907262F3327C90184595D
:10E9E000984FFC01B181BB3291F09BE29183669517
:10E9F00066956695A62FBB27A354B84F2770307035
:10EA00002F53374EF90164913C91362B3C93CA0148
:10EA100008951092C907E0CF862F8F5F803508F5E3
:10EA20008093C907262F3327F901E459F84F8181D4
:10EA30008D3291F07DE27183669566956695A62F7D
:10EA4000BB27A354B84F277030702F53374EF901AE
:10EA500094912C91292B2C9388279927841B950B13
:10EA600008951092C907DECFEF92FF920F931F9384
:10EA7000CF93DF93EC01162F92E0F92EE0E4FCE94E
:10EA800024E040E350E00EE06EE070E0CE17DF07D8
:10EA900020F0CE1BDF0B420F511DF695E795269512
:10EAA000CB0183709070892B49F5E12E1F5F2E2DCD
:10EAB0003327D901A459B84FFD015181541789F06A
:10EAC0004183E694E694E694AE2DBB27A354B84F59
:10EAD000277030702F53374EF9012491EC90E22AC1
:10EAE000EC92EF2DFF27EE0FFF1FEC5EFE4FFA9426
:10EAF0000190F081E02D28E040E350E001506150AA
:10EB0000704007FFC3CF9C2F905D812F8F5F8035B2
:10EB1000E0F01092C907212F3327F901E459F84F8B
:10EB2000F180F916A9F09183169516951695C12FC7
:10EB3000DD27C354D84F277030702F53374EF9015B
:10EB400014910881012B088303C08093C907E3CF88
:10EB5000DF91CF911F910F91FF90EF9008951F9338
:10EB6000CF93DF93EC01742F77FD55C0E72FFF277C
:10EB7000EE0FFF1FEC5EFE4F71500190F081E02D13
:10EB800040E350E0CE17DF0720F0CE1BDF0B48E359
:10EB900050E0CF0196958795C817D90720F0C81B7C
:10EBA000D90B4C5F5F4FCF019695879596958795CA
:10EBB000C817D90720F0C81BD90B4E5F5F4FF695D9
:10EBC000E795F695E795F695E795CE17DF0720F0E0
:10EBD000CE1BDF0B4F5F5F4F162F6F5F212F332749
:10EBE000D901A459B84FFD018181841709F4BCCF24
:10EBF0004183169516951695A12FBB27A354B84FA0
:10EC0000277030702F53374EF90124911C91122B2D
:10EC10001C9377FFABCFCA30D10508F1862F8F5FE9
:10EC2000803578F11092C907262F3327F901E4596E
:10EC3000F84F41814D3A59F15DEA518366956695E9
:10EC40006695C62FDD27C354D84F277030702F53D9
:10EC5000374EF90164913881362B388318C09C2FC8
:10EC6000905D862F8F5F803578F01092C907262F30
:10EC70003327F901E459F84F7181791741F09183F5
:10EC8000DDCF8093C907D0CF8093C907F0CFDF9144
:10EC9000CF911F910895482F9498F8945091650052
:10ECA0005C7F5093650078943BB33F70407F342B7A
:10ECB0003BBB90915606292F22952F702A95F1F78C
:10ECC000949A892F8F708A95F1F794980895CF922E
:10ECD000DF92EF92FF920F931F93CF93DF9394985D
:10ECE000F894109165001C7F1093650078944BB3E5
:10ECF0004F70082F007F042B0BBBD09056063D2D84
:10ED000032953F70E32EEA94F1F7949A2D2D2F70EF
:10ED1000C22ECA94F1F79498992782959295907F84
:10ED20009827807F9827482B4BBB3A95F1F7949A08
:10ED30002A95F1F794980CEC17E0F8948091D3079A
:10ED40009091D40740918800509189005093D40746
:10ED50004093D3074817590748F4A091D507B091BD
:10ED6000D6071196B093D607A093D5077894E09173
:10ED7000D107F091D2077091CD076091CC07CCEC10
:10ED8000D7E02091CF073091D0074E175F0730F4BE
:10ED9000E62EFF24DE2CCC242C193D097617A9F091
:10EDA000671708F042C0972F961BFF24EE24499F57
:10EDB0006001599FD00CE11C1124BB27AF2D9E2D63
:10EDC0008D2D280F391F7093CC073C832B835E83D6
:10EDD0004D83F090CE07FF2041F0EA01CE1BDF0B00
:10EDE0002C0F3D1FF80134832383BB27AA27479F9D
:10EDF000C001579F900DA11D1124492F5A2F6B2F31
:10EE00007727241B350B832F99278535F0F480E075
:10EE100090E0E8018A83892B49F1F89450916500CC
:10EE2000526050936500789421C0671BFF24EE2444
:10EE3000469F6001569FD00CE11C1124BB27AF2DCB
:10EE40009E2D8D2D281B390BBECF8C3A60F4A091DE
:10EE50003C08B0913D081196B0933D08A0933C0842
:10EE6000F8015483438380E890E0D3CF0E94F220DE
:10EE7000DF91CF911F910F91FF90EF90DF90CF9096
:10EE80000895CF92DF92EF92FF920F931F93CF934B
:10EE9000DF939498F894109165001C7F109365009F
:10EEA00078940BB30F70402F0BBBD09056063D2DBE
:10EEB00032953F70932F9A95F1F7949A2D2D2F70DC
:10EEC000C22ECA94F1F7949881E090E082959295D1
:10EED000907F9827807F9827482B4BBB3A95F1F776
:10EEE000949A2A95F1F794980CEC17E0F894809195
:10EEF000D3079091D4074091880050918900509396
:10EF0000D4074093D3074817590748F4A091D50771
:10EF1000B091D6071196B093D607A093D5077894F1
:10EF2000E091D107F091D2077091CD076091CC07A5
:10EF3000CCECD7E02091CF073091D0074E175F0778
:10EF400030F4C62EDD249C2D8827281B390B76171C
:10EF5000A9F0671708F042C0B72FB61BFF24EE24B4
:10EF60004B9F60015B9FD00CE11C1124BB27AF2D90
:10EF70009E2D8D2D280F391F7093CC073C832B833A
:10EF80005E834D83F090CE07FF2041F0EA01CE1B57
:10EF9000DF0B2C0F3D1FF80134832383BB27AA27E7
:10EFA000479FC001579F900DA11D1124492F5A2F33
:10EFB0006B2F7727241B350B832F99278535F0F48A
:10EFC00080E090E0E8018A83892B49F1F894509120
:10EFD0006500526050936500789421C0671BFF2440
:10EFE000EE24469F6001569FD00CE11C1124BB27E4
:10EFF000AF2D9E2D8D2D281B390BBECF8C3A60F482
:10F00000A0913C08B0913D081196B0933D08A093A3
:10F010003C08F8015483438380E890E0D3CF0E94FA
:10F02000F220DF91CF911F910F91FF90EF90DF9031
:10F03000CF900895CF92DF92EF92FF920F931F939C
:10F04000CF93DF931092C8079498F89410916500BD
:10F050001C7F1093650078940BB30F70402F0BBB8F
:10F06000D09056063D2D32953F70932F9A95F1F72B
:10F07000949A2D2D2F70C22ECA94F1F7949882E0A5
:10F0800090E082959295907F9827807F9827482BD3
:10F090004BBB3A95F1F7949A2A95F1F794980CECBA
:10F0A00017E0F8948091D3079091D407409188009D
:10F0B000509189005093D4074093D30748175907BC
:10F0C00048F4A091D507B091D6071196B093D60712
:10F0D000A093D5077894E091D107F091D207709171
:10F0E000CD076091CC07CCECD7E02091CF073091D1
:10F0F000D0074E175F0730F4C62EDD249C2D8827DD
:10F10000281B390B7617A9F0671708F042C0B72FF4
:10F11000B61BFF24EE244B9F60015B9FD00CE11CCB
:10F120001124BB27AF2D9E2D8D2D280F391F7093D5
:10F13000CC073C832B835E834D83F090CE07FF206A
:10F1400041F0EA01CE1BDF0B2C0F3D1FF801348389
:10F150002383BB27AA27479FC001579F900DA11D5E
:10F160001124492F5A2F6B2F7727241B350B832F00
:10F1700099278535F0F480E090E0E8018A83892BB7
:10F1800049F1F8945091650052605093650078946D
:10F1900021C0671BFF24EE24469F6001569FD00CC0
:10F1A000E11C1124BB27AF2D9E2D8D2D281B390B63
:10F1B000BECF8C3A60F4A0913C08B0913D08119606
:10F1C000B0933D08A0933C08F8015483438380E842
:10F1D00090E0D3CF0E94F2201092C907DF91CF9127
:10F1E0001F910F91FF90EF90DF90CF900895CF92F5
:10F1F000DF92EF92FF920F931F93CF93DF9398E0EC
:10F20000813009F4D2C0613009F4CDC0413009F435
:10F21000C8C09498F894109165001C7F1093650005
:10F2200078944BB34F70092F007F042B0BBBD09009
:10F2300056063D2D32953F70E32EEA94F1F7949AED
:10F240002D2D2F70C22ECA94F1F79498892F9927EB
:10F2500082959295907F9827807F9827482B4BBB6B
:10F260003A95F1F7949A2A95F1F794980CEC17E0F7
:10F27000F8948091D3079091D407409188005091E1
:10F2800089005093D4074093D3074817590748F48F
:10F29000A091D507B091D6071196B093D607A09349
:10F2A000D5077894E091D107F091D2077091CD07FE
:10F2B0006091CC07CCECD7E02091CF073091D007FC
:10F2C0004E175F0730F4E62EFF24DE2CCC242C19D9
:10F2D0003D097617A9F0671708F042C0972F961BD3
:10F2E000FF24EE24499F6001599FD00CE11C11249A
:10F2F000BB27AF2D9E2D8D2D280F391F7093CC0766
:10F300003C832B835E834D83F090CE07FF2041F03A
:10F31000EA01CE1BDF0B2C0F3D1FF8013483238342
:10F32000BB27AA27479FC001579F900DA11D1124FD
:10F33000492F5A2F6B2F7727241B350B832F9927A3
:10F340008535F0F480E090E0E8018A83892B79F13B
:10F35000F89450916500526050936500789427C0EE
:10F36000671BFF24EE24469F6001569FD00CE11CD2
:10F370001124BB27AF2D9E2D8D2D281B390BBECF01
:10F380008C3A60F4A0913C08B0913D081196B0937E
:10F390003D08A0933C08F8015483438380E890E043
:10F3A000D3CF916036CF926031CF9CE02CCF0E94BA
:10F3B000F220DF91CF911F910F91FF90EF90DF909E
:10F3C000CF900895CF92DF92EF92FF920F931F9309
:10F3D000CF93DF93982F90689498F89410916500DC
:10F3E0001C7F1093650078944BB34F70092F007FFA
:10F3F000042B0BBBD09056063D2D32953F70E32E6B
:10F40000EA94F1F7949A2D2D2F70C22ECA94F1F739
:10F410009498892F992782959295907F9827807F3D
:10F420009827482B4BBB3A95F1F7949A2A95F1F718
:10F4300094980CEC17E0F8948091D3079091D4073E
:10F4400040918800509189005093D4074093D3078E
:10F450004817590748F4A091D507B091D6071196DF
:10F46000B093D607A093D5077894E091D107F09197
:10F47000D2077091CD076091CC07CCECD7E02091FA
:10F48000CF073091D0074E175F0730F4E62EFF24E8
:10F49000DE2CCC242C193D097617A9F0671708F04B
:10F4A00042C0972F961BFF24EE24499F6001599F6D
:10F4B000D00CE11C1124BB27AF2D9E2D8D2D280FC4
:10F4C000391F7093CC073C832B835E834D83F09070
:10F4D000CE07FF2041F0EA01CE1BDF0B2C0F3D1FB2
:10F4E000F80134832383BB27AA27479FC001579F76
:10F4F000900DA11D1124492F5A2F6B2F7727241B04
:10F50000350B832F99278535F0F480E090E0E801F2
:10F510008A83892B49F1F894509165005260509389
:10F520006500789421C0671BFF24EE24469F60018C
:10F53000569FD00CE11C1124BB27AF2D9E2D8D2D85
:10F54000281B390BBECF8C3A60F4A0913C08B091D7
:10F550003D081196B0933D08A0933C08F8015483F0
:10F56000438380E890E0D3CF0E94F220DF91CF91D7
:10F570001F910F91FF90EF90DF90CF900895AF9281
:10F58000BF92CF92DF92EF92FF921F93CF93DF93C0
:10F59000182F8C3308F4ADC0982F985E906894981B
:10F5A000F894609165006C7F6093650078944BB32C
:10F5B0004F70592F507F542B5BBBB09056063B2D9C
:10F5C00032953F70C32ECA94F1F7949A2B2D2F7069
:10F5D000A22EAA94F1F79498892F99278295929553
:10F5E000907F9827807F9827482B4BBB3A95F1F75F
:10F5F000949A2A95F1F79498BCECEB2EB7E0FB2E89
:10F60000F8948091D3079091D4074091880050914D
:10F6100089005093D4074093D3074817590748F4FB
:10F62000A091D507B091D6071196B093D607A093B5
:10F63000D5077894E091D107F091D2077091CD076A
:10F640006091CC07CCECD7E02091CF073091D00768
:10F650004E175F0730F4C62EDD24BC2CAA242A19CD
:10F660003B097617A9F0671708F048C0972F961B3B
:10F67000DD24CC24499F5001599FB00CC11C11249A
:10F68000BB27AD2D9C2D8B2D280F391F7093CC07D8
:10F690003C832B835E834D83D090CE07DD2041F0E9
:10F6A000EA01CE1BDF0B2C0F3D1FF70134832383B0
:10F6B000BB27AA27479FC001579F900DA11D11246A
:10F6C000492F5A2F6B2F7727241B350B832F992710
:10F6D000853548F580E090E0E7018A83892B09F4BD
:10F6E00035C0F894709165007260709365007894ED
:10F6F0002DC0883298F0982F945150CF671BDD248D
:10F70000CC24469F5001569FB00CC11C1124BB272E
:10F71000AD2D9C2D8B2D281B390BB8CF8431A0F03B
:10F72000982F945D3BCF8C3A60F4A0913C08B09147
:10F730003D081196B0933D08A0933C08F70154830F
:10F74000438380E890E0C8CF982F28CF0E94F22012
:10F750001093C707DF91CF911F91FF90EF90DF903B
:10F76000CF90BF90AF900895AF92BF92CF92DF92AB
:10F77000EF92FF920F931F93CF93DF93F090550674
:10F78000F0FE98C0F89438E03ABB94981091650068
:10F790001D7F116010936500789400915606902F9C
:10F7A00092959F70A92EAA94F1F7949A0F70202F2A
:10F7B0002A95F1F7E9B294989A95F1F7949A0A95F7
:10F7C000F1F794980CEC17E0F8948091D30790919E
:10F7D000D40740918800509189005093D4074093FA
:10F7E000D3074817590708F4F3C17894E091D1077B
:10F7F000F091D2077091CD076091CC07CCECD7E0A7
:10F800002091CF073091D0074E175F0730F4A62E16
:10F81000BB249A2D8827281B390B7617A9F0671768
:10F8200008F0E2C1B72FB61BDD24CC244B9F50015A
:10F830005B9FB00CC11C1124BB27AD2D9C2D8B2DC3
:10F84000280F391F7093CC073C832B835E834D8335
:10F85000B090CE07BB2041F0EA01CE1BDF0B2C0F8E
:10F860003D1FF80134832383BB27AA27479FC0018C
:10F87000579F900DA11D1124492F5A2F6B2F7727C9
:10F88000241B350B832F9927853508F0C5C180E0EF
:10F8900090E0E8018A83892B09F4B9C1F89480913A
:10F8A00065008E7F82608093650048EF4ABB789444
:10F8B000E7FC30C21091C807512F569556955695C2
:10F8C000A52FBB27A354B84FC12FDD27FE01E7703A
:10F8D000F070EF53F74E94914C91D42ED9222D2DE8
:10F8E000332727FD3095222309F4BCC02091C70798
:10F8F000211709F4D4C11C3308F086C1183208F46A
:10F90000FBC1912F945190689498F894B091650040
:10F91000BC7FB093650078940BB30F70392F307FA4
:10F92000302B3BBBF0905606FF2DF295FF702F2F2A
:10F930002A95F1F7949A7F2D7F70E72EEA94F1F7DC
:10F940009498892F992782959295907F9827807F08
:10F950009827082B0BBBFA95F1F7949A7A95F1F753
:10F960009498BCECEB2EB7E0FB2EF8946091D30793
:10F970007091D40740918800509189005093D4072A
:10F980004093D3074617570748F48091D5079091C5
:10F99000D60701969093D6078093D5077894E09187
:10F9A000D107F091D2077091CD076091CC07CCECD4
:10F9B000D7E02091CF073091D0074E175F0730F482
:10F9C000862F9927B82EAA242A193B097617A9F061
:10F9D000671708F081C1972F961BDD24CC24499F1F
:10F9E0005001599FB00CC11C1124BB27AD2D9C2D7B
:10F9F0008B2D280F391F7093CC073C832B835E839C
:10FA00004D83B090CE07BB2041F0DA01AE1BBF0B97
:10FA10002A0F3B1FE7013C832B83BB27AA27479F65
:10FA2000C001579F900DA11D1124492F5A2F6B2FF4
:10FA30007727241B350B832F9927853508F01EC1A6
:10FA400080E090E0F7018283892B39F0F8944091AF
:10FA5000650042604093650078940E94F220109304
:10FA6000C70758C1912F9F5E9695969596958AE007
:10FA7000981708F0B7C0E92FFF27E354F84FE0814B
:10FA8000EE2371F4815009F441C19F5F9A3098F3DD
:10FA900090E0E92FFF27E354F84FE081EE2391F344
:10FAA000990F990F990F1E2F107F19F49C5FE29503
:10FAB000E07F5E2F507C19F49E5FEE0FEE0FE7FFA4
:10FAC0009F5F9093C807F894709165007D7F709355
:10FAD000650078940E94F2200CEC17E0F894609195
:10FAE000D3077091D40740918800509189005093BA
:10FAF000D4074093D3074617570748F4A091D5077A
:10FB0000B091D6071196B093D607A093D5077894F5
:10FB1000E091D107F091D2077091CD076091CC07A9
:10FB2000CCECD7E02091CF073091D0074E175F077C
:10FB300030F4A62EBB24DA2CCC242C193D097617E0
:10FB4000A9F0671708F08AC0F72EF61ADD24CC2436
:10FB50004F9D50015F9DB00CC11C1124BB27AD2DE2
:10FB60009C2D8B2D280F391F7093CC073C832B8342
:10FB70005E834D83D090CE07DD2041F0DA01AE1BCD
:10FB8000BF0B2A0F3B1FE8013C832B83DD24CC24D1
:10FB9000479F5001579FB00CC11C112477276D2D32
:10FBA0005C2D4B2D241B350B832F9927853508F0B1
:10FBB00044C080E090E0E8018A83892B09F4AAC060
:10FBC000F894F0916500F260F09365007894A2C01B
:10FBD000A091D507B091D6071196B093D607A09300
:10FBE000D50703CE922F47CF671BDD24CC24469F39
:10FBF0005001569FB00CC11C1124BB27AD2D9C2D6C
:10FC00008B2D281B390B1ECE912F985E7CCEF8943D
:10FC1000809165008C7F47CE8C3A60F4A0913C08BF
:10FC2000B0913D081196B0933D08A0933C08F801AF
:10FC30005483438380E890E02CCE8C3A60F480912A
:10FC40003C0890913D08019690933D0880933C08B4
:10FC5000F8015483438380E890E0ADCF671BFF2415
:10FC6000EE24469F6001569FD00CE11C1124BB2757
:10FC7000AF2D9E2D8D2D281B390B76CF8C3A60F43D
:10FC8000C0913C08D0913D082196D0933D08C09387
:10FC90003C08F7015483438380E890E0D3CE9095ED
:10FCA00049234C93C459D84FE981812F8F5F803508
:10FCB00040F11092C807F1FC08C0822F8F5F843199
:10FCC00021F0883211F08C3309F48FEF8093C7074D
:10FCD0008E2F0E94C6721EC0671BDD24CC24469F57
:10FCE0005001569FB00CC11C1124BB27AD2D9C2D7B
:10FCF0008B2D281B390B7FCE143130F0912F945D62
:10FD000002CE8093C807D7CF912FFDCD990F990FC1
:10FD1000990FD7CEDF91CF911F910F91FF90EF9068
:10FD2000DF90CF90BF90AF9008958093C90708955A
:10FD30008091C90799270895CF93DF93982FE09179
:10FD4000C9078E2F8F5F8035E8F01092C9072E2FDC
:10FD50003327D901A459B84FED0189818917A9F03A
:10FD60009983E695E695E695CE2FDD27C354D84FC7
:10FD7000277030702F53374EF90194912881292B29
:10FD8000288303C08093C907E2CFDF91CF91089504
:10FD9000CF93DF93AC01EC019881992319F52BC027
:10FDA0001092C9072E2F3327D901A459B84FED015E
:10FDB0008981891789F09983E695E695E695CE2F96
:10FDC000DD27C354D84F277030702F53374EF901B9
:10FDD00094912881292B28834F5F5F4FFA019081EE
:10FDE000992349F0E091C9078E2F8F5F8035C0F6C7
:10FDF0008093C907D7CFDF91CF910895CF93DF9339
:10FE0000FC01AC014F5F5F4F9491992371F16091B8
:10FE1000C90722C060E02E2F3327D901A459B84F5B
:10FE2000ED018981891789F09983E695E695E69534
:10FE3000CE2FDD27C354D84F277030702F53374E45
:10FE4000F90194912881292B2883FA014F5F5F4F94
:10FE50003491932F332339F0E62F862F8F5F80352F
:10FE6000C8F6682FD8CF6093C907DF91CF91089566
:10FE7000CF93DF93FC01AC014F5F5F4F94919923C7
:10FE8000A1F161506F3F89F17091C90725C070E001
:10FE90002E2F3327D901A459B84FED018981891735
:10FEA00089F09983E695E695E695CE2FDD27C35434
:10FEB000D84F277030702F53374EF9019491288115
:10FEC000292B2883FA014F5F5F4F3491932F3323FF
:10FED00051F061506F3F39F0E72F872F8F5F8035EA
:10FEE000B0F6782FD5CF7093C907DF91CF910895E1
:10FEF000CF93DF93E091C9078E2F81508F3450F557
:10FF000050E220C040E02E2F3327D901A459B84F2A
:10FF1000ED016981603289F05983E695E695E695B1
:10FF2000CE2FDD27C354D84F277030702F53374E54
:10FF3000F90194912881292B2883E42F342F315003
:10FF40003F3430F48E2F8F5F8035E0F6482FDBCFC3
:10FF50004093C907DF91CF910895CF93DF93582F36
:10FF6000E091C907EE2381F18E1770F1E03560F55D
:10FF700060E222C040E02E2F3327D901A459B84FA8
:10FF8000ED018981803289F06983E695E695E695F1
:10FF9000CE2FDD27C354D84F277030702F53374EE4
:10FFA000F90194912881292B2883E42F442351F0CF
:10FFB000541740F0403530F48E2F8F5F8035D0F6E7
:10FFC000482FD9CF4093C907DF91CF910895CF93A0
:10FFD000DF93E091C907EC3370F150E54E2FE51740
:10FFE00018F136C01092C9072E2F3327D901A45912
:10FFF000B84FED018981803291F060E26983E69526
:020000021000EC
:10000000E695E695CE2FDD27C354D84F2770307084
:100010002F53374EF90194912881292B28834F5F64
:100020004517B0F4E091C9078E2F8F5F8035D0F669
:100030008093C907D9CFE83228F05CE34E2FE5174B
:1000400098F306C0E43110F058E2C8CF54E1C6CFAF
:10005000DF91CF910895CF93DF93682F50E84091BF
:10006000C90723C0E42F842F8F5F803590F1492F7B
:100070002E2F3327D901A459B84FED018981803340
:1000800091F080E38983E695E695E695CE2FDD270E
:10009000C354D84F277030702F53374EF9019491C5
:1000A0002881292B28835695C1F0962F9523D1F2CC
:1000B000E42F842F8F5F803570F040E02E2F3327A0
:1000C000C9018459984FEC017981713361F381E35F
:1000D000D9CF482FCDCF482FF1CF4093C907DF911B
:1000E000CF910895CF93DF93682F282F22952F70FB
:1000F000E22FFF27E753F74E8491482F5527942F7F
:10010000E091C9078E2F8F5F803508F449C01092A7
:10011000C9072E2F3327D901A459B84FED015981B2
:10012000591789F04983E695E695E695CE2FDD27A8
:10013000C354D84F277030702F53374EF901949124
:100140003881392B3883E62FFF27EF70F070E753A3
:10015000F74E4491E42FFF274E2F9091C907892F26
:100160008F5F803500F11092C907292F3327D901FD
:10017000A459B84FED0169816417C1F0E9839695E0
:1001800096959695C92FDD27C354D84F27703070A8
:100190002F53374EF901B49178817B2B788306C0B9
:1001A0008093C907B6CF8093C907DFCFDF91CF9186
:1001B00008951F93CF93DF93482F843608F055C0DE
:1001C0001AE0612F0E943BC5582F982F905DE09157
:1001D000C9078E2F8F5F803508F07BC08093C907D9
:1001E0002E2F3327D901A459B84FED0189818917E2
:1001F00089F09983E695E695E695CE2FDD27C354E1
:10020000D84F277030702F53374EF90194912881C1
:10021000292B2883519FC0011124642F681B605D26
:10022000E091C9078E2F8F5F803508F455C010927A
:10023000C9072E2F3327A9014459584FEA011981C4
:10024000161709F44EC06983E695E695E695AE2F3C
:10025000BB27A354B84F277030702F53374EF90186
:1002600054913C91352B3C933CC0EAEDF8E1AF0151
:100270004F5F5F4F94919923A1F16091C90722C00C
:1002800060E02E2F3327D901A459B84FED017981B1
:10029000791789F09983E695E695E695CE2FDD27C7
:1002A000C354D84F277030702F53374EF9018491C3
:1002B000B881B82BB883FA014F5F5F4F2491922F1A
:1002C000222369F0E62F862F8F5F8035C8F6682FCE
:1002D000D8CF1092C90784CF8093C907AACF609363
:1002E000C907DF91CF911F9108950F931F93CF936B
:1002F000DF93EC0183E0C83ED80708F093C004E622
:1003000010E0CE01B8010E9447C5962F905D409144
:10031000C907842F8F5F803508F0B8C08093C90764
:10032000242F3327D901A459B84FFD0181818917A2
:1003300089F09183469546954695A42FBB27A354F3
:10034000B84F277030702F53374EF90194912C918C
:10035000292B2C93609FA001619F500D709F500D21
:1003600011248E01041B150BC8016AE070E00E9485
:1003700047C5962F905DE091C9078E2F8F5F80351E
:1003800008F48AC01092C9072E2F3327D901A45927
:10039000B84FED015981591789F09983E695E69593
:1003A000E695CE2FDD27C354D84F277030702F53DA
:1003B000374EF901B49138813B2B3883FB01EE0FA6
:1003C000FF1FEE0FFF1FEE0FFF1FE60FF71FE60FD9
:1003D000F71F0E1B1F0B602F605DE091C9078E2F6A
:1003E0008F5F803508F455C01092C9072E2F332730
:1003F000C9018459984FEC010981061709F451C0CD
:100400006983E695E695E695AE2FBB27A354B84FD2
:10041000277030702F53374EF90164911C91162BC1
:100420001C933FC0EDEDF8E1AF014F5F5F4F94913A
:100430009923B9F16091C90722C060E02E2F3327BC
:1004400089010459184FE8017981791789F0998356
:10045000E695E695E695CE2FDD27C354D84F277055
:1004600030702F53374EF9012491F881F22BF88325
:10047000FA014F5F5F4F3491932F332381F0E62FC2
:10048000862F8F5F8035C8F6682FD8CF1092C907A6
:1004900047CF8093C907AACF8093C90775CF6093D0
:1004A000C907DF91CF911F910F9108958C9A809188
:1004B000640083608093640008959FEFEDEBF7E0A4
:1004C00089E09193815087FFFCCF9093C7070895EF
:1004D000CF93DF9380936C071092C8071092C907DF
:1004E0008091550683FF35C0ECECF7E0409157064C
:1004F0004093CC074093CD07F8946091D307709157
:10050000D40720918800309189003093D40720933C
:10051000D3072617370748F4A091D507B091D6071F
:100520001196B093D607A093D507C9017894DD271B
:10053000CC27249FD001349FB00DC11D11249D01F3
:10054000AE01232F342F452F5527348323839683E1
:10055000858390E2EDE6F7E08FE49193815087FF89
:10056000FCCF9FEFEDEBF7E089E09193815087FF9F
:10057000FCCF9093C7079FB7F8948C9A5091640072
:100580005360509364009498409165004C7F409371
:1005900065003AB3306F3ABB9FBFDF91CF910895AA
:1005A000CF93DF9329ED20936C071092C807109228
:1005B000C9078091550683FF33C0ECECF7E040910A
:1005C00057064093CC074093CD07F8946091D3072A
:1005D0007091D40720918800309189003093D4071E
:1005E0002093D3072617370748F4A091D507B09179
:1005F000D6071196B093D607A093D507C901789472
:10060000DD27CC27249FD001349FB00DC11D1124BC
:100610002B2F3C2F4D2F552734832383968385839F
:1006200090E2EDE6F7E08FE49193815087FFFCCFF5
:100630009FEFEDEBF7E089E09193815087FFFCCFCE
:100640009093C7079FB7F8948C9A509164005360B9
:10065000509364009498409165004C7F40936500EE
:100660003AB3306F3ABB9FBFDF91CF9108952FEF20
:100670002093C7078CEF80936C070895282F90E094
:10068000EDE6F7E0822F890F81939F5F9035D0F3DD
:100690009FEFEDEBF7E089E09193815087FFFCCF6E
:1006A0009093C7070895CF92DF92EF92FF920F9336
:1006B0001F93CF93DF9330916C07232F2F5F832FEE
:1006C0009927873F9105C9F1883F91051CF5209333
:1006D0006C07843F910509F4F1C0853F91050CF446
:1006E000E9C0853F910509F4E9C0863F910509F409
:1006F0007BC23D3F08F4A8C26091C9076F5F609359
:10070000C907662309F44EC100916C07015000939C
:100710006C079AC28A3F910509F424C18B3F910569
:100720000CF4E7C08B3F910509F45CC18C3F910547
:1007300009F440C220936C07DCCF20936C0798E249
:100740009498F894309165003C7F309365007894DC
:100750004BB34F70592F507F542B5BBBF091560613
:100760003F2F32953F70132F1A95F1F7949A2F2F40
:100770002F70722F7A95F1F79498892F9927829587
:100780009295907F9827807F9827482B4BBB3A956E
:10079000F1F7949A2A95F1F794980CEC17E0F894F5
:1007A000E090D307F090D4074091880050918900E1
:1007B0005093D4074093D3074E155F0548F4C0917A
:1007C000D507D091D6072196D093D607C093D507E9
:1007D0007894E091D107F091D2077091CD076091A4
:1007E000CC07CCECD7E02091CF073091D0074E1743
:1007F0005F0730F4E62EFF249E2D8827281B390B37
:100800007617A9F0671708F045C0972F961BFF24AD
:10081000EE24499F6001599FD00CE11C1124BB2795
:10082000AF2D9E2D8D2D280F391F7093CC073C8343
:100830002B835E834D83B091CE07BB2341F0DA0159
:10084000AE1BBF0B2A0F3B1FF80134832383BB274A
:10085000AA27479FC001579F900DA11D1124492F22
:100860005A2F6B2F7727241B350B832F992785351C
:1008700008F067C080E090E0E8018A83892B39F0B6
:10088000F8944091650042604093650078940E941E
:10089000F220DAC1671BFF24EE24469F6001569FB9
:1008A000D00CE11C1124BB27AF2D9E2D8D2D281BB4
:1008B000390BBBCF833F910509F01BCF90E3949890
:1008C000F894209165002C7F2093650078941BB3E9
:1008D0001F70912B9BBB90915606092F02950F70AC
:1008E0000A95F1F7949A892F8F708A95F1F7949869
:1008F000ABC120936C07883F910509F45EC0893F26
:10090000910509F0F6CE9498F894409165004C7FDB
:100910004093650078943BB33F70432F3BBBF0900E
:1009200056063F2D32953F70532F5A95F1F7949A02
:100930002F2D2F70E22EEA94F1F794988CE090E03E
:100940001ECF8C3A60F4E0913C08F0913D0831965E
:10095000F0933D08E0933C08E8015C834B8380E81A
:1009600090E08ACF20936C079498F894C09165002A
:10097000CC7FC09365007894BBB3BF704B2FBBBBDB
:1009800070915606372F32953F70A32FAA95F1F735
:10099000949A272F2F70622F6A95F1F7949886E02A
:1009A00090E0EDCE9FEFEDEBF7E089E09193815081
:1009B00087FFFCCF9093C70747C1C0905506C4FE80
:1009C00043C1D09057068FEF90E08D199109082E02
:1009D000892F000C881F990B000C881F991F982FD6
:1009E0009068AECE20936C079498F894309165008F
:1009F0003C7F3093650078945BB35F70152F5BBBD1
:100A000020915606022F02950F70902F9A95F1F7BC
:100A1000949AF22FFF708F2F8A95F1F7949881E0C6
:100A200090E082959295907F9827807F9827182B49
:100A30001BBB0A95F1F7949AFA95F1F794980CEC90
:100A400017E0F894E091D307F091D4074091880023
:100A5000509189005093D4074093D3074E175F07F6
:100A600048F4A091D507B091D6071196B093D60758
:100A7000A093D5077894E091D107F091D2077091B7
:100A8000CD076091CC07CCECD7E02091CF07309117
:100A9000D0074E175F0730F4862F9927F82EEE24E3
:100AA0002E193F097617A9F0671708F0B0C0B72FC5
:100AB000B61BFF24EE244B9F60015B9FD00CE11C12
:100AC0001124BB27AF2D9E2D8D2D280F391F70931C
:100AD000CC073C832B835E834D83D090CE07DD20F3
:100AE00041F0DA01AE1BBF0B2A0F3B1FE8013C832C
:100AF0002B83BB27AA27479FC001579F900DA11D9D
:100B00001124492F5A2F6B2F7727241B350B832F46
:100B10009927853508F06AC080E090E0F80182836B
:100B2000892B39F0F894409165004260409365004C
:100B300078940E94F2206FEF6093C7071092C90764
:100B4000F0905506F3FE33C0ECECF7E04091570609
:100B50004093CC074093CD07F8940091D3071091B0
:100B6000D40720918800309189003093D4072093D6
:100B7000D3072017310748F4A091D507B091D607C5
:100B80001196B093D607A093D507C9017894FF2496
:100B9000EE24249F6001349FD00CE11C11245527C2
:100BA0004F2D3E2D2D2D34832383968385831092E4
:100BB0006C074AC08091C7078F5F8093C707982F43
:100BC00096959F3708F033C030936C0780FF08CFAD
:100BD000E92FFF27E0FF2EC0EF70F070E753F74ECC
:100BE00084910E94C67230C090E269CE8C3A60F463
:100BF000C0913C08D0913D082196D0933D08C09308
:100C00003C08F8015483438380E890E087CF671B5A
:100C1000FF24EE24469F6001569FD00CE11C112456
:100C2000BB27AF2D9E2D8D2D281B390B50CF209328
:100C30006C07CCCF829586958770E82FFF27E75306
:100C4000F74E84910E94C672DF91CF911F910F9150
:100C5000FF90EF90DF90CF9008950F931F93CF9365
:100C6000DF938C01462F97FD2AC0E091C9078E2F94
:100C70008F5F803508F58093C9072E2F3327C90170
:100C80008459984FEC0169816B3291F0BBE2B983D2
:100C9000E695E695E695AE2FBB27A354B84F27708F
:100CA00030702F53374EF90174913C91372B3C93A0
:100CB0006091C907C80130C01092C907DECF90917A
:100CC000C907892F8F5F803520F58093C907292FA9
:100CD0003327D901A459B84FED0189818D3291F0A4
:100CE0005DE25983969596959695C92FDD27C35455
:100CF000D84F277030702F53374EF90194912881C7
:100D0000292B28836091C90788279927801B910B7D
:100D100003C01092C907DBCF0E94AF75DF91CF915E
:100D20001F910F910895FC01E058FF4F119211920D
:100D3000108208950F931F93CF93DF939C018A0134
:100D4000DC01A058BF4FEC91EF3138F0FC01EF57B8
:100D5000FF4F80818F5F808349C04E2F4F5F4C9340
:100D6000423090F0542F5695A52FBB27AA0FBB1FDA
:100D7000AA0FBB1FFD01E80FF91F80819181EB01D4
:100D8000C81BD90BD7FD0CC0E42FFF27EE0FFF1FA8
:100D9000EE0FFF1FE20FF31F71836083028326C0F3
:100DA000E42FFF27EE0FFF1FEE0FFF1FE20FF31FD1
:100DB000A20FB31F8D919C91119791838083ED01B8
:100DC0001A811283452F5230F8F25695A52FBB2772
:100DD000AA0FBB1FAA0FBB1FED01C20FD31F888133
:100DE0009981FB01E81BF90BDAF2CECFDF91CF91AD
:100DF0001F910F910895CF92DF92EF92FF920F9380
:100E00001F93CF93DF936C01DC01A058BF4F8C91EF
:100E1000882339F4F601EE57FF4F80818F5F80837E
:100E200064C0E82EEA94EC92EE2009F45EC0E82F4C
:100E3000FF27EE0FFF1FEE0FFF1FEC0DFD1D0081C2
:100E40001181E6011D830C83F280FE8221E0F22EE7
:100E50003DC0062F1127D801AA0FBB1FAA0FBB1F29
:100E6000AC0DBD1D472F5527EA01CC0FDD1FCC0F60
:100E7000DD1FCC0DDD1D8D919C9128813981821B58
:100E8000930B97FD2FC0AF2DBB27AA0FBB1FAA0F37
:100E9000BB1FAC0DBD1DFA01EE0FFF1FEE0FFF1FB4
:100EA000EC0DFD1D4D915C91119720813181CA019E
:100EB000821B930BD2F011963C932E935183408367
:100EC000ED019A8112811A839283F72E7F2D770F7D
:100ED000E71658F0672F6F5FE61608F0BACF472F76
:100EE0005527D1CF762FA801CECFDF91CF911F917B
:100EF0000F91FF90EF90DF90CF900895CF92DF9207
:100F0000EF92FF920F931F93CF93DF936C01F60143
:100F100075836483468391E0F92E00E810E0C00EEB
:100F2000D11EE601E880E0E8FFEFCE0EDF1E3DC0F7
:100F3000062F1127D801AA0FBB1FAA0FBB1FAC0D8C
:100F4000BD1D472F5527FA01EE0FFF1FEE0FFF1FA4
:100F5000EC0DFD1DCD91DC9120813181C21BD30BA5
:100F6000D7FD2FC0AF2DBB27AA0FBB1FAA0FBB1FDA
:100F7000AC0DBD1DFA01EE0FFF1FEE0FFF1FEC0DB4
:100F8000FD1D4D915C91119720813181CA01821B19
:100F9000930BD2F011963C932E9351834083ED0135
:100FA0009A81F280FA829283F72E7F2D770FE716CF
:100FB00058F0672F6F5FE61608F0BACF472F552716
:100FC000D1CF762FA801CECFDF91CF911F910F9176
:100FD000FF90EF90DF90CF9008959C01862F992786
:100FE000AC01B90187E891E00E949A8608950895BE
:100FF0009C0180917A01882349F0A62FBB27AD017F
:10100000B90187E891E00E949A86089541E04093F3
:101010007A01E62FFF27AF01B90187E891E00E942E
:101020007E87089580917A01882319F010927A01C1
:10103000089587E891E00E94FB8608959C01862F21
:101040009927AC01B90187E891E00E947E87089555
:10105000E1ECF8E1249180913607982F9227909344
:101060003607822311F00E94724787E891E00E94C0
:10107000FB860895E2ECF8E1249180913607982FE1
:10108000922790933607822311F00E94884787E8C1
:1010900091E00E94FB8608950E94B64780912C0340
:1010A00090912D0348E050E0BC0187E891E00E9458
:1010B0007E8708950E94C74780913303909134033F
:1010C00049E050E0BC0187E891E00E947E870895E6
:1010D00080916C0680FF02C0C79A01C0C79820911A
:1010E0000A022F7E20930A0287E891E00E94FB8685
:1010F000089590916C0690FF1FC0C79820910A0236
:10110000206120930A0280910F038330F9F030911F
:101110000F03313029F140910F03442341F490FD36
:101120001DC0C79850910A025F7E50930A0287E85B
:1011300091E00E94FB860895C79A20910A022061DF
:1011400020930A0280910F03833009F787E891E02A
:101150000E94FB8684E080930F030895C79AE2CF34
:10116000A0911B03B0911C0341E050E0BD0187E852
:1011700091E00E947E8782E080930F030895809122
:101180006C0680FF36C0C79A30910A023F7E3093CA
:101190000A022091F90224FF24C04091F9024F7EF7
:1011A0004093F90280916D0680931603A091D307B6
:1011B000B091D407E0911B03F0911C03AE1BBF0B51
:1011C00040E1BD0188EF97E00E946F8E6091F802C8
:1011D00067FD11C087E891E00E94FB8610920F0323
:1011E0000895509116035523E9F28091160381501A
:1011F000DBCFC798C9CF409103035091040360919E
:10120000050370910603CB01AA27BB270097A10510
:10121000B10501F740911703509118038091030322
:1012200090910403A0910503B09106039C01DA019B
:101230009896A217B30798F4241B350BE091D307B7
:10124000F091D407E20FF31F40E050E0BF0187E8C0
:1012500091E00E947E8773E070930F03089528E267
:1012600030E0ECCF1F93CF93DF9360915C087091D7
:101270005D086431710508F433C0DB982091600883
:101280003091610890915F08992399F0192F1150BE
:10129000E901C60FD71F45E050E0BE0187E891E0A5
:1012A0000E947E87D0936108C093600810935F0806
:1012B0001BC090915E08892F82958695877081600A
:1012C000192F1F73FF27EE27689FE001789FD00D2D
:1012D000E11D1124CE01DF01E901C80FD91FDBCFC9
:1012E00087E891E00E94FB86DF91CF911F910895DE
:1012F000EF92FF920F931F9380915C0890915D088D
:10130000809720F1DB9A0091600810916108A0910C
:10131000D307B091D407A01BB10B149641E0BD01D7
:1013200083E698E00E946F8EE0905C08F0905D0884
:10133000E00EF11E44E050E0B70187E891E00E9422
:101340007E87F0926108E092600804C087E891E02F
:101350000E94FB861F910F91FF90EF90089520E26D
:1013600020937C0080917D00806280937D0087E8DF
:1013700091E00E94FB86089520E428BF89B780642D
:1013800089BF87E891E00E94FB860895809107025B
:101390008730B0F40E940CC5BC018EE36138780739
:1013A00040F09B0131706091D3077091D407620FB8
:1013B000731F46E050E087E891E00E947E87089521
:1013C00087E891E00E94FB860895209121033091E7
:1013D00022038091D3079091D407821B930B4997E6
:1013E00008F00FC130919406232F207F3F70432FC8
:1013F00055274230510571F1433051054CF44115E8
:10140000510509F441C04130510509F0FAC070C0DE
:101410004630510509F452C04730510509F0F1C07A
:1014200027FDC4C033272077307035952795359533
:101430002795359527953595279581E090E002C051
:10144000880F991F2A95E2F7782F709583B187232B
:1014500083B9D7C027FD7CC03327207730703595FE
:10146000279535952795359527953595279581E0CD
:1014700090E002C0880F991F2A95E2F7482F409507
:1014800085B3842385BBBDC027FD79C03327207772
:101490003070359527953595279535952795359550
:1014A000279581E090E002C0880F991F2A95E2F706
:1014B000982F90958BB389238BBBA3C027FD31C098
:1014C00033272077307035952795359527953595B5
:1014D00027953595279581E090E002C0880F991FE8
:1014E0002A95E2F7682F609582B3862382BB89C074
:1014F00027FD73C0822F99278077907095958795E7
:1015000095958795959587959595879502C0440FF4
:10151000551F8A95E2F7542F509588B3852388BBD1
:1015200070C0822F992780779070959587959595B3
:101530008795959587959595879521E030E002C030
:10154000220F331F8A95E2F782B3822B82BB59C0E8
:10155000822F992780779070959587959595879597
:10156000959587959595879521E030E002C0220FEB
:10157000331F8A95E2F785B3822B85BB42C0822F49
:1015800099278077907095958795959587959595EE
:1015900087959595879521E030E002C0220F331F93
:1015A0008A95E2F78BB3822B8BBB2BC0822F9927B6
:1015B0008077907095958795959587959595879562
:1015C0009595879521E030E002C0220F331F8A9560
:1015D000E2F783B1822B83B914C0822F99278077D9
:1015E00090709595879595958795959587959595FF
:1015F000879502C0440F551F8A95E2F788B3842B64
:1016000088BB87E891E00E94FB86089587E891E017
:101610000E94FB8680912C0890912D08A0912E08A5
:10162000B0912F080196A11DB11D80932C089093B5
:101630002D08A0932E08B0932F0808951F93CF93E1
:10164000DF93109107024091D3075091D407609126
:101650008800709189006417750748F4A091D50738
:10166000B091D6071196B093D607A093D5079B01EA
:101670002F5F3F4F112349F0C0918B01D0918C0116
:10168000FE01E21BF30B0AF45AC0232F332790917B
:10169000D707921729F17093D4076093D30720934B
:1016A000D70780913A02882331F0815080933A0223
:1016B000882309F460C080911302815009F455C059
:1016C0008093130280911C0890911D0801969093BD
:1016D0001D0880931C084091D3075091D407B7CFC1
:1016E000892F8F5F112341F1282F3327F22FEE2707
:1016F000E860AE014E1B5F0B1AF0D22FCC27C560FD
:101700002091880030918900A9012617370748F4F5
:101710008091D5079091D60701969093D607809334
:10172000D5072C5F3F4FDE01A21BB30B2450304086
:10173000BB230CF48CCF22C0282F3327DECF70932D
:10174000D4076093D30790918D01892F8F70880FF4
:10175000282F33272F51374EF90145915491892F66
:1017600082958F70FA0109956CCF56E05093130261
:101770000E94C230A7CF0E940AA59DCF3093D40704
:101780002093D307D0938300C093820012E010937C
:101790007C00DF91CF911F9108951F920F920FB699
:1017A0000F9211241F932F933F934F935F936F9347
:1017B0007F938F939F93AF93BF93CF93DF93EF93D9
:1017C000FF93109107024091D3075091D407609185
:1017D0008800709189006417750748F4A091D507B7
:1017E000B091D6071196B093D607A093D5079B0169
:1017F0002F5F3F4F112349F0C0918B01D0918C0195
:10180000FE01E21BF30B0AF45AC0232F33279091F9
:10181000D707921729F17093D4076093D3072093C9
:10182000D70780913A02882331F0815080933A02A1
:10183000882309F460C080911302815009F455C0D7
:101840008093130280911C0890911D08019690933B
:101850001D0880931C084091D3075091D407B7CF3F
:10186000892F8F5F112341F1282F3327F22FEE2785
:10187000E860AE014E1B5F0B1AF0D22FCC27C5607B
:101880002091880030918900A9012617370748F474
:101890008091D5079091D60701969093D6078093B3
:1018A000D5072C5F3F4FDE01A21BB30B2450304005
:1018B000BB230CF48CCF22C0282F3327DECF7093AC
:1018C000D4076093D30790918D01892F8F70880F73
:1018D000282F33272F51374EF90145915491892FE5
:1018E00082958F70FA0109956CCF56E050931302E0
:1018F0000E94C230A7CF0E940AA59DCF3093D40783
:101900002093D307D0938300C093820012E01093FA
:101910007C00FF91EF91DF91CF91BF91AF919F91AB
:101920008F917F916F915F914F913F912F911F9177
:101930000F900FBE0F901F9018959C01462F80911D
:10194000D3079091D40760918800709189007093BB
:10195000D4076093D3076817790748F4A091D50797
:10196000B091D6071196B093D607A093D507620F12
:10197000731F242F3327A90187E891E00E949A86DC
:1019800008959C01462F8091D3079091D4076091D0
:101990008800709189007093D4076093D30768170B
:1019A000790748F4A091D507B091D6071196B09366
:1019B000D607A093D507620F731F242F3327A901E1
:1019C00087E891E00E947E8708959C01462F8091D0
:1019D000D3079091D407609188007091890070932B
:1019E000D4076093D3076817790748F4A091D50707
:1019F000B091D6071196B093D607A093D507620F82
:101A0000731F20917A01222341F0E42FFF27AF01B9
:101A100087E891E00E949A86089531E030937A0138
:101A2000842F9927AC0187E891E00E947E87089572
:101A300020B5216820BD109289001092880014BC46
:101A40001DBC1CBC80B58F7780BD08951F93CF93BC
:101A5000DF9313E010938A0080917D008260809371
:101A60007D0010927A0187E891E00E9493860E949F
:101A7000668E10928900109288001DBC1CBC1092CA
:101A8000D4071092D307109107026091D307709189
:101A9000D40720918800309189003093D407209397
:101AA000D3072617370748F4A091D507B091D6077A
:101AB0001196B093D607A093D5072F5F3F4F112300
:101AC00049F0C0918B01D0918C01FE01E21BF30B18
:101AD0000AF456C0232F33279091D7079217E9F0C5
:101AE0002093D70780913A02882331F08150809368
:101AF0003A02882309F45CC080911302815009F4F2
:101B000051C08093130280911C0890911D0801968A
:101B100090931D0880931C08B8CF892F8F5F1123E5
:101B200061F1282F3327922F88278860AE01481B48
:101B3000590B1AF0D22FCC27C5606091D307709152
:101B4000D40720918800309189003093D4072093E6
:101B5000D3072617370748F4E091D507F091D60749
:101B60003196F093D607E093D5072C5F3F4FCE0117
:101B7000821B930B0AF489CF1EC0282F3327DACF9C
:101B800090918D01592F5F70550F252F33272F51BD
:101B9000374EF90145915491892F82958F70FA0142
:101BA000099571CF76E0709313020E94C230ABCFDB
:101BB0000E940AA5A1CFD0938300C0938200B2E017
:101BC000B0937C00DF91CF911F91089521B1809156
:101BD0007B01822790E082FF0FC080917C018530DD
:101BE00018F08D3308F491E010927C0180917D0112
:101BF0008E7F80937D0114C022FD10C080917C01F6
:101C00008F3F71F08F5F80937C01883C49F4809115
:101C10007D0180FD05C092E08160EBCF90937C0157
:101C200020937B01892F9927089591B180917B01A1
:101C3000892720E082FF15C080917C01853018F053
:101C40008D3308F421E010927C0180917D018E7F1C
:101C500080937D0190937B012130D9F0223021F1D6
:101C6000089592FD10C080917C018F3F99F38F5FA2
:101C700080937C01883C71F780917D0180FDEACFE3
